:0A0000000C94E4040C9400000C942E
:10000A0000000C9400000C9400000C9400000C9466
:10001A0000000C94443D0C9400000C9400000C94D5
:10002A003B080C9400000C9400000C9400000C9403
:10003A0000000C9400000C94E9070C9400000C9446
:10004A00FE390C9400000C943E3A0C9400000C9477
:10005A0000000C9400000C9400000C9400000C9416
:10006A0000000C9400000C9400000C9400000C9406
:10007A00A53B0C9400000C94E43C0C9400000C94F6
:10008A000000000001000200040008001000200027
:10009A004000800000010002000400080010002057
:1000AA0000400080000102040810204080005F49DF
:1000BA00440000000000000000000000390D80002C
:1000CA00100000005F5273323332494400000000CE
:1000DA000000390D82001F0000005F526F746174C6
:1000EA006500000000000000390D810003000000D7
:1000FA005F54617374656E58000000000000390D8A
:10010A000100040002005F54617374656E590000B7
:10011A00000000003A0D0100060002005F44656617
:10012A0061756C744B65790000003C0D010080001C
:10013A0000002A436F6465300000000000000000E0
:10014A00430D02000F2700002A436F646531000047
:10015A000000000000003D0D02000F2700002A43A6
:10016A006F64653200000000000000003F0D0200CD
:10017A000F27D0122A4D61784D6F64756C0000000C
:10018A000000410D0100100000002A5469736368E1
:10019A004500000000000000420D000001000000C0
:1001AA005F4D795465726D4E720000000000450D76
:1001BA000100080001005F4D617374657254657235
:1001CA006D730000460D0300080001005F454D6F86
:1001DA0064650000000000000000470D03000600EF
:1001EA0000005F45437265645774720000000000A6
:1001FA005D0D01007F003F005F5273304D6F6465F3
:10020A000000000000005C0D0100030000005F56C2
:10021A0034756E643500000000000000480D0000CF
:10022A00010000005F50756C736554696D650000CC
:10023A0000005B0D010064001E005F50617573656C
:10024A0054696D6500000000900D01006400000013
:10025A005F41736B43726564697400000000490D65
:10026A000000010000005F53656E644465626974B2
:10027A00000000004A0D0000010000005F437265A3
:10028A006469744D6F64650000005A0D0100020034
:10029A0000005F4372656469744D6173746572002E
:1002AA004B0D0000010000002A5461626C65537412
:1002BA006172740000004C0D02000F2700002A54DE
:1002CA0061626C65456E6400000000004E0D02001C
:1002DA000F27E7032A4A6F6231000000000000007E
:1002EA000000500D0300080001002A4A6F62320024
:1002FA000000000000000000510D0300080000008B
:10030A002A4A6F6233000000000000000000520D0C
:10031A000300080000002A4A6F623400000000004F
:10032A0000000000530D0300080000002A4A6F6213
:10033A0035000000000000000000540D0300080012
:10034A0000002A4A6F623600000000000000000028
:10035A00550D0300080000002A4A6F6237000000AA
:10036A00000000000000560D0300080000005F4571
:10037A0072726F7231000000000000005E0D04000E
:10038A000A002E005F4572726F7232000000000090
:10039A000000680D04000A002E005F4572726F7239
:1003AA003300000000000000720D04000A002E0055
:1003BA005F4572726F7234000000000000007C0D0D
:1003CA0004000A002E005F4572726F723500000049
:1003DA0000000000860D04000A002E000000000044
:1003EA00000000000000000000000000FF00000004
:1003FA0000005461737465722020000000024C6989
:10040A00745A20202020000004044C65697454208A
:10041A0020200000080750756C732020202000005F
:10042A000C0550756C732030202000008C06546136
:10043A007374203020200000800973657269656C2E
:10044A006C200000100B73657269656C2032000025
:10045A00500C546173742032202000004003546110
:10046A007374207061720000140A466F6C676554D9
:10047A002020000018083F3F3F3F3F3F2020000058
:10048A000002FEFDFBF7EFDFBF7F50726F64756BF2
:10049A007420000053706172746520200000706F30
:1004AA007274696F6E696572656E00002E666F6C94
:1004BA0067650000506F7274696F6E656E207369AC
:1004CA00636865726E000500C11100000300D90B54
:1004DA0000000300C1110300170E0300D90B00002E
:1004EA000500E00800000A00C1110A00170E0A0000
:1004FA00D90B0A00C1110A00170E2800D90B0000F7
:10050A003000436865662D4D656E75000000310048
:10051A004B206C697374656E0000000032004B203A
:10052A006C6F65736368656E000033004B206472FC
:10053A0075636B656E000000340054206C69737437
:10054A00656E00000000350054206C6F65736368A7
:10055A00656E000036005420647275636B656E0028
:10056A000000460053797374656D000000000000B6
:10057A004100506F7274696F6E0000000000430002
:10058A004B726564697465000000000044004B7298
:10059A0065642E436C72000000004A006D616E2E85
:1005AA00506F7274696F6E00000000000000000056
:1005BA00000000000000300053797374656D00007C
:1005CA00000000003700546573740000000000004A
:1005DA0000003900506172616D6574657200000037
:1005EA00380050726F64756B746500000000420039
:1005FA004B656C6C6E657200000000004500566524
:10060A006E74696C6500000000006300436F6C6FD4
:10061A0072730000000000000000000000000000EB
:10062A000000000000004572726F72200000000096
:10063A0000000000A40D0000080000004F70742E96
:10064A0020200000000000000000A70D00000300A9
:10065A000000496D70756C732000000000000000F6
:10066A00A50D00000800000054696D654F757420DF
:10067A00000000000000A60D0000140000002E205B
:10068A002C304142433144454632474849334A4B6C
:10069A004C344D4E4F3550515236535455375657A8
:1006AA005838595A2F391027E80364000A00010004
:1006BA000010000110000100507772552000424FCF
:1006CA007574200057646F672000454570726F6D1E
:1006DA0020006C7C736368656E203F0020204B3AD3
:1006EA000020493A0020543A0025303264003E3E48
:1006FA0000430058007265616479004B20006E6502
:10070A00696E006A610053544F5000202020202057
:10071A00202020202020202000567320312E333123
:10072A0000546F74616C006B65696E204545707288
:10073A006F6D00496E697469616C697A6564004914
:10074A00442000004B230054230042450043450047
:10075A0042410044530056430043430043420023AE
:10076A00502241534349492D492F4F222C22312EE1
:10077A003030222C323030382D30312D30313B00A0
:10078A0023482245636F222C22312E3030222C320C
:10079A003030382D30312D30313B00235322456320
:1007AA006F222C22312E3030222C323030382D302C
:1007BA00312D30313B00504F00504632333B5055BB
:1007CA00002564002B302B303B00533F000066614C
:1007DA006C73636865722054697363682000546996
:1007EA0073636820766F6E204B20004665686C65DF
:1007FA0072200056656E74696C20616B74697600AC
:10080A0054696D656F757400435349204E72200018
:10081A00436F646520006B65696E204B726564697D
:10082A00740058313939313030004D42005053008C
:10083A00504C5520203A00436F6465203A005469B1
:10084A00736368203A004B656C6C6E657220004DCC
:10085A0031004F3100535000435000445900627533
:10086A007379004D50002067657370657272740069
:10087A00256400004B2300425300422100424600F7
:10088A00542300544F004952004D5A00425100422D
:10089A005200435300426600256400253032580056
:1008AA00253130640025642E253264004F4E000045
:1008BA00253032580025303458002533642E25302F
:1008CA00326400253564002564002532640025332E
:1008DA006400444400004162726563686E756E6725
:1008EA00004B656C6C6E65722000546F74616C000D
:1008FA004D6F64756C2000202000433F006E6569CF
:10090A006E006A6120200073656300496D700050B3
:10091A004C553A20005370617274653A2000507247
:10092A00313A20005072323A2000536569746520CA
:10093A003A20005479703A20003A20563A20203062
:10094A002B2030003A003A20544F3A200053703A94
:10095A00004B2066726569204A6F62204A6F6246C0
:10096A006C616773004B20006672656920004A6FEC
:10097A0062202000562020204572722050676C2089
:10098A00496D7020544F005620004B656C6C6E65A3
:10099A00723A004D49004D42004D43004D50004D02
:1009AA004C0074657374202E2E004F4E0000010017
:1009BA002D4E414E000001007E10B8090000F89447
:1009CA00EE27ECBBF1E0F5BFE5BFE0936C00F8E180
:1009DA00F1BDE1BD8DE0A2E0BB27ED938A95E9F771
:1009EA0080E090E1A0E0B1E0ED930197E9F7E0EC57
:1009FA00F9E085919591009761F0A591B5910590DF
:100A0A001590BF01F00105900D920197E1F7FB01E6
:100A1A00F0CFEFEFEDBFE0E1EEBFC0E0D5E00C9420
:100A2A00A2091A9902C0E1E00895E0E008951A9334
:100A3A00E0E0EA930E941918E1E0E093110DE0E08A
:100A4A00EA930E94391811E0153080F41A930E9433
:100A5A001918E4E6F0E0E0931B0DF0931C0D1093D7
:100A6A00150D1A930E9439181F5FEECF9FC0E881B7
:100A7A00E03011F01A9801C01A9AE8C108950E944C
:100A8A00D8380895E2E0EA930E9455510E94E83866
:100A9A0008951A930E945A51E2ECF6E00E946451BA
:100AAA00A2E0B0E00E9468510E947351E8ECF6E0BF
:100ABA000E946451A3E0B0E00E9468510E947951FB
:100ACA00EEECF6E00E946451A4E0B0E00E946851A6
:100ADA000E947F51E4EDF6E00E946451A5E0B0E087
:100AEA000E94AB5D0E9485510E948D51ECEDF6E0AB
:100AFA000E9464510E9493511E2F1D3389F4A2E073
:100B0A00B0E00E949751A3E0B0E00E949751A4E0A0
:100B1A00B0E00E949751A5E0B0E0E0E00E94B75D26
:100B2A0045C01A930E94A0510E94A0510E94893880
:100B3A000E94A551E951F84F0E94AB51E6EEF6E04A
:100B4A000E946451E091AA09EA930E943343EBEEB2
:100B5A00F6E00E946451E091E407EA930E940F4391
:100B6A000E94A0510E9473510E94A551E851F84F6A
:100B7A000E94AB51EFEEF6E00E946451E0914E07FD
:100B8A00EA930E9433430E94A0510E9479510E9425
:100B9A00A551E751F84FE0810E9485510E947F518B
:100BAA000E94A551E651F84F0E94AB511991089540
:100BBA002A970E94595FEE85E03021F4A7E0B0E061
:100BCA00E0E008C0A7E0B0E00E94AB5DEC5FEF7028
:100BDA00A7E0B0E00E94B75DE4E0EA93E3E00E9498
:100BEA0055510E94D03800E0043018F5A7E0B0E073
:100BFA000E94AB5DE00F3E2FFE013496FA93EA9312
:100C0A00E3EFF6E0FA93EA93E32FEF5F0E94AF5126
:100C1A00E02FE85FEA93E32FE0580E94B9510E945F
:100C2A00A051FE013C96FA93EA930E9469390F5F3C
:100C3A00DBCFE6E0EA93EBE20E94B951E8EFF6E097
:100C4A000E94C3510E946939E7E0EA93E1E2EA931C
:100C5A00E2E00E94C651EBEFF6E00E94C3510E9407
:100C6A0069390E94E2380E94605F2F9608950E94B7
:100C7A00CE51E0E3E0935707E4E00E94D2510E948C
:100C8A00D038E0E0EA93E091AF0DF091B00D0E9408
:100C9A00D551E3E0EA93E091AF0DF091B00D3296B1
:100CAA000E94C3510E946939E3E00E94DE51EDEFD0
:100CBA00F6E00E94C3510E94693931E00E94E35173
:100CCA000E94E65111F03F5FF9CF0E94F5513017AB
:100CDA0018F4E0E0E09394070E94F55111E00E94B5
:100CEA00FD510E94E65111F0143008F019C0E12FAD
:100CFA00A4E0EA9FF001EA930E94FD510E9400528B
:100D0A000E94D551E4E0EA930E94FD510E940052EC
:100D1A0032960E94C3510E9469390F5F1F5FDFCF6D
:100D2A000E94E2380E94605FADC00E94EE380895CA
:100D3A000E94F4380895E1E00E94D2510E94E838F6
:100D4A000E940C520E947951EFEFF6E00E94645122
:100D5A000E940C520E948D51E5E0F7E00E94645116
:100D6A00E091A8090E9411520E941B4308950E9413
:100D7A00575F40E04431B0F40E941552AE0FBF1FD6
:100D8A001196E0E0EC930E941552AE0FBF1F139626
:100D9A00EFEFEC930E941552AE0FBF1FEFEFEC93EB
:100DAA004F5FE8CF0E94E8380E9419320E945E5FC6
:100DBA0026960895E881E1506E2FA091390DE091B1
:100DCA003A0DEA9FF001E69FF001E09397090E942D
:100DDA00D038B1DF3BC0E2E00E94D251E6E00E9487
:100DEA00DE51E8E0F7E00E94C3510E946939E7E06A
:100DFA00EA93EDE3EA93E1E0EA93EAE0EA93E0E0DA
:100E0A00EA93E1E0EA93EDE0F7E00E94C3510E9421
:100E1A0069390E94E23808951A930A930E94D038D9
:100E2A001981088101C012C0239608950E94A05119
:100E3A000E947351E881EA930E941C520E94265232
:100E4A000E947351E5E1F7E00E94645121960895EA
:100E5A000E94A0510E947351EA81FB810E94645151
:100E6A00A881B981A030E0E1BE0724F40E942D5286
:100E7A000E9424430E9426520E947351E5E1F7E042
:100E8A000E94645124960895E1E00E94D2510E9482
:100E9A00E8380E941C3908951A930A930E94325224
:100EAA000E2F11E00E94A051E12F0E9411520E94C0
:100EBA0039520A930E941C520E94A0510E943D522C
:100ECA000E9439520E9440520E9489380E9445521B
:100EDA000E944A520E9451520E9414430C94B50C2B
:100EEA000E94595FE62DF0E0EF54F24FBF01E6B3DE
:100EFA00EF70A0E1EA9FF001AE2FE0B1E07FE2954A
:100F0A00EF70EA2BDB01EC93E3E0E61511F00C94A9
:100F1A00DC0720E030E010E01430E0F400E00830B4
:100F2A00B8F40E945652EF54F24FE081AE2F0E945D
:100F3A00FD51E457FB4FE491EA2BEF3F39F0E02FE4
:100F4A00EE0FEE0FE10FEF5F2E2F3F5F0F5FE7CF40
:100F5A001F5FE2CF203011F0313009F01DC0E22FBF
:100F6A000E945952E22FE1580E945F52921671F480
:100F7A00EAE0BE1608F4B394E3E0EB1531F42A93E1
:100F8A00E7E0EA930E949044882405C0E0E18E16C7
:100F9A0008F0922EBB240BC0E0E1E81508F0839418
:100FAA00EFEFEB1521F0BE2E99240E946552E62D33
:100FBA00EF5FE3706E2EE62DF0E0E457FB4FE4910D
:100FCA00E09362000C94280D0E947052E4E6E2BF9E
:100FDA00772011F019916CC07894E1E07E2E80DFC1
:100FEA00AAEDBCE00E947F520E941F450E94332056
:100FFA000E949542E091F205EF5FE093F205A0911D
:10100A00F205AE3149F4A091F105E3E8EA27E0934D
:10101A00F105E0E0E093F205E091DA0CE87011F4F2
:10102A00C79A01C0C798F894A0918C09B0918D090C
:10103A00EFEFF0E0EA27FB27EBBBE0ECE5BBE0EEE5
:10104A00E5BB0000E0918C09F0918D090E949E5C3D
:10105A00AFEFB0E0EA27FB27EBBBE0EAE5BBE0EE47
:10106A00E5BB000078947724199122C00E9470523F
:10107A000A93E6E0E4BDE0E0EABBEFEFEBBBE09108
:10108A006500EB7FE093650000000000000009B3F3
:10109A001127E0916500E460E0936500EFEFEABB99
:1010AA001A930A930E940A200E947D42099119917B
:1010BA00E991EFBFF991E991B991A9919991899132
:1010CA0079916991F990199009901895E8EFFFEFD5
:1010DA006F010E94D0380E940C520E947951E3E2BB
:1010EA00F7E00E9464510E9485520E946C5C089548
:1010FA000E942B420E94A6410E9429360E94091E84
:10110A0008951A93A8950E947244E13011F00C9444
:10111A00F708E0919A07E1501E2FA0919907A13094
:10112A0021F40E948A52E03009F411C00E948A52C6
:10113A00E093AF07ACE01A9FF001E75FFA4FBF01F7
:10114A00E081E260DB01EC931A930E949152A09134
:10115A009907A23011F0A430D1F40E948A52E09388
:10116A00B007E5E1E093AF07ACE01A9FF001DF01B9
:10117A00E050FB4FE081E03031F0FD01E75FFA4FCC
:10118A00E081E27009F403C01A930E949552A0917B
:10119A009907A33019F41A930E94A625A0919907DA
:1011AA00A53029F4E0919A07EA930E94FB25A091C1
:1011BA009907A63061F4E0919A07E093B007E091AD
:1011CA009A07EF77EF5FE0939A070E94D842A091BF
:1011DA009907A73039F4E0919A07E158E093B007EC
:1011EA000E94D842E091F105E07841F0E091F105E2
:1011FA00EF77E093F105E170EA9339DCF894E0E0E7
:10120A00EABBE0E6E5BB000000000000E9B3AFEF8F
:10121A00AE27EFE3EA23E093AA09E0EEE5BBEFEF9E
:10122A00EABB789465DF0C94F40C1A930E94D038C8
:10123A00E1E0F0E00E94C3510E94893810E00E9468
:10124A0099520E940C52E12F0E9411520E94893831
:10125A00E0919A09E03041F4EBE2F7E00E94645130
:10126A000E949F520E941443A0919A09A130B8F09B
:10127A00E0919A09E150EA930E94AA520E94B1525F
:10128A000E9440520E948938E0919A09E1500E94D6
:10129A00B5520E94BB520E94945D0E9414431E5F85
:1012AA00E0919A09EF5FE0939A09163020F4A09131
:1012BA009A09AB3008F001C0C4CF0C94F40C1A930D
:1012CA000E94D0380E94995210E01330A0F5E12F05
:1012DA00A981EA0FEA930E9419180E94A051E12FEE
:1012EA00EE0F0E9411520E948938E0919B09EA93FD
:1012FA00E12FAA81EA0FEA930E94DD180E94C052E8
:10130A000E94B1520E94A051E12FEE0FEF5F0E949E
:10131A0011520E9489380E94C5520E94CA52E8E7B7
:10132A00EA930E94FA380E94CE520E94945D0E946B
:10133A0014431F5FCACF0C94420B14B7E0E0E4BF1A
:10134A00E5BFE0936D00E0936C00EFEFEBBBEABB07
:10135A00EFE3E8BBE0E9E7BBEFEFE4BBE0E8E5BBBE
:10136A00E0EEE5BBE0E7E2BBE1BBE0E3E3B9ECE9D1
:10137A00E2B9EFEFE0936200EFE0E0936100EFE1A2
:10138A00E0936500E0936400E0E0E0BFE7E0E3BFDC
:10139A00E4E6E2BFE0E0E1BFEFBDEEBDEDBDECBDCE
:1013AA00E7BDE6BDEBBDEABDE9BDE8BDE093790066
:1013BA00E0937800E3E0E5BDE6E0E4BDE0E0E3BD0C
:1013CA00E0938B00EAE0E0938A00E0E0E093890092
:1013DA00E0938800E0938100E0938000E2E1E093EB
:1013EA008700E4E3E0938600E0E0E0938500E09381
:1013FA008400E0938300E0938200E0936A00EABFEE
:10140A00E9BFE0E4E8BFE1E4E7BFE0E0E0937D00A4
:10141A00EBB9E8EDEAB9E6E0E0939500E0E0E093A5
:10142A009000E3E3E9B9E0E0E0939B00E8EDE093A4
:10143A009A00E6E0E0939D00E0E0E0939800E3E3A1
:10144A00E0939900E0E8E8B9E0E0E0BDE0E4E7B95C
:10145A00E7E8E6B9E0B5EF7EE0BDE0E2E0937000D0
:10146A00E0E0E0937200E4E4E0937400EEE1E1BDB1
:10147A00EEE0E1BD0E945F450E94D9390E9429171A
:10148A0010FF03C0A2E0B0E00CC012FF06C0A3E048
:10149A00B0E00E94AB5D0E94D75213FF06C0A4E0E1
:1014AA00B0E00E94AB5D0E94D7520E94E152E55A19
:1014BA00F64F10830E94E152E45AF64FA9E00E94C7
:1014CA00E7520E944317E030B1F40E940C520E9486
:1014DA00F052E1E3F7E00E946451A8950E94F652A7
:1014EA00E2E3F0E00E9404530E94F652ECE2F1E0DB
:1014FA000E940453F2CF0E94F7320E940853A89523
:10150A000E940F53A8950E940853A8950E940F5352
:10151A00A8957894DBDD0E940C520E94F0520E943A
:10152A007E1AE03089F00E940C520E948D51EDE340
:10153A00F7E00E9464510E941653A8950E94165320
:10154A00A8950E941653A8950E940C520E948D518C
:10155A00E9E4F7E00E9464510E941953EA930E9459
:10156A0033430E94A7420E9486080E949F2EFBCF07
:10157A00FFCFE0E0E0937100E0937400E2B3E36030
:10158A00E2BBE3EFE1BB85E38A95F1F7E0EFE1BB6C
:10159A00E4E4E093740080E991E00197F1F708959B
:1015AA001A9314EAE4EA0E941E5341F40E94235358
:1015BA00183011F0103111F4E0E011C2E2E00FC26C
:1015CA00E4E9E0937400E0E008951A93E981E160A8
:1015DA000E94285331F40E942353103411F4E0E09E
:1015EA004CC04AC01A93E9810E94285331F40E94E0
:1015FA002353183111F4E0E040C03EC01A93E98148
:10160A000E94285331F40E942353183211F4E0E067
:10161A0034C032C01A93E981E03011F0E4EC01C021
:10162A00E4E80E941E5371F40E942353E091730070
:10163A00AA81BB81EC93103511F0183519F4E0E05A
:10164A00188103C2E1E0188100C21A93E981E0938C
:10165A00740010E0E0917400E07811F4163908F093
:10166A0005C08BE18A95F1F71F5FF4CFE091740012
:10167A00E07811F0E0E001C0E1E0188122960895D7
:10168A000E94595F3D810C8120E08ADFE03009F534
:10169A00EE810E942C53E9F43A93B0DFE030C9F4AA
:1016AA000E943153B1F47CDFE03099F4EE81EA9381
:1016BA008CDFE03071F4EDB7FEB7FA93EA931F932B
:1016CA00E0E0EA93A7DF1F91E03019F479DFE12F18
:1016DA0002C04FDFDACF0E94605F279608950E940A
:1016EA00595F30E00E811D815BDFE03099F4EF81B4
:1016FA000E942C5379F40E94315361F41A937EDFCD
:10170A00E03041F4EC81EA9379DFE03019F458DFF4
:10171A00E0E002C02EDFE8CF0E94605F28960895BD
:10172A0022970E94575F50E02B853A85A89538DFAB
:10173A00E03011F00C94FA0BEE850E942C5311F054
:10174A000C94FA0B2A935ADFE03011F00C94FA0B3E
:10175A003A9354DFE03011F00C94FA0B21DFE030B9
:10176A0011F00C94FA0BEE85EA932FDFE030E9F5DD
:10177A00E0E0EE83EF83EC85FD853197AE81BF8192
:10178A00EA17FB0751F4EDB7FEB7FA93EA931F93F2
:10179A00E0E0EA933FDF1F9109C0EDB7FEB7FA9385
:1017AA00EA931F93E1E0EA9335DF1F910E2FEE8152
:1017BA00FF81A885B985EA0FFB1F10830E94365363
:1017CA00003039F4EC85FD85AE81BF81AE17BF07C5
:1017DA0008F001C0D0CFEC85FD85AE81BF81EA1744
:1017EA00FB0719F4EDDEE0E002C0C3DEA0CF0E94E1
:1017FA005E5F2F96089568970E94575F20E0E0E0A9
:10180A00EC8FED8F31E0A895E9A1FAA16627772739
:10181A000E942E5EEA87FB876C877D87EE8D0E9489
:10182A003C53EE83FF8368877987AA85BB858C85BD
:10183A009D850E94045FEA8BFB8B6C8B7D8B0E94DB
:10184A00945DFE017296FA93EA930E942751EE8BF9
:10185A00FF8B688F798F0E9442530E94F55DAF011A
:10186A000E944253AE8DBB27882799270E949B5D11
:10187A000E945553DE015A960E94F55DED93FC9342
:10188A000AA119A18DDEE030C9F5EDA10E942C5301
:10189A00A9F50E94315391F51A93B0DEE03071F543
:1018AA00303049F14F5F5F4FEC8DFD8D3196EC8FF3
:1018BA00FD8FAC8DBD8D1197EBA1FCA1EA17FB073B
:1018CA0011F430E017C0EC8DFD8D3197AF8DB8A1C2
:1018DA000E945A5393DEEE8DDA010E945F5351F44F
:1018EA006FDEEA8DFB8DA9A1BAA1EA0FFB1FE9A35E
:1018FA00FAA38ACFD5CF64DEE0E002C03ADEC2CFD7
:10190A000E945E5FA6960895A881A03310F0AA33BC
:10191A0008F003C0E881E05318C0A881A13410F090
:10192A00A73408F003C0E881E7530FC0EFEF0DC0FA
:10193A00A881AA3018F4E881E05D07C0A881AA301E
:10194A0018F0E881E95C01C0E8E5219608951A9348
:10195A000A93F8940091DA0C1091DB0C7894F80150
:10196A000991199108951A930A93F1DF8F01EA8177
:10197A00FB810E946353E01BF10BDF010E944D5F64
:10198A0014F4E0E001C0E1E0198108812696089587
:10199A00E091BA0CEA930E948E3EE091BB0CEA9366
:1019AA000E948E3E0895F4DF0E942D520E946853D1
:1019BA000E9468530E946F53AFC31A930E94DD3D81
:1019CA001E2F103021F0E12FE150E093B80CE0DF38
:1019DA00E091B80CEF5F0E9411520E946F53199167
:1019EA0008950E94595F31E00E947553A03320F098
:1019FA000E947553A43308F025C030E00E947B533F
:101A0A00E270E6951E2F0E947B53E1700E2FA09183
:101A1A00D20C1A1729F4E1E0EA27E093D20C31E05C
:101A2A00A091D30C0A1729F0E1E0EA27E093D30C3E
:101A3A0031E0E091D30CEE0FE05DA091D20CEA0FF9
:101A4A000E948153E32F0E94605F249608951A939F
:101A5A0010E00E948753E9F10E94761BEEE4F7E05A
:101A6A000E948D53E091990D0E9411520E946F536A
:101A7A00E1E5F7E00E948D530E9491530E946F5353
:101A8A000E949853A031E7E2BE074CF4E4E5F7E080
:101A9A000E948D53E0919A0DF0919B0D13C0E7E5DA
:101AAA00F7E00E948D53E9810E949D530E9498534A
:101ABA00EA0FFB1F0E94A353E0919A0DF0919B0D30
:101ACA00E051F742FA93EA930E94C03E0E94A8535B
:101ADA0011E00E94AC53E12F1EC324970E94575F66
:101AEA000E94AC530E94A43DE13010F40C945310B0
:101AFA00E091BA0CEB3441F4E091BB0CE33219F4F7
:101B0A000E94DD3D1E2FC7C2E435B9F4E091BB0C3B
:101B1A00E33221F40E94DD3DEE83FF83E091BB0CAA
:101B2A00EF3451F40E94DD3D1E2F1A93EF81F885A0
:101B3A00FA93EA930E947B17AEC2E23411F00C9436
:101B4A00E90EE091BB0CE13259F4AA85AF3F31F4BA
:101B5A000E94B3530E94A0510E9423380E94251C60
:101B6A00E091BB0CE134D9F40E94DD3D1E2F113007
:101B7A0071F4A091AE09A13019F40E94875309F4B7
:101B8A0002C00E94811BE0E0E093FD0C08C0E1E086
:101B9A00E093FD0CDCDEE093FF0CF093000DE09186
:101BAA00BB0CE534A9F4EAE5F7E00E948D530E94E4
:101BBA005E1BF3973CF00E94DD3D0E94A3530E94F6
:101BCA00B65301C0E0E3EA930E948E3E0E94A853F6
:101BDA00E091BB0CE634E1F40E94C25319F40E946E
:101BEA00DD3DAF01E885F9850E94CE530E2F003402
:101BFA0020F0A0914B0DA13059F40E94D2530E94BB
:101C0A00441CAA85AF3F21F40E94D2530E94233874
:101C1A00E091BB0CE23511F00C94A70E0E94C2535E
:101C2A0019F40E94DD3DAF0130E0A0914B0DA030C8
:101C3A0021F40E941953E13009F023C00E94203098
:101C4A00E030F1F00E94DA53E05DF64F0E94E05373
:101C5A000E94DA53EC5CF64F0E94E5530E94DA5375
:101C6A00EE5CF64F10830E94DA53ED5CF64F408328
:101C7A000E94DA53E15DF64FA1E0A0830E94EB5384
:101C8A005FC00E941A30E23010F40C94A50E0E9434
:101C9A00F3530E941D1D3E2F3F3F29F00E94F95326
:101CAA00A417B5070CF417C00E94FE53E41BF50BEA
:101CBA000E9403540E94FE53309739F4E0E0E09307
:101CCA009E0D3A930E94AA1D03C03A930E94A31D37
:101CDA00689420F803C0E0E0E887E9870E94E152AF
:101CEA00E55AF64FDF010E940854E452F34FE081AF
:101CFA00EC930E94E152E35AF64F0E94E0530E948D
:101D0A00E152EF59F64F0E94E5530E94E152E15A1F
:101D1A00F64F10830E94E152E45AF64FA5E00E9462
:101D2A00E752E885F985309759F00E94F353FA0192
:101D3A000E94815C0E940B540E94D2530E94D01BC5
:101D4A00689422F8E091BB0CE335E9F50E94DD3D89
:101D5A00E887F9870E940F54DF01E45AF64FE081C1
:101D6A00E23079F4FD01EF59F64F008011800E94AC
:101D7A001953D0010E945F5321F4A091AE09A230F9
:101D8A0009F01FC00E940F54E35AF64FDF010E9468
:101D9A00815DDF01E885F985EA17FB0779F40E947E
:101DAA000F54DF01ED59F64FE081EA93FD01E55A40
:101DBA00F64FE081EA930E94482403C0E7E0E093EB
:101DCA00E307689422F867C1E43411F00C94520FC7
:101DDA00E091BB0CE33559F4EDE5F7E00E948D5331
:101DEA000E949C3A0E941554E1E0E093B10AE09106
:101DFA00BB0CE03511F00C94510F0E941954E030DD
:101E0A0011F40C94510F20E00E947553A03240F057
:101E1A000E947553A23221F00E947553AB3309F424
:101E2A003BC0E22FE03061F40E947553A33211F4F3
:101E3A0021E005C00E947B53EA930E94773A29C0A9
:101E4A00E13049F40E947553A43211F422E001C032
:101E5A0020E010E01EC0E23011F0E330D1F40E941D
:101E6A007B53EA9351DDEF3F99F0E12FE295E07F52
:101E7A00EF930E947B53EA9347DDAF91EA0F1E2F3F
:101E8A002F5F243021F41A930E94773A20E001C090
:101E9A0020E00E941D54B8CFFEC0E63511F00C9424
:101EAA00C90FE091BB0CE33429F50E94DD3D1E2FDA
:101EBA00E091EF07E030C9F0E0E6F7E00E948D53C9
:101ECA00E091EF07E0580E9411520E942054E091DD
:101EDA00F207F091F307FA93EA930E942054E091F3
:101EEA00F407F091F5070E942654113019F0E0E04A
:101EFA00E093EF07E091BB0CE33511F00C94C80FA7
:101F0A00E0E0EA930E94641AE0E0E093010D0E9487
:101F1A00DD3DE093150D0E942954A9F50E94DD3D8F
:101F2A00E093180D0E94295471F50E94DD3D1E2F81
:101F3A00103019F0E1E0E093120D0E94295419F5CE
:101F4A000E94DD3DE0931B0DF0931C0D0E94295465
:101F5A00D1F40E94DD3DE093210D0E94295499F4A9
:101F6A000E942F541E2FE0E0EA931A930E944824FD
:101F7A00E03049F4E0E6F7E00E948D53E12F0E9439
:101F8A0011520E946F5387C0E33411F00C94501021
:101F9A00E091BB0CE534B9F4EAE5F7E00E948D5311
:101FAA000E945E1BF3974CF00E94DD3DE05FF84D06
:101FBA000E94A3530E94B65301C0E0E3EA930E9431
:101FCA008E3E0E94A853E091BB0CE634B1F441E086
:101FDA0050E00E94DD3D0E2F0E94295419F40E9400
:101FEA00DD3DAF011A930E94FD51E05FF84DFA936F
:101FFA00EA935A934A930E94441CE091BB0CE3353E
:10200A0069F50E94DD3D3197E887F9870E942954D6
:10201A0019F40E94DD3DAF01E8850E94345431F481
:10202A00E091010DEA930E942C1718C0E885EA9303
:10203A00FA01E058FF4FEA930E944824E03041F445
:10204A00E3E6F7E00E948D535A934A930E946F5336
:10205A00E885EA93EFEFEA930E944824E091BB0CEB
:10206A00E134C9F4E6E6F7E00E948D530E94DD3DB3
:10207A003197E887F987E885EA930E9419180E9440
:10208A007723E03011F0E1E301C0E0E3EA930E9434
:10209A008E3E0E94A8530E945B3D24CD0E945E5F43
:1020AA002B960895A091D00CA03529F4E091D10C7B
:1020BA00EA930E943918A091D00CA33529F4E09133
:1020CA00D10CEA930E946818A091D00CAB3429F481
:1020DA00E091D10CEA930E94A418A091D00CA635E5
:1020EA0029F4E091D10CEA930E94C818A091D00C6F
:1020FA00A43511F40E9465170E943B5408951A935F
:10210A0010E0103440F40E945652E25DF74FA98164
:10211A00A0831F5FF6CF1881229608950E94575F09
:10212A000E94A43DE13010F40C94D113E091D00C3C
:10213A00A091BA0CEA1709F0B5DFE091BA0CE332C4
:10214A0059F5E091BB0CEC3441F4E0E0EA93D7DFB7
:10215A00E4E0E09390090E944154E091BB0CE4351D
:10216A00D1F4E0E0EA93CBDFE091B70DE03029F05B
:10217A00EF77A1E0B0E00E94B75DE091B80DE030E2
:10218A0029F0EF77A6E0B0E00E94B75D0E944154C3
:10219A00E7E0E093900904C0EB3411F00C941A11B3
:1021AA00E091BB0CE13221F4EBE4EA93A8DF3CC0F6
:1021BA00E53211F477DF38C0E332D9F40E9447548C
:1021CA0031F00E9452540E9472180E9458540E9480
:1021DA005D54E081EB3461F4E0E0E093A90DE09313
:1021EA00AA0D0E945D54A0E0A083EBE4E093D00C1A
:1021FA001BC0E134C9F4EBE4E093D00CA091B80C15
:10220A00A03890F40E94DD3D9F012093A90D0E9401
:10221A00635451F00E94DD3D9F010E94635421F0F6
:10222A000E94DD3DE093AA0DB4C2E33511F00C948F
:10223A006111E091BB0CE13221F4E3E5EA935FDF3F
:10224A003AC0E332D9F40E94475431F00E94525402
:10225A000E944A180E9458540E945D54E081E33556
:10226A0061F4E091B80CEA930E94501A0E945D54FE
:10227A00A0E0A083E3E5E093D00C1DC0EE34D9F4CE
:10228A00E3E5E093D00CA091B80CAA30A0F4EAE000
:10229A00EA930E94663E10E01A3068F4ABE2BDE0B1
:1022AA00EE27A10FBE1F0E945652E454F34FE0815D
:1022BA00EC931F5FF1CF6DC2E63511F00C94B711A4
:1022CA00E091BB0CE13221F4E6E5EA9318DF49C05C
:1022DA00E332D9F40E94475431F00E9452540E94CA
:1022EA00B0180E9458540E945D54E081E63561F4AA
:1022FA00E091B80CEA930E94D5180E945D54A0E0C0
:10230A00A083E6E5E093D00C2CC0E63531F40E94B8
:10231A00DD3D9F012093A50D24C0E53471F40E9490
:10232A00DD3D9F012093A40D0E94635429F00E9471
:10233A00DD3D9F012093A70D14C0E43591F440E0E0
:10234A0050E00E94DD3D9F01022E032A11F042E077
:10235A0050E00E94635419F00E94DD3DAF014093A2
:10236A00A60D17C2E43511F00C948A12E091BB0C49
:10237A00E33231F40E94DD3D3197E093B80CC4C0DA
:10238A00E03511F00C94891210E00E947553A032C6
:10239A0050F00E947553AD3331F00E947553AB3340
:1023AA0011F01E3008F00DC00E945652E454F34F4B
:1023BA000F010E947B53D001EC931F5F0E941D54B2
:1023CA00E4CF0E9456520E946954EDE30E946E5473
:1023DA0011F00C948912E4E5E093D00C10E00E940D
:1023EA00735470960E94905DEF3FA0E0FA0711F4D3
:1023FA000C9489120E9479540E947354FA93EA93B6
:10240A000E94134FE03011F00C9487120E9473540B
:10241A000E947E5441F40E942F54E093B70DE0E8E5
:10242A00E093B80D6FC0E238A0E0FA0729F40E94E1
:10243A002F54E093B80D66C0E138A0E0FA0739F4EA
:10244A000E94DD3DA0E0B0E00E94B75D5BC030971E
:10245A0021F0E130A0E0FA0769F40E9473543E9635
:10246A000E94905DFF93EF930E94DD3DAF91BF9173
:10247A00EC9348C0E230A0E0FA0771F40E9473546A
:10248A003E960E94905DFF93EF930E94DD3DAF91CF
:10249A00BF91ED93FC9336C0E330A0E0FA0769F4EC
:1024AA000E9473543E960E94905DFF93EF930E94A0
:1024BA00BE3DAF91BF91EC9325C0E430A0E0FA078E
:1024CA0009F50E9473547296E491EA930E94663E5B
:1024DA000E9473540E94855400E00E9473540E9423
:1024EA008D5484F40E94FD51E454F34FE081A0918D
:1024FA00B50DB091B60DEC93A5EBBDE00E947F52ED
:10250A000F5FEBCF1F5F6BCF44C1E03511F00C9426
:10251A00CE13E091BB0CE332D1F40E94475431F060
:10252A000E9452540E9419180E9458540E945D54E5
:10253A00E081E03561F4E091B80CEA930E94641AF4
:10254A000E945D54A0E0A083E0E5E093D00CE09106
:10255A00BB0CE33221F0A091B80CA03408F019C1E9
:10256A00E0E5E093D00CE091BB0CE13221F4E0E528
:10257A00EA93C5DD0EC1E134C1F40E94DD3D1E2F90
:10258A0000E00C3088F40E9495543B96E491E117E0
:10259A0049F40E9495543A96E491A091120DEA2BBF
:1025AA00E093120D0F5FEDCFF4C0E63559F5E0E088
:1025BA00E093B90C0E949B54EA0FFB1FFF93EF9321
:1025CA000E94DD3DAF91BF91EC93EBE2EA930E944A
:1025DA006E3DE03059F00E94A154EA0FFB1FFF93B1
:1025EA00EF930E94DD3DAF91BF91EC930E94A754F7
:1025FA00A091B90CA33018F40E94635409F401C0E5
:10260A00D9CFC7C0ED34D1F4E0E0E093B90C0E9411
:10261A00AD54EA0FFB1FFF93EF930E94DD3DAF918C
:10262A00BF91EC930E94A754A091B90CA33018F45F
:10263A000E94635409F401C0EACFABC0E434C9F57F
:10264A00E0E0E093B90C0E94DD3D9F01E2E0EA93ED
:10265A000E947B3DAF01E3E70E946E5469F40E9439
:10266A00B354BF01D901E4E6F0E00E94E15CE40F53
:10267A00F51FDB01ED93FC93E9E40E946E5469F4C3
:10268A000E94B354208331830E94BD54EA0FFB1F7A
:10269A000F010E94BD540E94C3540E94A754A091E6
:1026AA00B90CA33018F40E94635409F401C0CBCFCB
:1026BA0070C0EE34A9F4EAE0EA930E94663E10E0A4
:1026CA001A3068F4A2E0BDE0EE27A10FBE1F0E94F7
:1026DA005652E454F34FE081EC931F5FF1CF59C097
:1026EA00E33449F40E9419540E94DD3DE0930D0D34
:1026FA00F0930E0D4EC0E33589F40E94DD3D9F0133
:10270A0000240216030624F42B30E0E03E070CF006
:10271A0004C0F9013197E0930F0D3BC0E53529F468
:10272A000E94DD3DE093110D34C0EF3491F40E9414
:10273A00DD3D1E2FECE2EA930E946E3DE12FE29509
:10274A00E07FEF930E94DD3DAF91EA0FE093100D19
:10275A0020C0E035F1F4E0E0E093B90CA4E2BDE07A
:10276A000E94CA540E94CE54FF93EF93E2E0EA9388
:10277A000E94283EAF91BF91ED93FC930E94A7540B
:10278A00A091B90CA23018F40E94635409F401C054
:10279A00E5CF0E945B3DC4CCE0E0E093BB0B0E9416
:1027AA005E5F269608950E94595F0E94A43DE1301B
:1027BA0010F40C945D16E091BA0CE332A9F4E0919E
:1027CA00BB0CE03519F4E9E6F7E009C0E83419F47E
:1027DA00EAE8F7E004C0E33531F4E5EAF7E0FA9312
:1027EA00EA930E949F3E61C2E43511F00C949E1454
:1027FA00E091BB0CE43229F4E5E2F0E00E94D35404
:10280A0097C0E33211F4D9D893C0E03511F00C9493
:10281A009D14BED8A091B80CA53210F00C949D144A
:10282A000E94D7540E948D53EDE3EA930E948E3E94
:10283A000E94D7540E947E5439F40E9419530E9470
:10284A0011520E94C03E74C0E238A0E0FA0739F47F
:10285A000E94DF540E9411520E94C03E69C0E138B2
:10286A00A0E0FA0739F40E94E4540E9411520E942F
:10287A00C03E5EC0309721F0E130A0E0FA0759F47B
:10288A000E94D7543E960E94905DE0810E941152A8
:10289A000E94C03E4DC0E230A0E0FA0759F40E94FF
:1028AA00D7543E960E94905DDF010E94E9540E942F
:1028BA00C03E3EC0E330A0E0FA0751F40E94D7546C
:1028CA003E960E94905DE081EA930E94CE3E30C01F
:1028DA00E430A0E0FA0761F50E94D7540E948554BB
:1028EA0010E00E94D75472960E94905D0E94EE54A6
:1028FA00AE17BF0794F40E945652E454F34F0F01E7
:10290A00A091B50DB091B60DEC91D001EC93A5EB69
:10291A00BDE00E947F521F5FE4CF0E94D754729697
:10292A000E94905D0E9469540E9479540E942F3F30
:10293A00BCC1E33569F5E091B80CEA930E944A18E4
:10294A00E091BB0CE43229F4EAE0F0E00E94D354AF
:10295A001EC0E33211F431D81AC0EE34C1F418D8CB
:10296A0010E01A3058F40E945652E454F34F0F0103
:10297A00ABE2BDE00E94F1541F5FF3CFE0E0E093C9
:10298A00C60C0E9479540E942F3F0E94A8538DC101
:10299A00E63511F00C940E15E091B80CEA930E94FA
:1029AA00B018E091BB0CE43229F4E8E0F0E00E94B0
:1029BA00D3542EC0E33219F40E94E20C29C0E53444
:1029CA0059F40E94CD0CE091A40D0E9411520E946C
:1029DA00F854E091A70D19C0E63529F40E94CD0CF0
:1029EA00E091A50D12C0E43599F40E94CD0CE09156
:1029FA00A60DE03011F0E1E301C0E0E3EA930E94A2
:102A0A008E3E0E94FE54E091A60DF0E00E942654EC
:102A1A004CC1E03511F00C943016E091B80CEA93F1
:102A2A000E941918E091BB0CE43229F4E0E4F0E0CA
:102A3A000E94D3540FC1E33219F40E94E20C0AC176
:102A4A00E13411F00C9468150E94CD0C12E0A091AB
:102A5A00120DECEDEA233E2F00E00C3068F40E94E0
:102A6A0095543A96E491E31729F40E9495543B96BB
:102A7A00149102C00F5FF1CFE12F0E9411520E9400
:102A8A006F53E091100DE03079F0E0ECF7E00E942E
:102A9A008D530E9402550E94F854E091100DEF7078
:102AAA000E9411520E946F53E091110DE03051F0D3
:102ABA00E3ECF7E00E948D53E091110D0E94115250
:102ACA000E946F53C7C0E43479F50E940755A0915C
:102ADA00B90CA33040F5E091B90CE03011F00E9436
:102AEA00FE540E94BD54AE0FBF1FEC91E17051F429
:102AFA00ABE1BDE00E94CA540E944A520E940D55A1
:102B0A00E3E70BC0ABE1BDE00E94CA540E944A52FF
:102B1A00FA93EA930E94C03EE9E4EA930E948E3E49
:102B2A000E94A754D4CF92C0ED34B1F40E94075545
:102B3A00A091B90CA33078F4E091B90CE03011F00F
:102B4A000E94FE540E94AD540E9411550E94C03E3C
:102B5A000E94A754EDCF7AC0E63501F50E940755C9
:102B6A00A091B90CA330C8F4E091B90CE03011F08F
:102B7A000E94FE540E949B540E9411550E94C03E1E
:102B8A00EBE2EA930E948E3E0E94A1540E941155E4
:102B9A000E94C03E0E94A754E3CF58C0EE34C1F44D
:102BAA000E94CD0C10E01A3058F40E945652E45498
:102BBA00F34F0F01A2E0BDE00E94F1541F5FF3CF73
:102BCA00E0E0E093C60C0E9479540E942F3F3EC079
:102BDA00E33499F40E94CD0C0E947954EBECF7E0AF
:102BEA00FA93EA930E9415550E9451520E941A556F
:102BFA000E9479540E942F3F29C0E03579F40E943F
:102C0A00CD0C0E941F550E940D550E94FE54E09162
:102C1A00260DF091270D0E940D5518C0E33531F4A9
:102C2A000E94CD0CE0910F0DEF5F0BC0EF3491F4D1
:102C3A000E94CD0C0E9402550E94F854E091100D9A
:102C4A00EF70F0E0FA93EA930E94C03EEBE3EA9356
:102C5A000E948E3E2AC0EB3441F5E091B80CEA930B
:102C6A003CD2E091BB0CE43229F4E0E8F0E00E94A7
:102C7A00D3541BC0E33219F40E94E20C16C0E134AB
:102C8A00A1F40E94CD0C0E9424550E94F8540E947F
:102C9A0024550E94F854E091AA0D0E9411520E94F4
:102CAA00C03EEEECF7E00E948D530E945B3D7DCD65
:102CBA000E94AC5348C10E9429550E9431550E9476
:102CCA00AC530E943855E181E43471F40E943855BE
:102CDA0002800E941953E05DE01529F00E943855E0
:102CEA00E281EA3209F401C057C00E943D550E94B0
:102CFA003855E1810E9440550E943855E2810E9470
:102D0A0040550E9446551C910E94385533960E94A0
:102D1A004B55E12FE23131F40E945055E6E0EC9335
:102D2A00FDD93AC0E13131F40E945055E2E1EC9309
:102D3A003ADD32C0EF30A9F40E945055EEE0EC9330
:102D4A000E94F60CE13039F4A091AD09A03019F0D7
:102D5A000E94875309F402C00E94811B0E945655A3
:102D6A001BC0EE30C9F40E945055EFE0EC930E946C
:102D7A00F60CE13089F4A091AD09A03019F00E9457
:102D8A00875309F402C00E94811BE0E0E093AD0979
:102D9A00EFEFEA930E94720D55C01A930E945D5597
:102DAA00E4EBF9E00E944B55EAE7EA930E948E3E73
:102DBA000E94465511971C91E12FE23131F4E6E069
:102DCA00EA930E948E3EAAD937C0E13131F4E2E19A
:102DDA00EA930E948E3EE7DC2FC0EF3099F40E94FE
:102DEA0062550E94F60CE13039F4A091AD09A03089
:102DFA0019F00E94875309F402C00E94811B0E94A5
:102E0A0056551AC0EE30C1F4EFE0EA930E948E3EA6
:102E1A000E94F60CE13081F4A091AD09A03019F0BE
:102E2A000E94875309F402C00E94811BE0E0E093EC
:102E3A00AD09EA930E94720DA091B009AA3211F06D
:102E4A000E942C40199108950E943B5408950E94B3
:102E5A00665517FD10E01A3008F41F5F0E9473557B
:102E6A0007C30E94665517FD02C0103011F4E0E056
:102E7A00FFC211500E947355E1E0FAC21A930A93F5
:102E8A0010E00E941653A8950E94D50AE03021F45A
:102E9A00E0EA0E942C5309F002C001E001C000E000
:102EAA000E94E50A1F5F003011F4153008F001C0D6
:102EBA00E8CFE02F0991199108950E947E5517C411
:102ECA000E947E550E948B550895A881B9810E945F
:102EDA004D5F24F4A83EE3E0BE070CF005C00E9453
:102EEA0091550E94450BC5C2E0E0C3C2A881B981D1
:102EFA000E944D5F24F4A83EE3E0BE070CF005C033
:102F0A00EA81E03011F4EFEFEA830E949155ED81F6
:102F1A00EA930E94740B42C10E94595F20E030E09C
:102F2A00283EE3E03E077CF4A8953A932A93CDDF46
:102F3A001E2F1F3F29F0EFEFEA933A932A93D6DF29
:102F4A002F5F3F4FEDCF0E94605F249608951A933A
:102F5A000A93E0E0F0E0E093B90DF093BA0DAA818C
:102F6A00A03458F40E949A55E55FFB4F8F010E94E6
:102F7A00A155E9EBFDE00E94AA55E091B90DF09147
:102F8A00BA0D0AC11A931FEF1F5F1A93E0DFA981D6
:102F9A00BA81EA17FB0711F0113408F001C0F4CF27
:102FAA00E12F1881FBC0EA81EF5FEA83EA93CFDF62
:102FBA00A881B981EA17FB0719F0AA81A13408F0A0
:102FCA0001C0F1CFEA81EAC00E94575F10E01034D5
:102FDA0030F50E94EE54E8E2F0E00E94E15CE05035
:102FEA00FC4FAF01E0EAEA93FA017096FA93EA938A
:102FFA000E94450BEC713E2FE0EAEA93FA017396C0
:10300A00FA93EA930E94450B0E2F303119F4EE81A0
:10301A00E01709F002C0E12F03C01F5FD8CFEFEF1E
:10302A000E945E5F279608951A930A93E091010D14
:10303A00AA81EA17C1F0A03468F40E949A55E050B8
:10304A00FC4F8F010E94AE550E94950BEA81E093D6
:10305A00010D09C0EFEFE093010D0E94C0520E94DA
:10306A00B755E0930C0D98C01A930A930E949A558B
:10307A00E050FC4F8F01AA81A03430F40E94AE5573
:10308A00E0E2EA930E94000C87C01A930A93E09147
:10309A002A0DAA81EA17B1F00E94C15540F40E9494
:1030AA00CD550E94AA55EA81E0932A0D0BC0EFEF95
:1030BA00E0932A0DEBE2FDE0FA93EA930E94B755FA
:1030CA00E093350D69C01A930A930E94C15520F402
:1030DA000E94CD550E948B555FC01A930A93E091C6
:1030EA00A80DAA81EA1751F10E94D85508F50E9445
:1030FA00A155E9EAFDE00E94AA55EA81E093A80DEC
:10310A00E0E0E093E607A091AA0DA13020F0A0919B
:10311A00AA0DA83008F00BC0A0E5BDE0E091AA0D09
:10312A000E94E255AE0FBF1FEC91E093E60706C07E
:10313A00EFEFE093A80DE0E0E093A90D2DC01A93FC
:10314A000A930E94D85530F40E94A155E9EAFDE09D
:10315A000E948B5521C01A930A93E091A30DAA816C
:10316A00EA1781F00E94E55540F40E94EF550E944B
:10317A00AA55EA81E093A30D05C0EFEFE093A30DF2
:10318A000E94FA5509C01A930A930E94E55520F441
:10319A000E94EF550E948B55198108812396089544
:1031AA000E94FA55E881EF5FE093A50D21960895F4
:1031BA0024970E94575F0E940656AB85A13010F0F3
:1031CA00A63008F007C0EB850E94E2550E9412560D
:1031DA000E941856EB85E03079F5E0E0EE83EF8344
:1031EA00E887E98740E050E020E030E02530E0E081
:1031FA003E07C4F4F9010E9412560E9418560E9412
:10320A00C5524E0F5F1F0E94CE52AE81BF81888584
:10321A0099850E947C5CEE83FF83688779872F5F9C
:10322A003F4FE4CF4093930D5093940DEE81FF816D
:10323A00688579850E942C560E945E5F2C960895B7
:10324A001A930A93AB81A13010F0A63008F01BC084
:10325A00EB810E94E2550E94995C0E94955CDF0115
:10326A00EA810E943556E8E0F0E00E94E15CE05015
:10327A00FA4E8F01E0EA0E9439561A930A93E1E95D
:10328A00FDE00E948B55198108810C94071E1A9340
:10329A000A93EA810E94345421F4198108810C941A
:1032AA00071E0E94551E0E2F10E01017E0F5EB8145
:1032BA00EA93EB81EA937CDFA3E9BDE00E947F52A7
:1032CA00A091950DB091960D8091970D9091980DC2
:1032DA000E941F550E94A95C0E947C5C0E942C5689
:1032EA00EB81EA93EB81EA93ABDFEB81E093990DF3
:1032FA000E941555309759F40E9419530E949D5304
:10330A00EF5EF84DDF01EA810E943F5602C00E943B
:10331A001555E0939A0DF0939B0D0E9443560E9417
:10332A0048561F5FC2CF198108810C94071E0E945C
:10333A00595F00E00B3060F40E9445520E94995C8C
:10334A00AE0FBF1F0E944E560E948B5D0F5FF2CFD9
:10335A000E944E560E94535600E00034F8F40A9335
:10336A0063DEE0919B09EA930A9322DFE0910F0D55
:10337A000E94B552EA0FFB1F0F01E0910F0D0E9448
:10338A00B5520E94BB52DF01CB010E94CE520E946D
:10339A007C5CD0010E948B5D0F5FDFCFA091910909
:1033AA00A330F1F530E03031D8F50E94E3510E94A4
:1033BA005C56A1F500E00A3088F5E32FE05DEA9358
:1033CA00E4EDF7E00E946156E02FE05D0E94685646
:1033DA0019F513E00E9445520E946D56FF93EF9330
:1033EA000E9445520E94995C0E94BB527F936F9340
:1033FA00FF93EF93EDB7FEB7FA93EA931F930E94F8
:10340A00863F1F91AF91BF918F919F910E947C5CE3
:10341A00AF91BF910E948B5D0F5FCDCF3F5FC3CF4E
:10342A0000E00A30A0F40E9445520E94995C0E9472
:10343A00BB52A091A209B091A3098091A4099091CD
:10344A00A5090E947C5C0E9453560F5FEACFD8C33D
:10345A001A93A895A981A63058F40E94065610E03E
:10346A00103430F4E981EA931A93EADE1F5FF8CF49
:10347A001881229608951A9311E0163020F41A93AF
:10348A00E7DF1F5FFACF4BC3E1E0E093A90DE093BA
:10349A00AA0D0C94C51EA895EBE2FDE0FA93EA93F7
:1034AA00EEE9F4E00E947256E093330D0E948156D1
:1034BA00E093340DE0E0E093350D0C94C51EA89519
:1034CA00E1E0FDE00E948856E9E2F0E00E948D56B4
:1034DA000E94C052E4E9F4E00E947256E0930A0D99
:1034EA000E948156E0930B0DE0EBE093100D0C94D3
:1034FA00C51E0E94575F0E94DF54E03228F0A6E002
:10350A00B0E0E0E00E94B75D00E0D7DCA091360DA4
:10351A00B091370DA633E2E1BE07C1F1E3E50E949F
:10352A0091561A3030F41A93B6DF1A93CCDD1F5F26
:10353A00F8CFE0E50E949156103430F41A93BFDFB9
:10354A001A9392DD1F5FF8CF0E941C05EBE40E94DC
:10355A009156103830F41A9397DF1A93F0DD1F5FF3
:10356A00F8CFE1E4EA930E94FA3885DFE4E5EA93CA
:10357A000E94FA38A1E0B0E0E0E00E94B75DE6E31D
:10358A00F2E1E093360DF093370D01E010E01532C9
:10359A0010F00C943A1B0E9473543E960E94905D60
:1035AA009F010E9473543E960E94905DAF010E9453
:1035BA00735470960E94905D309721F0E130A0E03C
:1035CA00FA0789F4D9016C910E94735472960E9489
:1035DA00905DA62FB0E0EA17FB0724F40E9473540B
:1035EA000E94965640C0E230A0E0FA07C9F4DA0118
:1035FA006D917C910E94735472960E94905DE617B9
:10360A00F7072CF0DA010E94815DFF2342F40E9441
:10361A00735474960E94905DDA01ED93FC9323C073
:10362A00E330A0E0FA0749F4D901AC91AF3F21F4A5
:10363A000E9473540E94965616C0E430A0E0FA071E
:10364A0091F4D901AC91AF3F71F400E00E94735438
:10365A000E948D5444F40E9473540E9496562F5F20
:10366A003F4F0F5FF3CF1F5F92CF2ADC10E0183075
:10367A0060F41A9370DDA091A40DA93020F01A937A
:10368A008FDD1A9380DD1F5FF2CFE02F0E945E5F0D
:10369A009FC0E881EF5FE883A881A43610F0E0E0DC
:1036AA00E883E8810C94C51E0E949B5630960C94C0
:1036BA00C51EA091AC0DBB27E091AB0DA6C0F9DFEA
:1036CA00329774F00E94A256E091AB0D0E94A9565F
:1036DA000E948B55E091AB0DEA93DBDFE093AB0DD3
:1036EA0008950E94A256E091AC0D0E94A956FA9341
:1036FA00EA930E94950B0895E9E9FDE00E94B1560C
:10370A000E94A256E091AC0D0E94A9560E948B55C8
:10371A00E091AC0DEA93BDDFE093AC0D08950E94F1
:10372A00595FE0E0E093AB0DE093AC0D10E030E0C0
:10373A00343680F5A8950E94A2563A93B5DFFA93DB
:10374A00EA93E9E9FDE00E94AA5500E0A091990DEB
:10375A00A13010F0A03808F001C001E0E12FE030FC
:10376A0041F4013029F43093AC0D3093AB0D11E0E4
:10377A000FC0E13031F4003019F43093AB0D12E090
:10378A0007C0E23029F4013019F43093AC0D13E08C
:10379A003F5FCECF35C21A93A091470DA870B9F0FA
:1037AA0010E0E981FA810E94EE54AE17BF077CF45B
:1037BA00ED81E093990DEB81FC81E851FC4F0E9469
:1037CA00A353E0E0F0E00E9448561F5FEACF188159
:1037DA0026960895E881EF5FE883A881A43610F061
:1037EA00E0E0E883E8810C94C51EE881E150E883B3
:1037FA00A881A43610F0E3E6E883E8810C94C51E9C
:10380A00A091AE0DBB27E091AD0DF0E031960E947C
:10381A00B856EC59FF4FDF01E4E6F0E00E943E5D46
:10382A0008950E949B56E050FE4F0C94C51EEEE987
:10383A00FDE00E94B156E881EA9380D10C94C51E3E
:10384A001A936ADBE1E0E093FE0C69C1A89510E0E7
:10385A00143680F41A936BD1A0919E0DAF3F31F4C8
:10386A000E94BD56AF3FEFEFBE0711F01A93DFDF9C
:10387A001F5FEECF0E94C256689420F850C10E9482
:10388A00595F1091AE0DAD81AA23E2F5E091AD0D1D
:10389A00E11719F0AD81AA230AF033C01A9347D170
:1038AA000E94BD56EE81FF81EA17FB0729F4E885DD
:1038BA00A0919E0DEA1709F021C00E94F953EC81EC
:1038CA00FD810E94815CEA17FB0764F40E94FE53A3
:1038DA000E9463530E940354E0E0EC83ED831A9341
:1038EA002DD10CC00E94FE530E946353EC83FD83CA
:1038FA00E0E0F0E00E9403540E94C8560E94CE56AF
:10390A00C5CF41C0E091AD0DE11729F0AC81BD8171
:10391A000E944D5F0CF01DC01A9309D10E94BD563A
:10392A00EE81FF81EA17FB0729F4E885A0919E0D35
:10393A00EA1709F00BC00E94FE530E9463530E94CB
:10394A0003541A93FBD0E0E0EC83ED830E94CE5639
:10395A00D9CFAC81BD810E944D5FACF4E885E0937C
:10396A009E0DEE81FF810E94D356EC81FD810E945B
:10397A000354E091AD0DEA93E1D0E091AD0DEA93E5
:10398A0029DFE093AD0D3CDF7E9714F00C94151DF2
:10399A001091AD0D0091AD0D1A9327DF1E2F1A93CA
:1039AA00C6D0A0919E0DA13010F0A03808F022C018
:1039BA000A931BDF0E2F1017E9F00A93BFD030E0ED
:1039CA003330C0F4ABE03A9FF001DF01EE54F84F18
:1039DA00E081E03031F0FD01EF54F84FE0811E172D
:1039EA0009F006C0ABE03A9FF001EF54F84F0083AC
:1039FA003F5FE6CFE091AE0DE11771F6101781F047
:103A0A00EEE9FDE00E94B156102F0A93EEDE0E2F6A
:103A1A000A9394D0E091AE0DE017B9F71093AE0D6A
:103A2A00689420F8EC81FD810E94605F29960895D0
:103A3A001A93A8951091AE0DE091AD0DE117C1F062
:103A4A000E94D8560E944D5F64F4EB81A0919E0DAE
:103A5A00EA1739F40E94BD56E981FA81EA17FB0791
:103A6A0009F003C0E12F1881CDC00E94CE56E4CFE1
:103A7A00EFEF1881C7C00E94F9530E944D5F84F48A
:103A8A00E091E607E87031F4E091A809A0919E0D53
:103A9A00EA1731F40E94DC560E94CE53E03408F053
:103AAA0001C015C112C1A895E091AD0DA881EA1710
:103ABA0049F0E8810E94E15611F0E88161C10E9453
:103ACA00E856F2CFEFEF5CC11A93A8951091AE0DAC
:103ADA00E091AD0DE117E1F00E94D8560E944D5FCA
:103AEA008CF4E091E607E87031F4E091A809A0911E
:103AFA009E0DEA1739F40E94BD56E981FA81EA1748
:103B0A00FB0709F002C0E12F7DC20E94CE56E0CF2A
:103B1A00EFEF78C21A931091AE0D1A93C4DF199180
:103B2A0008950E94E856E881EA93BDDF29C10E9400
:103B3A00A2560E94EE560E94AA5522C10E94A2567F
:103B4A000E94EE560E948B551BC1E091AE0DA881D2
:103B5A00EA1741F40E94F953109721F4A0919E0D9F
:103B6A00A03009F01CC0E881EA9361DE0E94E856A1
:103B7A00E881E093AE0DE091AD0DA091AE0DEA178C
:103B8A0019F0E881EA93D3DF0E94F953109721F4E0
:103B9A00A0919E0DA03009F001C0E5CF03C0E881D5
:103BAA00EA93CCDFEDC00E94595F0E94C25610E032
:103BBA0030E0343628F5A8953A93B9DF00E0A091B1
:103BCA009E0DA03808F401E0E12FE03041F4013005
:103BDA0029F43093AE0D3093AD0D11E00FC0E130F2
:103BEA0031F4003019F43093AD0D12E007C0E23021
:103BFA0029F4013019F43093AE0D13E03F5FD9CFA9
:103C0A000E94605F249608951A930A93A0919109DD
:103C1A00A43009F458C11091A8090091FD0DE09152
:103C2A00AA09E03059F0E093A809689424F80E94A0
:103C3A00F756E0E0E093A909E0E520C0E091A90980
:103C4A00E03021F0E093A809E2E518C0E0E0E09353
:103C5A00A809E093FD0DE0913C0DE03031F0E091D0
:103C6A003C0DE150EA930E947218A091A90DA1702F
:103C7A0039F0E0913C0DE093A809E4E4E093FD0DEE
:103C8A00A091A8091A1721F4A091FD0D0A1711F0A5
:103C9A00689423F818C1A091120DECE1EA23089563
:103CAA00A091120DA07411F0E2E00895A091120DF6
:103CBA00A07859F40CC0A091010DAF3F31F0EBDFB1
:103CCA00E43019F0E8DFE03111F4E0E00895E1E0D2
:103CDA0008950895A881AF3F09F451C0DCDFE430AC
:103CEA0011F4E1E04DC04BC0A881A23019F4D3DF32
:103CFA00E83011F0E1E044C042C0E881F0E00E94FF
:103D0A00FD56E25DF74FE081E13010F0E43108F052
:103D1A0002C0E1E035C033C0A881A13118F0E881C2
:103D2A00E051E883E8810E9402570E940657A09159
:103D3A00480DA13018F0A881A43009F004C0E6E9C2
:103D4A00F0E00E9406571CC0A881A13010F0A930EB
:103D5A0008F007C0E8810E94E255EF51F24FE08176
:103D6A000FC00DC0A881A13010F0A93008F007C01B
:103D7A00E8810E94E255E751F24FE08101C0E0E09C
:103D8A00219608950E94595FEC81EA93EBDFEF7365
:103D9A001E2F1030E1F0EC81EA93E4DFE0743E2F4D
:103DAA00E12FE150A1E00E948D5CA091E207EA2395
:103DBA000E2F303011F4003009F002C0E1E008C0E3
:103DCA00303011F0003009F402C0E1E001C0E0E057
:103DDA000E94605F259608951A930A93E1ECFDE02C
:103DEA00FA93EA93E0E00E9439560E94054F10E0E8
:103DFA00183090F51A930E94B0180E94EE54AF51F1
:103E0A00B24FE091A50DEC930E945652E751F24F42
:103E1A000F01A091A40DEFE3EA23AE2FE091A70DC5
:103E2A00E295E07FEE0FEE0FEA0FD001EC93E091FE
:103E3A00A50DE1500E2F0F3F69F0E02F0E94135796
:103E4A000E94CE54BF01E091A60D0E949D53DB0152
:103E5A00ED93FC931F5FCCCF36C01A930A93E6EF1B
:103E6A00F7E0FA93EA93EFEF0E9439560E94054F62
:103E7A0010E0103440F51A930E9419181A932ADF99
:103E8A00E130F9F4E091150DEA935EDFE1500E2F6F
:103E9A000F3FB9F00E94FD51EA50F84F1083A02F4E
:103EAA00B0E0A250B84FE091150DEC93E02F0E94BC
:103EBA0017570E941B57E0911B0DF0911C0DED93B3
:103ECA00FC931F5FD6CF099119910895A09191098A
:103EDA00A23031F0A83021F0A73011F0A53009F452
:103EEA000DC0EEE2F8E00E948856E0EFF0E00E9492
:103EFA008D5672DFB2DFE0E0E093EF0708951A9380
:103F0A00E981E058E98310E01530D0F40E94565256
:103F1A000E94FD560F01E05DF74FE081AE2FE98167
:103F2A00EA1749F4F001E15DF74FE081AE2FE09125
:103F3A00A809EA1709F002C0E12F03C01F5FE4CF06
:103F4A00EFEF1881229608950E94595FED81EA9356
:103F5A00D6DF1E2F1F3FD1F00E9456520E94FD56F7
:103F6A00E25DF74F9F01D9011296EC91EF77EC933E
:103F7A00EC81D9010E9420570E942757EF77DB0175
:103F8A000E942057E75FFA4FA1E0A083E12F0E9429
:103F9A00605F2EC41A931FEFE0914C0DF0914D0D06
:103FAA00A981BA81AE17BF073CF0E0914E0DF0919E
:103FBA004F0DEA17FB070CF411C0E981FA81FA9355
:103FCA00EA930E946A171E2F103031F01F3F21F02A
:103FDA00E091A809E11711F4E1E014C01F3F39F498
:103FEA00E8EDF7E0FA93EA93EB81FC8106C0E8EE8C
:103FFA00F7E0FA93EA930E945652FA93EA930E94E0
:10400A002D07E0E01881239608950E94595FE091F8
:10401A00E407F091E507AC81BD81EA27FB279F0100
:10402A0010E0183090F4F901E17039F00E94EE5472
:10403A00A951B84FEC91EF5FEC93D901E2E0F0E0BF
:10404A000E940C5D9F011F5FECCFEC81FD81E09324
:10405A00E407F093E5070E94605FCAC326970E94AF
:10406A00575F3091E40710E01830A8F50E945652C5
:10407A00EF50F24F0081E12FA1E00E948D5C2E2FBC
:10408A00E22FE32391F0003810F0003C08F001C061
:10409A000F5F003C31F4E22FA091E207EA2BE09394
:1040AA00E207003808F400E80FC0003408F40F5F94
:1040BA00003439F4EFEFE227A091E207EA23E09314
:1040CA00E207003808F000E00E945652EF50F24F23
:1040DA0000831F5FC9CFE0E0F0E0E0938E09F09320
:1040EA008F09E0919509EF5FE0939509E0915B0DE7
:1040FA00A0919509EA1751F4E0915B0DF0E0A0E078
:10410A00B1E00E94A45DEA1BE0939509A091910990
:10411A00A13019F0A93009F0A6C0A091DA0CB0912B
:10412A00DB0CE4E1F0E00E943E5D309719F4E1E037
:10413A00E0939809E091EF07E030D9F0E091F007B9
:10414A00EA93EADDE091F107EA93E6DD0E942C5753
:10415A00E951F84FE081A091F407B091F5070E9468
:10416A003F560E942F570E943457A2EFB7E00E9491
:10417A007F520E943957109721F0E0915007E0785A
:10418A0009F44EC00E9432525E2F5A930E941918A7
:10419A00A091110DA03049F48EDDE13031F4E091A7
:1041AA009209EA93A1DDE03009F43AC00E943E5731
:1041BA000E943556EC91EC71EC3021F4E0919509AE
:1041CA00E07851F40E944357A7DDA8E1BDE00E94C0
:1041DA0049570E945A53A0DDE52F0E944D570E946D
:1041EA001B570E947F520E944357AEDD1E2F11308B
:1041FA00B8F00E9451570E94CE540F010E945157A5
:10420A000E944A52DF01E12F0E94E2550E9456574E
:10421A00D001ED93FC93E12F0E94E2550E9434579E
:10422A0010E0183000F50E945652EA50F84F5081BB
:10423A005F3FB9F00E9456520E945A570E94515746
:10424A000E94CE540F010E9451570E944A52DF0128
:10425A000E9456520E945657D0010E9460570E94EF
:10426A0034571F5FDECFA0919109A23039F0A830F0
:10427A0029F0A53019F0A73009F0B5C1E0E0E093C4
:10428A00990900E0053010F00C94F8220E94FD51C3
:10429A000E94FD56E25DF74FE887F987A885B98540
:1042AA00AC91A03019F0A281A07809F09AC1E091EE
:1042BA009909EF5FE0939909A885B98513960E9439
:1042CA00815D309781F0A885B9850E9463570E9465
:1042DA006A5719F00E946F5709F004C0A885B9857A
:1042EA000E9474577EC10E943957109739F00E9474
:1042FA006A5719F00E946F5709F473C120E030E041
:10430A00333010F00C949A220E94FD510E94FD56FF
:10431A00ED5CF74FDF010E94E3510E947A57E60FE6
:10432A00F71FEE83FF83AE81BF81EC91E27031F417
:10433A00EE81FF81A381B481109709F4D8C0EE8180
:10434A00FF81A581B681109751F003801480AE8158
:10435A00BF8115960E94815D0E161F060CF00EC0D5
:10436A00AE81BF8115960E948057E091900D0E9400
:10437A009D53A885B9851396ED93FC93AE81BF81B1
:10438A00EC91E17021F40E946357319650C00E946B
:10439A008557DADCE1501E2F0E945652E951F84F38
:1043AA00E081E03011F50E948A570E947F52E12F86
:1043BA000E9413570E944A52309761F00E948A570E
:1043CA000D901C90E12F0E9413570E944A52E0154B
:1043DA00F1050CF009C00E94FD510E948F5711F09F
:1043EA000E9494570E949C5719C0EE81FF81339610
:1043FA00BF01DF010E94815DDF010E945652E9512F
:10440A00F84FE081F0E00E94B856DB010E94605745
:10441A000E9434570E948A570E948057EE81FF817A
:10442A00A481AA2322F4AE81BF810E947457AE816F
:10443A00BF81EC91EC71EC3021F4E0919509E078C0
:10444A00C1F4EE81FF81A381B4815E972CF4AE8121
:10445A00BF81EC91E07209F404C0EE81FF81A18171
:10446A0006C00E94855758DCEE81FF81A281AA937B
:10447A0053DC0E94A45789F0AE81BF8117960E942F
:10448A00AB570E94A45749F40E94FD510E948F57CE
:10449A0011F00E9494570E949C570E94855772DC23
:1044AA00E03029F10E94FD510E948F5771F00E945D
:1044BA009457A885B985EC91E150ACE0EA9FF001E8
:1044CA000E942757E058DB01EC93A885B98512961C
:1044DA00EC91E058A885B9851296EC93E3E0E09355
:1044EA00E3070E9485573EDCEF73E093FA0DAE8135
:1044FA00BF8113960E94815D3097A9F42F5F3030F7
:10450A0041F4E885F985E685ED7FA885B9851E968B
:10451A00EC93313041F4E885F985E789ED7FA88588
:10452A00B9855796EC933F5FEBCE233011F00C948C
:10453A00F6220E946A5711F00E9494570E941A307C
:10454A00E030B1F00E94E1520E94B157E8E0EC93EA
:10455A00A885B9851296EC91AA85BB851496EC9329
:10456A00A885B985EC91AA85BB85EC930E94B957B9
:10457A00A885B985E0E0EC93E885F985A581ECE1A9
:10458A00EA23E83071F50E941953AE2FE885F985C0
:10459A00E08DEA1741F4E885F985E18DE150EA9367
:1045AA000E942C171EC00E941A30E030D1F00E94DF
:1045BA00E1520E94B157E3E0EC93AA85BB85EFEF85
:1045CA00EC931696E885F985E08D0E94C157AA8575
:1045DA00BB851296E885F985E18D0E94C1570E9434
:1045EA00B9570F5F4FCEA0919109A23029F0A83098
:1045FA0019F0A53009F066C010E0183010F00C94DC
:10460A0067230E945652EA50F84F50815F3F11F4D7
:10461A000C9465230E9456520E945A570E94C5570D
:10462A000E94CE540F010E94C5570E944A52DF01D0
:10463A000E9456520E945657D0010E9460570E940B
:10464A0034570E94C5570E944A52DF010E944D5FAB
:10465A00D4F4E12F0E9417570E944A52DF010E94A8
:10466A004D5F8CF40E94C5570E941B570D901C90F9
:10467A00E12F0E9417570E944A52D001AE1BBF0B6E
:10468A000E944D5F0CF01CC00E94C5570E94CE5478
:10469A00BF010E94C5570E941B570D901C90E12F25
:1046AA000E9417570E944A52DF01F001EA1BFB0BD6
:1046BA00DB01ED93FC935A93E5E0EA930E94904460
:1046CA001F5F9BCFE0919409E03041F4E0918E099D
:1046DA00F0918F09E0938C09F0938D090E945E5F37
:1046EA002C9608950E94575FD6DAE03111F40C94A3
:1046FA00FA2320E030E040E050E010E0133060F5AB
:10470A000E94CA570E944A52309721F10E94CD57FF
:10471A000E9402570E94905D2E2B3F2B0E94CD577C
:10472A000E94D45729F0E3E0E093E307E0E05EC09B
:10473A000E94D9570E9402570E94905D2E2B3F2B50
:10474A000E94D9570E94D45729F0E3E0E093E30787
:10475A00E0E04CC01F5FD2CF00E00530E0F50E94D8
:10476A00FD510E94FD56E25DF74FE081E03089F18C
:10477A0010E0133070F50E94FD510E94FD56ED5C69
:10478A00F74FDF010E9456520E947A57DB01AE0FA3
:10479A00BF1F1196EC910E9402570E94905D4E2B0A
:1047AA005F2B0E94FD510E94FD56ED5CF74FDF0121
:1047BA000E9456520E947A57DB01AE0FBF1F129613
:1047CA00EC910E9402570E94905D4E2B5F2B1F5F57
:1047DA00D0CF0F5FC2CFF901E423F523309729F038
:1047EA00E1E0E093E307E0E001C0E1E00E945E5F00
:1047FA00269608951A93E091FB0DE03011F40C947B
:10480A004624E0915C0DE13059F4A091FB0DA133EF
:10481A0011F4EFE001C0E0E0EA930E94773A31C078
:10482A00E23059F4A091FB0DA13311F4E6E001C086
:10483A00E5E1EA930E94773A24C0E330B1F410E04C
:10484A00173040F40E945652E854F54F0E94E05740
:10485A001F5FF6CFA091FB0DA13311F4E1E301C074
:10486A00E0E3EA930E94773A0CC00E94E457E9E435
:10487A00EA930E948E3EE091FB0D0E94EB570E9444
:10488A00C2401991089522970E94575F30E0A09183
:10489A009109A23029F0A83019F0A53009F028C1F1
:1048AA00A985A03410F00C947B25E091A809E0308A
:1048BA0009F443C1E985EA930E941918ECD9E03159
:1048CA0031F4E1E3E093FB0D95DFE1E036C1F3D982
:1048DA00E03009F432C110E0153078F40E945652E3
:1048EA000E94FD56E25DF74FE081AE2FE885EA1798
:1048FA0011F4E0E022C11F5FEFCFF4DEE03011F4E3
:10490A000C947B2510E00E9456520E94FD56E25DEF
:10491A00F74FEE83FF83AE81BF81EC91E03011F057
:10492A000C9474250E94745700E0033010F00C9424
:10493A0044250E9456520E94FD56ED5CF74FDF0156
:10494A000E94FD510E947A57E60FF71FAF01DA0164
:10495A0015960E9480570E94F257DA011196EC933D
:10496A000E94F957DA011296EC93A091120DECEF1E
:10497A00EA230E2E0E940058E029DA01EC938BD923
:10498A00E43121F4DA01EC91ED7F03C0DA01EC9114
:10499A00E260DA01EC930A93A7D9E03011F40C949F
:1049AA003125FA01A181AA93CFD92E2F213070F097
:1049BA00E22F0E94E2550E943457E22FE150A1ED06
:1049CA00BDE0F0E00E941B570E9480570E940858E1
:1049DA000E944A52DA011396ED93FC93013031F4A6
:1049EA00E0911D0DF0911E0D309709F006C0AE81C1
:1049FA00BF811596EC91E062EC93023031F4E091BC
:104A0A001F0DF091200D309709F006C0AE81BF81CD
:104A1A001E96EC91E062EC93AE81BF815796EC91C1
:104A2A00E062EC930E94F257EA939CD9E07831F461
:104A3A000E94F957EA9396D9E07869F00E940858DB
:104A4A000E944A52DF01E2E0F0E00E940C5DDA01C6
:104A5A001596ED93FC9303C0DA010E9474571BD993
:104A6A00EC3019F4E0E0E09395090E940B580E949B
:104A7A009D53DA011796ED93FC930F5F56CFA091E1
:104A8A009109A23011F0A53019F4A885A03808F0D0
:104A9A0007C0E091A809EA93EA85EA930E944C19B3
:104AAA00E885AE81BF81EC93E091A809AE81BF8110
:104ABA001196EC93E985AE81BF811296EC93A88595
:104ACA00A03830F4E885E1500E941258A1E0A08392
:104ADA00AE81BF811596EC91ED7FEC9331E01F5FBB
:104AEA00303011F4153008F001C00DCFE32F25C086
:104AFA00A0919109A13009F5A985AF3F41F0E98557
:104B0A00EA930E941918E0E0EA930E94B542E88508
:104B1A00E093EF07E091150DE093F007E091180D8F
:104B2A00E093F107E0E0F0E0E093F207F093F30797
:104B3A000E942F570E943457E1E00E945E5F2A9636
:104B4A0008951A930A93A0919109A23011F0A53001
:104B5A0049F4EA810E941258A0E0A083EA81EA930C
:104B6A000E949552A0919109A830E1F5EA810E942C
:104B7A001258A0E0A083EA81EA930E949152EA8146
:104B8A00ACE0EA9FF001E050FB4FE081EF771E2F87
:104B9A00EA81ABE0EA9FF001E554F84FA0E0A08378
:104BAA00A0915A0DA03039F40E941858DF010E94D2
:104BBA00815D309709F010C00E941E5800810E9442
:104BCA001E58AFEFA0830E9418580E9424581A93C7
:104BDA000E941807689420F8E0915A0DE03011F00D
:104BEA00689420F8198108812396089564970E9491
:104BFA00595FA0919109A23039F4E091A809EA938A
:104C0A00E98DEA930E944C19A0919109A83011F0FC
:104C1A000C946F260FEF30E0383048F40E94E351CD
:104C2A00EA50F84FE081AE2FE88DEA1709F402C086
:104C3A003F5FF2CF0E94E351EA5EF74F00810F3FD8
:104C4A0011F40C946F260E94295810810E94D8569C
:104C5A000E944D5F04F5A1EABDE00E94AB570E9495
:104C6A002F580E94F953A083B1831A930E94A31D5F
:104C7A00ABE00A9FF001ED54F84F20810A930E949D
:104C8A0035580E945E312A930E9435580E94E244A8
:104C9A002A930E9495520E94FE533097D9F40E949B
:104CAA0029580E943A58EA50F84F0E943A58EA5E48
:104CBA00F74FAFEFA0830E942F580E942458E0E0DC
:104CCA00F0E00E9403540E94C8560A930E941807F3
:104CDA00689420F80E94605F699608951A9310E01C
:104CEA001031A0F40E945652E751F24FE081EF735F
:104CFA00AE2FE981EA1729F4E12FEF5F0E94D4571A
:104D0A0009F402C0E1E003C01F5FEACFE0E01881C6
:104D1A00229608951A930E943D580E9485520E9435
:104D2A00B80CE030F1F00E94445810E01830C8F492
:104D3A00A091000EAF5FEA2FE770E093000EEF5FDD
:104D4A00EA93CCDFE03059F0E3E0E093E307E09147
:104D5A00000EF0E0EF5FFF4EE093FA0D6FC31F5FA6
:104D6A00E5CF6CC31A93E091E207E093F90DE8E707
:104D7A00F0E0FA93EA93ECEDF0E0FA93EA930E94FA
:104D8A00E03810E0183018F5E12FEF5FEA93A6DF5C
:104D9A00E030D9F00E94A051E12FEA5F0E9411523F
:104DAA000E948938E5EFF7E00E946451AEE5BDE064
:104DBA000E945652BD01AAE0B0E00E94B95CE60F1B
:104DCA00F71FFA93EA930E94B1521F5FDBCF36C3F3
:104DDA00A1DFA091E307A13021F4EDEFF7E00E94F3
:104DEA004B58A091E307A23021F4EAE0F8E00E94D0
:104DFA004B58A091E307A33059F4E5EFF7E00E947E
:104E0A005358F0E0E050F04FFA93EA930E942D07CE
:104E1A00A091E307A43041F4E2E1F8E00E9453587C
:104E2A000E9411520E942D07A091E307A53029F490
:104E3A00E091FA0DEA930E941B07A091E307A630BE
:104E4A0041F4EAE1F8E00E9453580E9411520E948C
:104E5A002D07A091E307A73021F4E0E2F8E00E94D1
:104E6A004B58E0E0E093E3070895A881B9811196D1
:104E7A00E1E0EC930E94DC56A881B9811296ED9389
:104E8A00FC930E94551EA881B9811596EC930E9445
:104E9A001953A881B98116960E94C157E0919A07C1
:104EAA00A881B981EC93E0919E0DA881B9811496ED
:104EBA00EC93E091010DA881B9811896EC9361C435
:104ECA0064971A930A93A0915A0DA230E1F4E98DDE
:104EDA00EA930E9419180E94551EA1EABDE00E9499
:104EEA00C157AFE9BDE0E98D0E94C157E091A80919
:104EFA00E0939E0D0E941555309721F00E9415559A
:104F0A000E94D35614C0A88DAF3F09F4C8C0E88DDB
:104F1A00EA930E949C1DA98DAF3F29F40E94DC569A
:104F2A000E94CE53E98FE98DEA930E9419180E94D4
:104F3A00551E0E2FAF89AF3F21F00E94601EE03050
:104F4A0009F001C0ACC00E94F9530E94FD51AE178E
:104F5A00BF071CF0C7DBE13009F0A1C0A091490DE1
:104F6A00A03021F4A0915A0DA23021F50E941953C4
:104F7A00E13041F00E941A30E03021F00E943030D6
:104F8A00E03009F004C00E94E1520E9458580E9481
:104F9A001953E13021F40E942030E03009F409C0AD
:104FAA000E94DA53E25DF64FFA93EA935EDF0E94BB
:104FBA00EB5373C0E98DEA930E945F581E2F11309C
:104FCA0011F00C945228A0914B0DA13059F4E091A4
:104FDA00A809EA930E94DC56FA93EA93EFEFFFEFEF
:104FEA000E940B540E94F9530E94FD510E94B85628
:104FFA000E940354689420F8A0915A0DA03019F425
:10500A00AE89AF3F09F42EC00E946458E954F84FA4
:10501A000E94F953A083B183EE89EA93FE01339685
:10502A00FA93EA930E945E310E946458ED54F84F55
:10503A00E081EA93FE013396FA93EA930E94E244EE
:10504A000E946458E554F84FA1E0A0830E94645876
:10505A00E754F84FFF93EF930E94AC0CAF91BF91C6
:10506A00ED93FC930E94FE53309741F4E0E0E09305
:10507A009E0DE88DEA930E94AA1D04C0E88DEA936A
:10508A000E94A31DE091A809EA930E9415550E9467
:10509A006958FA93EA930E94D01BE1E001C0E0E06C
:1050AA00198108816A9608951DDBE13031F4BDD774
:1050BA00E03019F0D0D7E03009F009C00E94155548
:1050CA000E94D3560E94E1520E9458587DC285C25E
:1050DA001A930A930E946C581F3F11F40C94BC282F
:1050EA00E091FB0DE03011F00C94BB281A930E945A
:1050FA001918E5E0E093E3071093FA0DA0919109DE
:10510A00A23031F40E9473580E94CF1FE13009F097
:10511A000EC0A091FC0DA13331F4E091A809EA93E5
:10512A001A930E944C19E1E3E093FB0D96C3A091F8
:10513A009109A83081F40E941555FA93EA930E94C6
:10514A00691D0E2F1A930A93EFEFEA93EA93B8DEDA
:10515A00E03009F082C3A0919109A53021F4A4DFBF
:10516A00E03009F07AC3E0E3E093FB0D06C0E0E328
:10517A00E093FB0DE4E0E093E3076FC3E091B80A24
:10518A000E94775808950E94595FA091B70AA534E2
:10519A00D9F50E948358E2E3F0E0E093BD0DF09365
:1051AA00BE0DA091B80AA73731F4ECEBFAE00E94E1
:1051BA008A580E947758A091B80AA03310F0AA33EF
:1051CA0008F021C02091A0093091A1090E9431550F
:1051DA00E2E0EA930E94083E0E2F0E948F58E09365
:1051EA00FA0D0E948F580E9493580E946C580A9395
:1051FA001A930E944C192093A0093093A109E2E561
:10520A00EA930E94773A1DC0E091BB0DF091BC0D64
:10521A00FA93EA93E091BD0DF091BE0D0E94985861
:10522A00E03079F0E0E0E093B20AE5E4EA930E9424
:10523A00773A0E948358E8ECF0E0E093BD0DF093D2
:10524A00BE0D0E94605F249608950E949C580E9499
:10525A00A0510E9439520E94A0510E94A0510E945E
:10526A008938E8EAF4E00E946451E09192090E94C8
:10527A00A058E6EBF4E00E946451E2E0E093F40502
:10528A000895EEE2F8E00E948856E0E4F0E00E9419
:10529A008D56EEEAF8E00E948856E0E4F0E00E94BB
:1052AA008D56E7EEF7E0FA93EA93E0E00E9439566A
:1052BA000E94054FE881E03009F406C0A0919209E6
:1052CA00AF5FE3E00E943B5DE09392090E94F11E0A
:1052DA000E94321F20C11A930A9310E0103410F072
:1052EA000C94C9291A930E94191800E0E12F0E9410
:1052FA004D570E944A523B97ECF0ABE1BDE00E9449
:10530A0049570E94CE540F01E12F0E944D570E9427
:10531A004A52D001ED93FC930E943E570E943F5699
:10532A000F010E943E570E943556EC91EE7FD00144
:10533A00EC9301E0AEEAB8E00E9456520E944A524B
:10534A007597DCF0ABE1BDE00E9449570E94CE544C
:10535A000F01AEEAB8E00E9456520E944A52D001AA
:10536A00ED93FC930E943E570E943F560F010E9404
:10537A003E57F0E00E94C35401E0013019F41A9339
:10538A000E9439181F5FAACF68C21A9323FE03C06E
:10539A000E94A45820D60E94A144E030F1F1E0E036
:1053AA000E94A958103818F5113219F40E94A4580D
:1053BA0012D61D3439F40E94B0580E945C40E3E0D2
:1053CA00E09390091B3261F40E94B558EAE2EA932D
:1053DA00E7E3F8E0FA93EA93E09192090E94BB5856
:1053EA001F3221F4E1E0EA930E94DF062EDF103833
:1053FA00A0F00E94BF5889F0A0919907A23031F419
:10540A00E091110DEA930E94DF061FDFA091990730
:10541A00A43019F4E3E0E09390090E9439571097F9
:10542A0019F00E94C7580CF409C0E0919809E030BD
:10543A0029F00E945107E0E0E09398091991089534
:10544A000E94CF580E94D3580E949C580E94A05193
:10545A000E948938A0919309A23021F4EAE3F8E086
:10546A000E946451A0919309A13021F4E1E4F8E08B
:10547A000E946451E0919309E03021F4E8E4F8E0F5
:10548A000E9464510E94DA580E9489380E94DF58AB
:10549A000E94E4583197FA93EA93E0914407F09115
:1054AA0045070E94E9580895E1E003C0E0E001C021
:1054BA00E2E0E0939309C4DF0895A881A03310F0D5
:1054CA00AA3308F01AC00E94ED580E94F258AAE0C6
:1054DA00B0E00E94E15CDF01E881E0530E943F56A0
:1054EA00E0939E09F0939F09E1E0E093F4050E949E
:1054FA00DA580E9439520E94DF58A881A33459F41D
:10550A000E94D358E1E0E093F4050E94DA580E9421
:10551A0039520E94DF5821960895A0E023FCA1E0A9
:10552A00A03019F0A881A03009F016C0E89423F839
:10553A00E7E0E09390090E948838A091AA09A03078
:10554A0019F40E94F75809F407C0E7E0EA930E94A9
:10555A00B35341D5E89424F824FE19C00E94FC589C
:10556A00EAE5F0E00E949858E13019F0A881A130EC
:10557A0069F45BD5E03051F00E940359E981EA935E
:10558A00E091A809EA930E94735825D50CC00E949D
:10559A00FC58ECE2F1E00E949858E13021F40E94B4
:1055AA000A59E093A909EDC0E0913F0DF091400D31
:1055BA000E940E5911F4E2E00895E0913D0DF09138
:1055CA003E0D0E940E5911F4E1E00895E091430D59
:1055DA00F091440D0E940E5911F4E0E00895EFEFA6
:1055EA000895A0919109A23021F40E94D0380E9416
:1055FA00A006A0919109A83009F446D5A091910975
:10560A00A53009F42DD10FC51A93E2E0EA930E945E
:10561A00B542E1E0E093F405E981EA934EDFA9811E
:10562A00AF3721F4E091E607E37009F403C0E2E042
:10563A00E0939009A981A13261F0A33421F40E9478
:10564A00ED58109709F004C0A0919109A23009F011
:10565A0011C0A0919309A33009F42ADFA0919309FC
:10566A00A23019F4E1E0EA93BCDFE0919309E0305B
:10567A0009F41CDFA981AD3311F00C949F2B0E9411
:10568A008838E0919309E030B9F4E0919E09F091ED
:10569A009F09FA93EA930E94CF1F1E2F113051F4EB
:1056AA00E0919E09F0919F090E949358E0E0EA93E5
:1056BA0098DF01C0FBDE3EC0E13079F475DFEF3FD1
:1056CA0041F0E3E00E9412590E94B0580E94185912
:1056DA0003C0E1E0EA9385DF2DC0E230E9F40E94DD
:1056EA00ED58A034E0E0BE07ACF4E0919E09EA93DD
:1056FA000E941F590E949C580E94A0510E948938FA
:10570A000E94C0520E94B1520E94F006E3E0E09368
:10571A00930901C0CDDE0EC0E33061F4E0919E0929
:10572A00EA930E941918E0919E09EA93EFEFEA932F
:10573A00AAD8BEDEA981AD3409F4B6DEA981A435A2
:10574A0021F4A0919109A23009F001C0AFDEA9812C
:10575A00AB3231F4E0919609EF5FEA930E94DF06DB
:10576A00A981AD3231F4E0919609E150EA930E94A1
:10577A00DF06A981AF3221F4E1E0EA930E94DF0655
:10578A00188122960895E091110DE33631F4A09123
:10579A009109A23009F48ADE14C0E23611F488DED7
:1057AA0010C0A0919907A23011F0A63029F4E09117
:1057BA00110DEA930E94DF06A0919907A43009F41B
:1057CA0073DE08950E946B1F0E94D038E0E0E093D8
:1057DA009309A881A13039F40E94F75821F0A091C9
:1057EA00420DA03009F402C061DE02C00E94A00688
:1057FA001AC41A930A930E94235979F10E943059C4
:10580A0060F10E94BF5841F50E9438590E94A91FB1
:10581A00EF3F19F50E9473580E94CF1FE13021F41F
:10582A000E94601EE13009F016C00E94501EE83145
:10583A0039F4E091010DEA930E943617E03009F03D
:10584A0001C00BC01A930E945F580E2F013019F441
:10585A001A930E941B0701C096DF099119910895B6
:10586A000E946B1FE89421F8E0E0E09397090E94F8
:10587A00A00608951A930E94235949F00E943059AC
:10588A0030F00E94BF5811F40FDC01C07CDF37C42E
:10589A000E94595F0E94235911F40C94AE2C0E9465
:1058AA00A4440E2F0A93B0DEA0915A0DA03021F421
:1058BA00003810F0033808F00AC00F770E94295800
:1058CA001081EFEFEA930E9438590A93F9DAA0910E
:1058DA005A0DA03011F0003808F43BC00F770A9334
:1058EA000E941918E091110DE03091F50A93E091A8
:1058FA009A07EA930E94A91FEF3F19F00E94605F7E
:10590A0087C30E94601EE13011F50E94551EE030E7
:10591A0061F40A930E945F58E03031F0E091A809DF
:10592A00EA930A930E944C1912C0A0919709E02F9A
:10593A00EA1BAEECB8E0F0E00E94995CAE0FBF1F24
:10594A001C910A930E943859EFEFEA93B9DA01C021
:10595A001ADF20FE0AC0E0915A0DE03019F4D1D3C3
:10596A0008D501C061D5E89420F830E03330F8F466
:10597A00ABE03A9FF001DF01E554F84FE081E030F7
:10598A0051F0A754B84F0E94E954E8EEF3E00E94A0
:10599A009858E03009F409C0ABE03A9FF001E554A9
:1059AA00F84FA0E0A083689420F83F5FDFCF0E9401
:1059BA00605F2EC30E94575FA0919109A33011F432
:1059CA000C949E2EE091B209ED3411F00C94C12D85
:1059DA00E091B309EA3511F00C94762D24FC81C0CC
:1059EA00E091B409E0532E2FE091B509E0533E2F20
:1059FA00E6EBF9E00E944B550E947553AB3429F44B
:105A0A000E941D540E94DD3D0E2F0E947553A4353D
:105A1A0029F40E941D540E94DD3DAF01E091450D1D
:105A2A00E31731F5E0E0E093C00D0E94035940937B
:105A3A00A0095093A109A091A9090A1759F0E7E012
:105A4A00E09390090093A9092093BF0DE0E0E09349
:105A5A00A8090DC0A091BF0D2A1721F0A091A7098E
:105A6A00A03009F004C0209390092093BF0D35C0DF
:105A7A00A091A909A03049F4A091460D0E94E351D2
:105A8A00E255FF4FE491EA2309F40CC0E7E0E09302
:105A9A0090092093BF0DE0E0E093A809E091B109D5
:105AAA00E093C00DE091B109A091C00DEA17A9F4E5
:105ABA004093A0095093A1090093A9090E94035990
:105ACA00A091BF0D2A1721F0A091A709A03009F0D3
:105ADA0004C0209390092093BF0D273011F40E942F
:105AEA00F756E091B309E93439F4E7E00E94125914
:105AFA000E940A59E093A809E091B309E03039F409
:105B0A00E4E00E9412590E940A59E093A809E09120
:105B1A00B309E03519F4E1E0E0939009E091B309A3
:105B2A00EC3449F4E4E0E0939009E091B409E053DD
:105B3A00EA930E946409E091B309E334E9F4A0917D
:105B4A00B409A13320F0A091B409A93308F014C014
:105B5A000E943D59E0919B09EA930E942D1AE09117
:105B6A00B109EA93E9E5F8E0FA93EA930E944E56FE
:105B7A000E94945D0E944F40E091B209E03521F401
:105B8A00A0919109A13009F003C00E94B5585DDBCC
:105B9A00E091B209EF3459F4E091B309EE3439F4E3
:105BAA00E091B109EA93ECE5F8E00E944359E091EB
:105BBA00B209E33579F5E091B309EF3359F5A091CC
:105BCA00B409A03360F0A091B409A93340F4A091BC
:105BDA00B509A03320F0A091B509AA3308F01AC07C
:105BEA000E943D59E091B509E0531E2F103011F47F
:105BFA000E949C19E091B109EA93EFE5F8E0FA9363
:105C0A00EA93E12F0E94B5520E94BB520E94945D12
:105C1A000E944F40E091B209E33411F00C94632ED4
:105C2A00E091B309EF3311F00C94632EE091B509BA
:105C3A00E03319F4EFEFE0939C09A091B409A03383
:105C4A0020F0A091B409A93308F01BC00E943D5965
:105C5A00E0919C09EF5FE0939C09E0919B09EA932C
:105C6A00E0919C09EA930E94DD18A091930DB091EE
:105C7A00940D109721F4A0919C09A03408F001C05A
:105C8A00E7CFE0919C09EA930E9419180E945D559A
:105C9A00E2E6F8E00E948D530E94C5520E945152DA
:105CAA000E941C3F0E94CE520E94945D0E941C3F9B
:105CBA000E94C0520E94443F0E942C40E091B209C7
:105CCA00E434B9F5E091B309E43499F514E0E1E07C
:105CDA00E093B10A103538F40E945652E055F64F57
:105CEA00E081E03208F41AC00E945652E055F64F9D
:105CFA00E081E33259F40E945652EF54F64FE081A4
:105D0A00E053EA930E94773A1F5F06C00E945652F8
:105D1A00E055F64F0E94E0571F5FDCCFE091B009D3
:105D2A00EA930E941040E5E6F8E00E948D530E9433
:105D3A002C4054C41A930A930E94495911F40C94A2
:105D4A00192FE0919009EF770E2F009390090E9486
:105D5A00D0380E940C52E4E0F0E0FA93EA930E94F1
:105D6A008938013021F0A0919109A13009F00BC0C6
:105D7A00EEEBF4E00E946451AEDA0E9485520E9472
:105D8A00C0440E94D038073049F40E946B1FE0E0FB
:105D9A00E09393090E9449070E94B726043031F420
:105DAA00E8E6F8E00E9464510E944705083019F4B9
:105DBA000E944F5969D1053019F40E944F5950DD9C
:105DCA00013051F4E89423F8E0E0EA935ADA0093B8
:105DDA0091093BDA0E94A006093071F4E0E0EA93E7
:105DEA0050DAE0E0E0939709E89423F80E94A006CD
:105DFA000A93E1E0EA9391DB023081F4E0E0E09378
:105E0A009709E0E0F0E00E949358E89423F80A9397
:105E1A00E1E0EA9382DBE1E0EA93D4DC033011F4B7
:105E2A000E94B34E00939109A0919109A73011F0F5
:105E3A000C94C82F0E943D58E4E6F0E00E9498585E
:105E4A00E03021F0A0919309A03009F00AC00E9425
:105E5A004458E091F90DA091E207EA1711F00E9467
:105E6A00B7260E94A144E030E9F0E2E00E94A95876
:105E7A001A9323DB1D3409F417DB1D3399F40E94AE
:105E8A00883892DBEF3F41F0E3E0E09390090E940B
:105E9A00B0580E94185906C0E7E8E0939009E0E07C
:105EAA00E0939309A091A809A03031F0E091A809E4
:105EBA00A091A709EA1709F457C0E091A809E1508F
:105ECA00EA930E947218A091A90DE1E0EA23E13059
:105EDA0021F4E091E607EF7C09F429C0E0E0E093C1
:105EEA00A709E091BF0DE03019F0E09390091EC0B8
:105EFA0012E0E091E607EC7009F018E0E0913C0D41
:105F0A00A091A809EA1781F0E091E607E07439F058
:105F1A0011E0EAE2EA93EDE6F8E00E944359E091E3
:105F2A00E607E07809F019E0109390091DC00E9475
:105F3A00D0380E9449070E940C52E4E0F0E0FA933C
:105F4A00EA930E948938EBE4EA930E94FA38E091D6
:105F5A00A809EA930E943343E0E7F8E00E946451FB
:105F6A00E091A809E093A709A091A809A03021F41B
:105F7A00A091A709A03009F406C0E0E0E093A709C0
:105F8A00E7E8E0939009A0919109A33011F40E94E7
:105F9A00B44CA0919109A13009F4F7D9A0919109C3
:105FAA00A23009F426DCA0919109A83009F470DC2A
:105FBA00A0919109A53009F45DDCA0919109A9305D
:105FCA0049F4E0E0E0939909E0919109EA93E0E06D
:105FDA00EA93A3DA3CC30E94E152E45AF64FA6E0E0
:105FEA00A0830E94E152E55AF64FAB81A0830E943A
:105FFA00E152E15AF64FAA81A0830E94E152E35A84
:10600A00F64FA881B981A083B1830E94B9571CD6E3
:10601A0024960895E881EF5FE883A881A53010F0FF
:10602A00E0E0E883E88121960895A0918B09BB27D7
:10603A00E0918A0905C0A0918909BB27E0918809E6
:10604A00F0E031960E94B8563596DF01E5E0F0E0BF
:10605A000E943E5D08951A9310918B09E0918A0976
:10606A00E11781F0A9E01A9FF001E45AF64FE081A6
:10607A00E13011F0E23011F4E1E041C01A93CADFD5
:10608A001E2FECCFE0E03BC01A930E946B1FE1EB9E
:10609A00F7E00E948856E1E2F0E00E948D5610E097
:1060AA00133050F40E941E58AFEFA0830E94185874
:1060BA000E9424581F5FF4CFE6E1F8E0FA93EA93CE
:1060CA00EFEF0E9439560E94054FE091E607E37010
:1060DA0019F00E94F75809F402C0689401C0E894C4
:1060EA0021F8EFEFE093A609E0915A0DE03029F488
:1060FA0008D03FD1E89420F802C00E94BC0619914A
:10610A0008950E94575F00E0033058F40E945959DD
:10611A00A0E00E945F59EC54F84FA0E0A0830F5F03
:10612A00F3CF00E0033078F50E942958E081EF3F71
:10613A0041F10E942958E0810E94E156B1F00E9483
:10614A002F58DF010E94815D0E94F953EA17FB076D
:10615A0041F00E942F580E94F953A083B1830E94F4
:10616A0064590E945959A1E00BC0ABE00A9FF001A3
:10617A00E554F84FE081E03021F40E942958AFEF4E
:10618A00A0830F5FCFCF0E948F1D1E2F1F3F11F4D8
:10619A000C941F3150E000E0033048F40E94295863
:1061AA00E0811E1711F451E002C00F5FF5CF5030A5
:1061BA00D1F500E00330B8F50E942958E081EF3F9D
:1061CA0081F50E94295810830E942F580E94F95382
:1061DA00A083B183ABE00A9FF001EB54F84FA09182
:1061EA009E0D0E945F59EA54F84FFF93EF930E9465
:1061FA00DC560E94CE53AF91BF91EC930E94645932
:10620A000E945959A1E00E945F59E754F84FFF9341
:10621A00EF930E94AC0CAF91BF91ED93FC9351E0C8
:10622A0002C00F5FC7CF503029F01A930E94961D03
:10623A001E2FACCF30E03830D8F550E000E0033004
:10624A0048F5503029F5ABE00A9FF001EA54F84FBF
:10625A0020812A930E9419180E945959E081E1303D
:10626A0059F42A930E946F1EE13031F4A32FAF5FD5
:10627A00E091150DEA1709F00BC00E94E351EA50AC
:10628A00F84F20830E94E351EA5EF74F008351E002
:10629A000F5FD5CF503051F40E94E351EA50F84FC6
:1062AA000E943A58EA5EF74FAFEFA0833F5FC3CF31
:1062BA0095C10E94595FAC81BD81EBE4EC93EC81FE
:1062CA00FD8131960E946C59EB54F84FE0810E948F
:1062DA00AF5100E00E947759EC91E03011F00F5F66
:1062EA00F9CF0E947759E0E2EC930F5FE02FAC817F
:1062FA00BD810E943F560E946C59E954F84FDF0154
:10630A000E94815D0E9451520E941A55EE81ABE0B3
:10631A00EA9FF001EA54F84F10811A930E94191863
:10632A0000E00E947759EC91E03011F00F5FF9CF4D
:10633A000E947759E8E7EC930F5F0E947759E0E2F1
:10634A00EC930F5F30E03A3068F4E02FAC81BD8106
:10635A000E943F560F01A2E0BDE00E947D590F5FE7
:10636A003F5FF1CF0E947759EC930E94605F2796B6
:10637A00089564970E94595F00E010E0133040F4DA
:10638A000E941E58E081EF3F09F40F5F1F5FF6CFAE
:10639A00033021F0A091A609A03009F406C0E0E07C
:1063AA00E093A609EA930E941107033021F4A09111
:1063BA00A609A13009F406C0E1E0E093A609EA9330
:1063CA000E94110710E0133058F5ABE01A9FF00154
:1063DA00DF01EE54F84FE081E03031F0FD01EC547A
:1063EA00F84FE081E03009F419C01A930E94355839
:1063FA0060DFABE01A9FF001EA54F84F30813A931C
:10640A000E9419181A930E9435580E941907ABE086
:10641A001A9FF001EC54F84FA0E0A0831F5FD3CF7E
:10642A000E94605F689608950E94575FA0915A0D76
:10643A00A23009F4D3C030E0343168F40E948459A0
:10644A000E946D56AF01DA011296E0E0EC93DA0190
:10645A00EC933F5FF1CF0E948F1D0E2F0F3F11F477
:10646A000C947A320E94DC560E94CE531E2F1F3F94
:10647A0031F0E09197091E1710F0103408F030C07F
:10648A00A0919709E12FEA1B3E2F343100F50E94B3
:10649A0084590E946D56AF01FA0132960F01E081CC
:1064AA00AE2F0E94FE53B0E0EA0FFB1FD001EC931F
:1064BA00FA01A281A43620F0DA011296E3E6EC93FF
:1064CA00DA01AC91AF3F19F4E02FDA01EC931A9399
:1064DA000E94DC56FA93EA930E94D8171E2FC7CF60
:1064EA000A930E94961D0E2FB9CF30E0343110F076
:1064FA000C94F3320E9484590E946D56AF01FA013E
:10650A00A381AF3F11F40C94F1320E9488590E9482
:10651A001918A091120DA07839F4FA010280DA0153
:10652A001196EC91E01509F457C0DA0113962C91F3
:10653A00ACE02A9FF001E55FFA4F0F01DA011296EB
:10654A00EC91D001EC930E9488590E94841FEF3F7E
:10655A0041F0ACE02A9FF0010E942757E058DB0186
:10656A00EC93DA011296EC91E030B1F0ACE02A9F9C
:10657A00F001E95FFA4FDF01E091100DE295EF704B
:10658A00EC93ACE02A9FF001E85FFA4FDF01E0915B
:10659A00100DEF70EC930EC0ACE02A9FF001E85F9B
:1065AA00FA4FA7E0A083ACE02A9FF001E95FFA4F17
:1065BA00A8E0A0830E9488590E94841FEF3F19F027
:1065CA00ECE0E093F505DA011296EC91DA01119606
:1065DA00EC932A930E9491523F5F88CF0E945E5F9C
:1065EA0026960895E7E0E09390090E946217A8951D
:1065FA000E94941BA8950E94D81DA895EFEFE093DE
:10660A002A0DE093010DE093A80DE093A30D0E94DB
:10661A00E454EC7F29F0A0E0B0E0E0E00E94B75D2E
:10662A0008950E948E5999F0E0E0E093B10A10E0D3
:10663A0000E00E9456520E94945949F00E94565214
:10664A000E9499590E9456520E949C59F2CF099170
:10665A00199108951A930A930091470DAA81A534B6
:10666A0011F4E0E062C0AA81A23539F4A091AD0923
:10667A00A13019F40E94875309F405C00E94811BB6
:10668A00E0E0E093AD09AA81AB3411F0A33599F4A7
:10669A00E02FE470E43011F414E001C013E0E02FBD
:1066AA00E270E23009F41C5FE02FE170E13009F496
:1066BA001F5FE12F3AC0AA81A13511F0A13799F4E1
:1066CA00E02FE470E43011F417E001C016E0E02F87
:1066DA00E270E23009F41C5FE02FE170E13009F466
:1066EA001F5FE12F22C0AA81A33441F413E0E02FF7
:1066FA00E170E13009F41F5FE12F17C0AA81A737C3
:10670A0041F417E0E02FE170E13009F41F5FE12F57
:10671A000CC0AA81A03441F415E0E02FE170E13009
:10672A0009F41F5FE12F01C0EFEF19810881239659
:10673A00089524970E94575FA091B80AA53411F0D2
:10674A000C947034E0E0E093AD090E94E457E0E075
:10675A00E093D50CE0914B0DE03081F5E09188098A
:10676A00A0918909EA1739F00E94A259E15DF64F12
:10677A00E081E13009F022C0E7E7EA930E948E3E09
:10678A000E94A259EE5CF64FE0810E9411520E94CB
:10679A00A859E05DF64FDF010E94E9540E94A8590A
:1067AA00ED5CF64FE0810E941554E2E0E093AD09FA
:1067BA000E94A259E15DF64FA2E0A083E091AD09E3
:1067CA00E03011F00C9463340E94875311F40C9456
:1067DA004C340E94761BE1E0E093AD09A091470D8D
:1067EA00A87081F00E949853E8EEF3E00E940C5DD5
:1067FA00DF010E944D5F14F4E1E301C0E0E3EA9394
:10680A000E948E3EE091990D0E941152E2E0F0E062
:10681A00FA93EA930E94EB3EA091470DA47091F07F
:10682A000E949853E0E1F7E20E943E5DAF01A09119
:10683A00470DA07111F0415050405A934A93E4E039
:10684A00F0E00FC00E9498530E94F258AF01A09145
:10685A00470DA07111F0415050405A934A93E3E01A
:10686A00F0E0FA93EA930E94EB3EA091470DA072E2
:10687A0029F00E949153E4E0F0E004C00E94915391
:10688A00E3E0F0E0FA93EA930E94EB3E17C018E0C7
:10689A00A091470DA47009F01F5FA091470DA87041
:1068AA0009F01F5FA091470DA07209F01F5F0E94B7
:1068BA00A051E12F0E9411520E94EB3EA091470D78
:1068CA00E1E0EA23E13029F4E091D50CEA930E9451
:1068DA008E3E0E94AF59A091B80AA73729F4E2E088
:1068EA00E093AD09E03009F479C00E94E457E2E58B
:1068FA000E94EB5796DEE9EBFAE00E948A581E2FB7
:10690A000E948F58AF01E1E0EA930E94083E0E2FE1
:10691A00E0918809A0918909EA1739F00E94A259E1
:10692A00E15DF64FE081E23009F055C00E94A259BC
:10693A00E05DF64FDF010E94815D4E175F0711F09F
:10694A000C94EA340E94A259EC5CF64F0080118044
:10695A000E941953D0010E945F5379F10E94A259F3
:10696A00EC5CF64FDF010E94B5590E94A259EC5C1B
:10697A00F64FDF010E94815DE452F34F0E94BF5936
:10698A000E9462550E94C359E12F0E9411520E942F
:10699A006F53E1E8F8E00E948D53003029F05A93D2
:1069AA004A930E94C03E04C0E0E3EA930E948E3EEE
:1069BA000E94A8530E942C4008C0003031F00E9467
:1069CA00C65918F40A930E945F58E0918909EA931C
:1069DA0021DBE0938909E0E0E093AD09A091B80AD0
:1069EA00A33419F422DBE03009F40DC00E94E45705
:1069FA00E2E50E94EB5715DE0E94B3530E94A051B4
:106A0A001DD30E94251CA091B80AA03419F40DDBED
:106A1A00E03009F427C0E9EBFAE00E948A58E887D7
:106A2A00F987E2E0EA930E94083E1E2F0E94F35380
:106A3A000E947B170E94E152E35AF64F0E94E053EC
:106A4A000E94E152E15AF64F10830E94E152E45A41
:106A5A00F64FA7E00E94E7520E94E457E2E50E943F
:106A6A00EB57DFDDA091B80AAB3439F0A33529F032
:106A7A00A13519F0A13709F074C00E94051C33979B
:106A8A001CF0D3DAE03009F466C00E94E4570E9491
:106A9A00CD59E9EBFAE00E944B55A091470DE2E08F
:106AAA00EA23E23029F4E4E0EA930E94083E02C0B5
:106ABA00E1E0F0E0E887F987A091B80AA13511F082
:106ACA00A13721F40E948F581E2F02C010915D0D2C
:106ADA00A091470DE4E0EA23E43011F4E4E001C0B8
:106AEA00E3E0EA930E94083EAF01A091B80AA335F9
:106AFA0011F0A13731F4E885F9850E94815CE887B5
:106B0A00F9870E94C65920F0A0914B0DA130C9F413
:106B1A001A935A934A93EB85FC85FA93EA930E9457
:106B2A00441CEE83FF83AF81AA235AF40E94E457E0
:106B3A00E6E6EA930E948E3E0E943653AF81AA236C
:106B4A00BAF31A935A934A93EB85FC850E940B5425
:106B5A000E94AF5906C00E94B3530E94A0510E94DE
:106B6A00441C0E945E5F2A9608950E94D159E894B7
:106B7A0022F80E945D55E2E7EA930E948E3EE09178
:106B8A00B309EA930E948E3EEFE0EA930E948E3E9A
:106B9A00A091B009AA3221F41A930E94720D1BC067
:106BAA00A091B3090E945652E452F34FE081EA17CA
:106BBA0021F4E091B309E03351F40E94EE54A45257
:106BCA00B34FE091B309EC931A930E94720D22FC21
:106BDA0002C00E942C4036C00E94D159E091B309EC
:106BEA00E053AE2F0E945652E351F34FE081EA1769
:106BFA0049F51A930E94720DA091AE09A23019F4B8
:106C0A000E94D95909F402C00E94DF59A091AE0925
:106C1A00A33019F40E94D95909F402C00E94DF591D
:106C2A00E0E0E093AE09E093030E0E945652E3516E
:106C3A00F34FBF01E081EF5FAE2FEAE00E943B5DB8
:106C4A00DB01EC93199108950E94595F25FCF3C169
:106C5A000E94D95911F40C946D370E940F54E55AC9
:106C6A00F64F9F01D9011196EC91E43071F50E941B
:106C7A00E7590E94F459F901A481A03021F4A281B4
:106C8A00B381109709F007C0E4E8F8E00E948D5339
:106C9A000E94A85315C00E94C3590E94FB590E9422
:106CAA006F53E7E8F8E00E948D530E94005A0E9451
:106CBA002054F901A681B781BA93AA930E94C03ED3
:106CCA000E94065A0E94605F76C2E730C9F40E94A9
:106CDA00E7590E94F459EAE8F8E00E948D530E94AD
:106CEA00005A0E946F53EDE8F8E00E948D530E940B
:106CFA00FB590E94C03E0E94065A0E94605F5BC216
:106D0A00E93099F40E94E7590E94F459E0E9F8E061
:106D1A000E948D53D901EC910E9411520E946F5327
:106D2A000E94065A0E94605F46C2E63029F5EAE2EE
:106D3A00EA930E941040E3E9F8E00E948D53D901DA
:106D4A00EC910E941554E091450D0E941554EBE414
:106D5A00EA930E948E3E0E94FB590E94C03E0E9406
:106D6A000D5A0E94005A0E94C03E0E942C400E9466
:106D7A00DF590E94605F1FC2E530E1F4D90116961F
:106D8A000E94B559D9010E94115A0E9462550E9467
:106D9A00C3590E94FB590E946F53E1E8F8E00E9430
:106DAA008D530E94005A0E94C03E0E94065A0E94B9
:106DBA00605F01C2E83049F50E94E7590E94F45920
:106DCA00E6E9F8E00E948D53F901A481AA930E9492
:106DDA0019180E941555309719F00E94155504C0CC
:106DEA00D90114960E94155AFA93EA930E94C03E5A
:106DFA000E94A8530E942C40D9011196E0E0EC931E
:106E0A000E94DF590E94605FD6C1E13011F00C94F4
:106E1A004E37A0919109A53029F4E091450DE65F1E
:106E2A001E2F01C011E0E12FE05D0E94185A0E9456
:106E3A005652E351F34FE0810E9415540E94625565
:106E4A000E94C3590E94FB590E946F53E9E9F8E076
:106E5A000E948D530E94005A0E942054D90115960F
:106E6A00EC910E9411520E94C03EA0919109A53056
:106E7A0069F4EAE3EA930E948E3EF901A085AA9397
:106E8A000E9419180E941F550E940D550E941C5AF3
:106E9A0092C1E330E9F4D90116960E94815DF09619
:106EAA000E94185AD90116960E94815DE351F34F48
:106EBA00E0810E9415540E946255ECE9F8E00E94B4
:106ECA008D530E94005A0E94C03E0E941C5A73C1F0
:106EDA000E94875361F0A091AE09A03041F4A091BD
:106EEA004A0DA13021F40E941953E13009F42BC054
:106EFA00A091FD0CA03061F0E091FF0CF091000D23
:106F0A00FA93EA93E8EEF3E00E949858E130D9F454
:106F1A00E1E30E94185AE091EE0C0E9415540E9477
:106F2A0062550E941953EA930E942C0DE093AE0910
:106F3A000E942C400E94AC0CE093010EF093020ECA
:106F4A00E0E0E093FD0CA091AE09A03061F0E09181
:106F5A00010EF091020EFA93EA93E4E6F0E00E9441
:106F6A009858E13009F025C0A091AE09A23019F471
:106F7A000E94D95909F402C00E94DF59A091AE09B2
:106F8A00A33019F40E94D95909F410C0A091030E34
:106F9A00A33030F00E94DF59E0E0E093030E06C010
:106FAA000E940F54E45AF64FA8E0A083E0E0E09371
:106FBA00AE09A091FE0CA130F1F5E091AE0DA091C1
:106FCA00AD0DEA1799F1EAE20E94185AE091EC0C29
:106FDA000E9415540E946255E091AE0DEA930E94F8
:106FEA009C1D0E94C359E0919E0D0E9411520E945D
:106FFA006F53EFE9F8E00E948D530E94DC56FA9332
:10700A00EA930E9420540E94FE530E9426540E9432
:10701A002C40E091AE0DEA930E941C1CE091AE0D4B
:10702A00EA930E94EF1BE093AE0D05C0E0E0E09307
:10703A00FE0C689420F80E94605FBDC00E941A305E
:10704A00E030E9F00E94E152E35AF64FAA81BB818F
:10705A00A083B1830E94E152EF59F64FA881B9810A
:10706A00A083B1830E94E152E15AF64FAC81A0831A
:10707A000E94E152E45AF64FA4E00E94E7520C94AF
:10708A00FC39F2D1E03031F4E5E0F0E00E9404533B
:10709A00A895F7CF0E94E457E2E0EA930E948E3E59
:1070AA00E0E0E093D50C0E942D5AE091040E0E9474
:1070BA001554A091040E0E94315AE093040E0C94C8
:1070CA00793D1A930A93E3E0EA930E948E3EE09197
:1070DA00D50C0E94365AE091D50C0E943D5A0E9466
:1070EA00EB5710E00E9456520E94945931F00E94C8
:1070FA0056520E9499591F5FF5CF09911991089527
:10710A000C94793D58C008950E944A5AE7E4EA93DC
:10711A000E948E3EEA81FB81F096EA930E948E3E9F
:10712A00E881F981F096EA930E948E3ECADFEA81ED
:10713A00FB81E0934207F0934307E881F981E093EA
:10714A004407F093450737C00E944A5AE6E4EA9397
:10715A000E948E3EEA810E941554E9810E941554CC
:10716A00E8810E9415540E94E454E2700E9415546A
:10717A00A8DF5BC00E944A5A0E94CD59E9810E9449
:10718A001554E8810E9415549CDF229608950E94A6
:10719A004A5AE4E54FC00E944A5AE3E4EA930E943D
:1071AA008E3EE0E347C00E944A5AE3E4EA930E9413
:1071BA008E3EE1E33FC0249608950E944A5A0E94F7
:1071CA004F5AE0E337C00E944A5A0E944F5AE3E3FB
:1071DA0031C00E944A5A0E944F5AE1E32BC00E94D2
:1071EA004A5A0E944F5AE2E325C00E944A5A0E9414
:1071FA000D5A0E942D5A65DF0E94535A0C94793D0C
:10720A001A930E944A5A0E940D5A10E00E94575A35
:10721A00EC91E03041F00E94575A0E94115A1F5FC8
:10722A000E94535AF3CF4DDF1881239608950E9486
:10723A004A5AE9E4EA930E948E3E43DF08951A937C
:10724A000A930E944A5A0E940D5A00E010E00E94D6
:10725A005D5AE03021F00832E0E01E070CF00AC067
:10726A000E945D5AEA930E948E3E0E94535A0F5F13
:10727A001F4FEDCF26DF198108810C94063E1A9321
:10728A000A930E944A5A0E940D5A00E010E0F8013F
:10729A00AB81BC81AE0FBF1FAC91A03021F0EA8157
:1072AA000E94645A0CF00CC0F801AB81BC810E94A8
:1072BA005A530E948E3E0E94535A0F5F1F4FE7CFC8
:1072CA0000DF1981088193C06E970E94575F0E9460
:1072DA004A5AEBE4EA930E948E3EEDA50E941554A9
:1072EA00ECA5EA930E948E3EEBA50E941554EAA5EE
:1072FA000E941554E9A50E941554E8A50E94155448
:10730A00E0E0EE83EEA1FFA1309741F00E94695AB6
:10731A00E8A5F9A5FA93EA930E94304FECA1FDA1E2
:10732A00309741F00E94695AEEA1FFA1FA93EA93BD
:10733A000E94254F30E0343148F40E94E351DE01C7
:10734A001696AE0FBF1FAC91A03009F40AC00E9476
:10735A00E351DE0116960E945A530E948E3E3F5F09
:10736A00EACFAFDE0E945E5FAE960895E091BA0A58
:10737A00E03599F4E091BB0AEA93E6E0EA930E94C9
:10738A009044A091BB0AA03840F0E091BB0A0E9449
:10739A005952E091BB0A0E945F52E091BA0AE03763
:1073AA0011F40E9465520895EDE0E093F805E0E3D8
:1073BA00E09357070895AC81A03310F0AA3308F080
:1073CA0006C00E946E5AE0530E94765A0FC0AC81E2
:1073DA00A13410F0A73408F006C00E946E5AE75391
:1073EA000E94765A03C0A881B981E0E0EC93259601
:1073FA000895AA93EA93FA93EFB7EA931A930A9332
:10740A001BB10CB1E0913B0EF0E0E75FF14F008356
:10741A00A0913B0EAF5FA0933B0EA23319F4E0E0BC
:10742A00E0933B0E09911991F1C21A93E0913C0E37
:10743A00A0913B0EEA17D1F3F0E0E75FF14F10811C
:10744A00A0913C0EAF5FA0933C0EA23319F4E0E08A
:10745A00E0933C0EE12F8DC4E0913C0EA0913B0ECF
:10746A00EA1709F082C383C30E947F5A09F47DC3D5
:10747A007EC30A921A92FA926A937A938A939A9399
:10748A00AA93BA93EA93FA93EFB7EA930E947F5AC0
:10749A0049F0A091B10AA03021F00E941605E1300E
:1074AA0009F401C011C0E091A20EF0E0E35CF14FD3
:1074BA00E081ECB9A091A20EAF5FA093A20EA43610
:1074CA0019F4E0E0E093A20EE991EFBFF991E99196
:1074DA00B991A9919991899179916991F9901990A4
:1074EA00099018951A930E947F5A59F45D9B09C016
:1074FA00A091B10AA13021F40E941605E03009F0EA
:10750A0013C01091A10E0E945652E35CF14FA9815B
:10751A00A0831F5F143609F410E0E091A20EE11770
:10752A00E1F31093A10E02C0E981ECB94CC40E94A8
:10753A007F5A21F40E941605E13009F001C015C3F3
:10754A0016C30E94595F88DFE03011F40C94A43B03
:10755A006CDF1E2FA091080EA53618F0E0E0E0932C
:10756A00B20A3091B20AE091B20AE03011F00C94FA
:10757A000B3BA0915C0DA13021F0A0915C0DA230D3
:10758A0031F4E12FEF77E093B80AEBE4CEC01A3575
:10759A0021F4E1E0E093B20ACAC0123049F4E4E10E
:1075AA00E093B20AE0E0E093B30AE093B50ABFC001
:1075BA00A0915C0DA33069F4173729F01A3310F43F
:1075CA00103308F402C0E7E001C0E0E0E093B40A37
:1075DA0005C01A930E942F33E093B40AA091B40A0B
:1075EA00AF3F99F01093B80AE1E0E093B30A109321
:1075FA00B50AE091B40AE03011F4E5E404C0EAE027
:10760A00E093B20AE0E0E093B70A91C0E13069F48E
:10761A00103039F4E2E0E093B20AE0E0E093B70A0E
:10762A0003C0E0E0E093B20A82C0E23059F410935A
:10763A00B40A1093B50AE0E0E093B30AE3E0E093FA
:10764A00B20A75C0E330F1F40E94855A0E948B5A3F
:10765A00EA0F0E94955AA9F4E091B50AE03071F454
:10766A00E4E0E093B20AE091B30A0E94E2550E9474
:10767A009E5A0E94855AA0E0A08303C0E0E0E093EE
:10768A00B20A55C0E43049F41D3019F4EAE5E09332
:10769A00B70AE0E0E093B20A4AC0EA3079F40E94FD
:1076AA00855A0E948B5AEA270E94955A31F4E0E0E3
:1076BA00E093B20AE5E4E093B70A39C0E431B9F4D9
:1076CA000E94855A1083E12FA091B50AEA27E09318
:1076DA00B50AE091B30AEF5FE093B30AE0E0E09302
:1076EA00070E133019F4E5E1E093B20A20C0E53140
:1076FA0011F0E63159F41A93E7E0FEE0FA93EA93BF
:10770A00E2EBFAE0FA93EA9356DE11C0E73179F434
:10771A00E0E0E093B20A173131F4E091070EA0914C
:10772A00B50AEA1709F003C0E3E4E093B70AA091A7
:10773A00B20A3A1719F0E0E0E093080E04CF5FC2EC
:10774A00AA93BA93EA93FA93EFB7EA931A930A932E
:10775A0010919B0000919C00E12FEC71A9F4E0913B
:10776A006B0FF0916C0FED55F14F0083ABE6BFE064
:10777A000E947F52E83CA0E0FA0731F4E0E0F0E032
:10778A00E0936B0FF0936C0F09911991E991EFBF98
:10779A00F991E991B991A99118951A930E94A35A5E
:1077AA000E94A85AD9F30E94A35AED55F14F1081AD
:1077BA00ADE6BFE00E947F52E83CA0E0FA0731F450
:1077CA00E0E0F0E0E0936D0FF0936E0FE12FD1C28D
:1077DA000E94A35A0E94A85A09F0C7C1C8C10E94B0
:1077EA00595FF6DFE03021F0A091060EA03009F0D3
:1077FA00E5C0D3DF1E2FA091770FA53618F0E0E081
:10780A00E093710F3091710FE091710FE03059F4EC
:10781A00113019F4E4E0E093710F1A3519F4EAE033
:10782A00E093710FC3C0E430C1F4E0E0E093710F5C
:10783A001A3229F00E941953E05DE11769F4109396
:10784A00B0091093720FE5E0E093710FE0E0E09366
:10785A00060EE1E0E093740FA9C0E530A9F4E0E078
:10786A00E093710F0E941953E05DE11761F00E94E5
:10787A00AF5A0E94B85AE091740FEF5FE093740F09
:10788A00E6E0E093710F92C0E63091F4E091740F54
:10789A000E94B85A0E94AF5AEF5FE093740FE0E07B
:1078AA00E093750F133019F4E7E0E093710F7EC08F
:1078BA00E73011F0E83059F41A93E5E7FFE0FA935C
:1078CA00EA93E1E7FFE0FA93EA9375DD6FC0E930E6
:1078DA0081F4E0E0E093710F173131F4E091750F14
:1078EA00A091720FEA1709F003C0E4E5E093060ECF
:1078FA005DC0EA3041F4103011F4EBE001C0E0E081
:10790A00E093710F53C0EB3071F4E0E0E093740F31
:10791A001093730F1093720FECE0E093710FE0E095
:10792A00E093060E43C0EC30A1F5E091740FF0E04D
:10793A00E854F54F10830E94AF5AEF5FE093740F3B
:10794A00E091730FE150E093730FA091730FA03091
:10795A0021F4A091720FA03009F00EC0EDE0E0937F
:10796A00710FE091740F0E94E2550E949E5AE091B5
:10797A00740FF0E00E949E5AA091730FA03021F478
:10798A00A091720FA03009F403C0E0E0E093710FF8
:10799A000DC0ED3059F4E0E0E093710F1D3031F481
:1079AA00EAE5E093060EEFEFE093050EE091710F22
:1079BA00E31719F0E0E0E093770F13CF20C1AA9301
:1079CA00EA93FA93EFB7EA93E0917910A0917810CD
:1079DA00EA1791F0E091AF09E03019F0E89426F83F
:1079EA000AC00E94BD5AF0E0E030A1E0FA0719F49B
:1079FA00E0E0E093791003C0E89425F826F8E091D6
:107A0A00050EE03019F0E0E0E093710FE991EFBF65
:107A1A00F991E991A99118951A93E0917910A09199
:107A2A007810EA1721F4E0919B00E072C1F4E0912A
:107A3A007810F0E0E858F04FA981A08310917810EF
:107A4A001F5F0E94EE54A030E1E0BE0709F410E087
:107A5A00E0917910E117E1F31093781003C0E981FE
:107A6A00E0939C00B0C1E0E0E0937910A091781017
:107A7A00A13020F00E94BD5A689426F80895AA936E
:107A8A00BA93EA93EFB7EA93E091050EE03041F436
:107A9A00E0E0E09379100E941953EF5FE093AF0999
:107AAA00E991EFBFE991B991A99118950E9475538F
:107ABA00A03220F00E947553AB3309F403C00E9430
:107ACA001D54F4CF0E947553AB3311F40E941D5418
:107ADA0008950E947553E881EA1729F40E941D54FB
:107AEA003197E1E001C0E0E0219608950E94CB5A67
:107AFA00EEE20E946E54F9F420E030E0EC81D90104
:107B0A00F0E0AE17BF07BCF40E94D05A8F010E9462
:107B1A007553A03320F00E947553AA3308F008C0A9
:107B2A000E947B530E94D65A0E0F1F1F0E941D549B
:107B3A002F5F3F4FE3CFF8010E94605F6AC20E9445
:107B4A007553A03228F00E943855E181E03208F4DA
:107B5A000EC00E947B53E093BA0C0E941D540E94EF
:107B6A007B53E093BB0C0E941D54E1E00895E0E0D2
:107B7A0008951A930A9310E00E9446550C910B330C
:107B8A0011F0003208F412C0013310F0093308F082
:107B9A0007C0E02F0E94D65AE255FF4FE4911E2BF0
:107BAA000E941D540E9446550C91E9CFE12F6FC2E5
:107BBA000E94CB5A0E947553AD3229F40E941D547B
:107BCA002FEF3FEF02C021E030E00E947553A0334F
:107BDA0020F00E947553AA3308F00DC00E94D05AB3
:107BEA000F010E947B530E94D65AE00DF11D8F01AE
:107BFA000E941D54EACFF901D8010E94E15C0E945B
:107C0A00605F249608950E94595F20E030E000E00A
:107C1A0010E0EC810E94645A94F4D901EAE0F0E0A1
:107C2A000E94E15C0F010E947B530E94D65AE00D2C
:107C3A00F11D9F010E941D540F5F1F4FEACFF901EA
:107C4A000E94605FE6C10E94CB5A20E030E00E94A9
:107C5A007553A03320F00E947553AA3308F017C059
:107C6A00AC81A13050F00E94D05A0F010E947B5380
:107C7A000E94D65AE00DF11D8F0131E0213018F033
:107C8A00AC81A13008F403C0EC81E150EC830E947E
:107C9A007553AE3211F422E031E0313011F40E9412
:107CAA001D54313099F2AC81A13038F00E94D05A7B
:107CBA008F01EC81E150EC83F6CFF8010E94605FFE
:107CCA00A8C11A9310E00E941954E030E9F00E940A
:107CDA007553A03258F00E947553A23239F00E94AF
:107CEA007553AB3319F0E9811E1708F00DC00E94D5
:107CFA005652E454F34F0F010E947B53D001EC9388
:107D0A001F5F0E941D54E3CF0E9456520E9469547D
:107D1A005AC0E8810E944055E881A091D40CEA0F2C
:107D2A00E093D40CE881A091D50CEA27E093D50C16
:107D3A000C94D6421A9310E00E94D95AE491E0308A
:107D4A0039F00E94D95AE491EA93E3DF1F5FF4CF36
:107D5A000C94FC431A9310E00E9456520E94DD5A7A
:107D6A0041F00E945652E454F34F0E94BF591F5FDC
:107D7A00F3CF199108950E947954E2EAF8E0FA9350
:107D8A00EA93EC81FD810E9451520E941A55E2DF6A
:107D9A001BC01A93ECE3EA93BCDF11E0193080F4BC
:107DAA000E945652E255FF4FE491A981EA2319F045
:107DBA00E12FE05D01C0E0E2EA93ABDF1F5FEECFA7
:107DCA00EEE3EA93A6DF1881229608951A930E9499
:107DDA007954EAEAF8E0FA93EA93EF81F8850E9487
:107DEA0051520E941A5510E00E945652E454F34F21
:107DFA00E081E03241F40E945652E454F34FA0E38A
:107E0A00A0831F5FF1CFA981BA81EAE0F0E0EA1B03
:107E1A001E2F0E9456520E94DD5A41F00E9456526D
:107E2A00E454F34F0E94BF591F5FF3CFF1C00E9481
:107E3A00E25AE2EAF8E0FA93EA93EE85FF85688966
:107E4A0079890E94945D0E941A5584DF0E94A85382
:107E5A000C9410441A93E2E2EA935BDF10E00E946A
:107E6A00575AEC91E03031F00E94575A0E94115A49
:107E7A001F5FF5CFE2E2EA934CDF0C94FC431A93BE
:107E8A0010E00E94575AEC91E03031F00E94575AA4
:107E9A000E94115A1F5FF5CF0C94FC431A930E945B
:107EAA007954EFEAF8E0FA93EA93AD81BE81E4E609
:107EBA00F0E00E940C5D0E945152A985BA85E4E661
:107ECA00F0E00E943E5D0E9451520E94E75A10E083
:107EDA000E9456520E94DD5A91F00E945652E45472
:107EEA00F34FE081E03211F4E0E305C00E945652FC
:107EFA00E454F34FE081EA930CDF1F5FE9CF0C945F
:107F0A00FC4324971A93E0E0E983EA83EB83EC834A
:107F1A00AD81BE810E94155AE055F64F108110338B
:107F2A0010F01A3308F022C0A981BA818B819C8192
:107F3A00EAE0F0E060E070E00E94E65CDF01CB017D
:107F4A00E12FE053FF27662777270E947C5CE983AD
:107F5A00FA836B837C83AD81BE81EC91EF5FEC93F6
:107F6A000E94155AE055F64F1081D9CFE981FA815E
:107F7A006B817C81188199C00E94CB5AAC81BD81EA
:107F8A000E94155AE055F64F3081303310F03A33DB
:107F9A0008F013C00E94D05ADF01E32FE0530E9479
:107FAA003F568F01AC81BD81EC91EF5FEC930E944B
:107FBA00155AE055F64F3081E8CFF8010E94605F0C
:107FCA0097C01A9310E0AB81BC810E94155AE05504
:107FDA00F64FE081E03210F0EB3708F015C00E944E
:107FEA00D95A0F01AB81BC810E94155AE055F64F50
:107FFA00E081D001EC93AB81BC81EC91EF5FEC9313
:10800A001A3008F41F5FDFCF0E94575AEC93E12F12
:10801A0018812596089525FE06C0E5E0F0E00E9445
:10802A000453A895F8CFE8E7FFE0E093D60CF09365
:10803A00D70CE1E0EA936DDEE0E0E093D40C0E9415
:10804A002D5A0E9419530E9415540C94D6421A9321
:10805A000A93E091050EE030D1F4E3E0EA9359DEA9
:10806A00E091D40C0E94365AE091D40C0E943D5AF9
:10807A00EA934FDEE8E7FFE0A091D60CB091D70C67
:10808A000E94A45DEA1BE0937810689425F8099190
:10809A0019910895EE81EA93BEDFEC81FD810E9479
:1080AA008D530E94EC5AC3DED2DF27960895EB81E6
:1080BA00EA93B1DFE981FA810E948D530E942D5A19
:1080CA00C6DF0C949E43ED81EA93A5DFEB81FC8128
:1080DA000E948D53EA81EA931CDEE981E03011F0B7
:1080EA00EA9317DEE881E03011F00E942D5AAFDFE3
:1080FA00269608950E94575F10E0E6EBF8E0A885FF
:10810A00B985EA17FB0719F444E150E002C048ECCC
:10811A0050E0EA85E093B00AE89431F8EA93E985F9
:10812A00FA85FA93EA93EA85EA93EA85EA93E0E024
:10813A00EA93C9DF0E94AC0C9F010E9486083A9319
:10814A002A935A934A930E94B80C0E2F31FC02C00C
:10815A00003009F001C0F1CF31FE07C0E89431F8D0
:10816A00E1E00E945E5F0C9443431F5F123088F285
:10817A00E0E00E945E5F0C9443430E948E5911F422
:10818A000C945C45E0E0E093B10AE2E0EA93AAD9F4
:10819A0010E003E00E9456520E94945961F00E9436
:1081AA0056520E9499590E945652E854F44FE0815F
:1081BA000E271F5FEFCFE3E0EA9394D9E02FE29511
:1081CA00EF700E94F35AE02FEF700E94F35AE7E132
:1081DA00EA9388D90C945C450E948E5911F40C9448
:1081EA005C450E94DF54E03021F0E091BA0BEA329C
:1081FA0009F405C00E94DF54E05DE093BA0BE0E0A9
:10820A00E093B10AEAE5EA936DD9E0E0EA936AD924
:10821A0010E00E9456520E94945911F01F5FF9CF44
:10822A001F5F012F0A935ED910E00E9456520E94E6
:10823A00945949F00E9456520E9499590E945652E6
:10824A000E949C59F2CFE02FE195EA934BD9EDE0D9
:10825A00EA9348D90C945C451A930A93F894E0E09F
:10826A00E093AF09E0917910E09378107894E09167
:10827A00B80BE03011F40C945C45EAE5EA93CCDBE8
:10828A00E0E0EA93C9DB10E00E9456520E9494593A
:10829A0011F01F5FF9CF1F5F012F0A93BDDB10E0BA
:1082AA000E9456520E94945961F00E945652E85414
:1082BA00F44FE081EA93B0DB0E9456520E949C5927
:1082CA00EFCFE02FE195EA93A7DBEDE0EA93A4DB99
:1082DA000C945C45E881EA939EDEEAE5EA9319DDAF
:1082EA00E091B80AEA9315DD0E947B53E03029F049
:1082FA000E947B530E948153F7CFA9DE52C10E948C
:10830A002955E091B309EA9304DDE4E4EA9301DD37
:10831A00E091B109EA93FDDC14E00E945652E0555F
:10832A00F64FE081E43040F00E945652E055F64F95
:10833A000E94BF591F5FF1CFE0E0EA93EADC4CDF0D
:10834A0018C31A930E94A63AE091B70AE03011F4D2
:10835A000C942342A091B70AAA3541F4A091B30A1A
:10836A00A33020F0E091B90AE43409F04BC00E942E
:10837A00DF54E03021F0E091BA0AEA32C1F40E94F7
:10838A001953E05DA091BA0AEA1721F0E091BA0AFE
:10839A00EA3221F40E9460161FDF08C0EBEBFAE014
:1083AA000E944B55E091BA0A0E94F95A2BC00E94CA
:1083BA00DF54E05DA091BA0AEA1721F50E94195329
:1083CA001E2FE091BB0AED3421F4E091BC0AE3329E
:1083DA0009F007C0EDEBFAE00E944B55E9DB1E2FCE
:1083EA0065DB0E941953E11729F0E12FE05D0E9435
:1083FA00F95A08C00E941953E05DE093BA0A0E9434
:10840A006016EADEA091B70AA53449F4A0915C0D82
:10841A00A33019F40E94C82802C00E949E33A0917A
:10842A00B70AA33411F40E94BB39A091B70AAB343E
:10843A0011F40E94C328E0E0E093B70AA0915C0D12
:10844A00A33011F40E94C828E0E093C2C8D9A091D1
:10845A00060EA43529F4A0E025FCA1E0A03009F01D
:10846A003CC0E091B209E03579F4E091B309EA93AE
:10847A00E6E0EA9350D2A091B309A03820F0E09147
:10848A00B3090E94595226C0E03739F4E0E0F0E01F
:10849A00E0934E07F0934F071DC0EA3519F40E9486
:1084AA00D21618C0EA3711F42ADF14C0E23519F4DB
:1084BA000E94BA350FC0E23719F40E94F1350AC09A
:1084CA000E94DF2CE091B109A091B00AEA1711F4D9
:1084DA00689431F8E0E0E093060EA091060EAA3502
:1084EA0031F40E946016B8DEE0E0E093060E11C295
:1084FA00A0E025FCA1E0A13049F4A0E026FCA1E01F
:10850A00A03021F4A091AF09A03009F001C0ABDA84
:10851A00E091AF09E03019F0E150E093AF09089516
:10852A00E091770FEF5FE093770FE091080EEF5F2E
:10853A00E093080EE091050EE03019F0E150E09367
:10854A00050E0895A0915C0DA13021F0A0915C0D5B
:10855A00A23029F4E3E0E0939000E8E3E9B9089552
:10856A00E881E03011F40E94005BA881A13021F477
:10857A00E0EDF4E00E94075BA881A23021F4ECED63
:10858A00F4E00E94075BA881A33021F4EAEEF4E04C
:10859A000E94075BA881A43021F4E0EFF4E00E9476
:1085AA00075B219608950E94005B08951A930A9327
:1085BA00E0E0E0935207E093530710E0143190F49F
:1085CA0000E0033068F4A3E01A9FF001E85AF84F7C
:1085DA00DF01EE27A00FBE1FE0E2EC930F5FF1CFA1
:1085EA001F5FECCF64C21A9311E0E981E11788F0AA
:1085FA000E945652E255FF4FE491AA81EA2319F0EC
:10860A00E12FE05D01C0E0E2EA930E94FA381F5FC1
:10861A00ECCFEDC00E94E25AEAEBF8E028C00E94D3
:10862A00E25A0E940C5B0E94295BF5C00E94E25A42
:10863A000E942E5B0E941A550E94295BF8C00E9474
:10864A00E25AE1EDF8E0FA93EA93EE85FF850E949B
:10865A0051520E941A550E94295BE9C00E94E25AAF
:10866A00E4EDF8E004C00E94E25AE8EDF8E0FA937B
:10867A00EA93EE850E94AF510E94295B2B960895DA
:10868A000E94595F10E0E1E3E093B00AE89431F800
:10869A00EA930E941040ECEDF8E00E948D5300E04E
:1086AA00E09155070E17E0F40E94FD51E85AF84F81
:1086BA00E081E03258F4E3E2EA930E948E3E0E949F
:1086CA00FD51E85AF84FE081E05D05C00E94FD5176
:1086DA00E85AF84FE081EA930E948E3E0F5FE0CF9E
:1086EA000E942C400E94AC0C9F010E9486083A937B
:1086FA002A93E8ECF0E00E9498580E2FA0E031FC93
:10870A00A1E0A03011F4003009F001C0EECF31FE33
:10871A0007C0E0E0E0935507E89431F8E1E007C0CC
:10872A001F5F123008F4AFCFE0E0E09355070E94D4
:10873A00605F24960895E0915407E03021F4E881BF
:10874A00EA930E94773AA0915407A13021F4E88174
:10875A00EA930E94113DA0915407A230F1F4E091EE
:10876A005507F0E0E85AF84FA881A083E091550731
:10877A00EF5FE0935507E0915607EF5FE0935607E6
:10878A00A03218F4EF5FE0935607A0915607A7337B
:10879A0021F476DFE0E0E09356070C942E48A0918E
:1087AA005407A13039F4E8ECF0E00E940453E9E1FF
:1087BA00E0939900A0915407A23021F461DFE0E030
:1087CA00E0935607E0E0E09354070895EDE0EA935A
:1087DA00B2DFEAE0EA93AFDF08951A9310E0E98185
:1087EA001E1728F4EA81EA93A6DF1F5FF8CF1881E3
:1087FA0023960895EDE201C0EDE3EA93E8E2EA93F5
:10880A00ECDFE4DF08950E94E25A0E940C5BFE014D
:10881A000E9488560ED02E9608950E94E25A0E940F
:10882A002E5B0E941A55FE010E94885602D02C9691
:10883A0008951A930A9310E0EA81E03011F408E2ED
:10884A0001C00A81AB81BC81EE27A10FBE1FAC918A
:10885A00A03011F0101708F007C0AB81BC810E944C
:10886A00365B0E943B5BEECFEA81E03039F0EA8169
:10887A001E1720F4E0E20E943B5BF9CF19810881C0
:10888A000C94B0481A930A9310E0EA81E03011F48C
:10889A0008E201C00A81E12FAB81BC810E943F56E8
:1088AA00E491E03011F0101708F009C0E12FAB8114
:1088BA00BC810E943F56E4910E943B5BECCFEA8167
:1088CA00E03039F0EA811E1720F4E0E20E943B5BB7
:1088DA00F9CF198108810C94B048E0919807A091CA
:1088EA009707EA17B1F00E94405B0E941B57EC9170
:1088FA00E0939A070E94405B0E94CE54E181E09384
:10890A009907A09198070E94315AE0939807E1E0ED
:10891A000895E0E008950E94465BA981A0830E9421
:10892A00465B3196A881A083A09197070E94315A8D
:10893A00E093970722960895E091B00708951A9355
:10894A00E091B007E03059F40E9486080E94495924
:10895A0021F4A091B007A03009F001C0F5CF109121
:10896A00B007E0E0E093B0070E94495909F011E22C
:10897A00E12F199108950E94595F0E94AC0C8F0152
:10898A000E948608EC81FD81E00FF11FFF93EF93AF
:10899A000E94AC0CAF91BF91AE1BBF0B9D0100248E
:1089AA00021603061CF40E94495909F001C0E8CFD7
:1089BA00E0E00E94605F0C946B480E94595F30E0CF
:1089CA00EE81ACE0EA9FF001E65FFA4F108116FFF4
:1089DA0017C0E12FEF730E2F0E944C5B11F03A3053
:1089EA0008F008C00E94545B0E94E3510E945B5B3E
:1089FA003F5FF2CF0E94545BEE27A30FBE1FEC939A
:108A0A0017FF17C0E12FEF730E2F0E944C5B11F076
:108A1A00343108F008C00E94615B0E94E3510E9451
:108A2A005B5B3F5FF2CF0E94615BEE27A30FBE1F25
:108A3A00EC93B4C11A930A930E94685B3097B9F118
:108A4A00E0914007F0914107309769F50E94685B11
:108A5A000E94905DE0934007F0934107309731F40C
:108A6A00E0E0F0E00E94075BE0E01AC00E946D5B64
:108A7A000E94685B0E94905DF595E7958F01D80189
:108A8A00E0E0F1E00E940C5DE0938700D801E0E0AD
:108A9A00F1E00E943E5DE09386000E946D5BE0E497
:108AAA00E0938B0004C0A0E4B7E00E94AB570991A1
:108ABA00199108950E94D03879DDE5E1E093AF0776
:108ACA00089568970E94575FE0EEF8E00E94885682
:108ADA00D9DE7CDEE0919B09E03059F0EBEEF8E05C
:108AEA000E948856CFDEE0919B090E9411520E9493
:108AFA00755B6CDE0E949C1930E03A3078F43A9348
:108B0A000E94AA52EFE0EA9394DEE32F0E94B55244
:108B1A000E94BB520E94795B3F5FEFCF6BDEE4EFAE
:108B2A00F8E0FA93EA93EFE0EA93ACDE0E949F52F0
:108B3A006ADE4CDE61DE4ADE00E0003110F00C94A1
:108B4A0049460E941953E017D9F5EAEFF8E00E9466
:108B5A00885698DE0E94FD51FA93EA930E94755B4B
:108B6A00E0E0E0939709A0919709A03438F5E091E5
:108B7A009B09EA93E0919709EA930E94DD180E9403
:108B8A00C5523097A9F0E0919709EA930E94191803
:108B9A000E94C552FA93EA930E947F5B73DE0E9499
:108BAA00C052EAE0EA9345DE0E94CE520E94795B07
:108BBA00E0919709EF5FE0939709D5CF07DE06DECC
:108BCA000E94FD510E945C5611F00C944746EAEF50
:108BDA00F8E00E94885656DE0E94FD51FA93EA9305
:108BEA000E94755B0E94845BE0E30E94685651F420
:108BFA0013E0EDB7FEB7FA93EA931F930E94C13FC1
:108C0A001F91AF01042E052AD9F11F5FEDB7FEB7F8
:108C1A00FA93EA931F930E94863F1F91EA8FFB8F74
:108C2A006C8F7D8F1F5FEDB7FEB7FA93EA931F93A0
:108C3A00FE013896FA93EA930E94E63F1F915A93EF
:108C4A004A930E947F5B1EDE0E94695AEAE0EA9319
:108C5A00F0DDEA8DFB8D6C8D7D8D0E94795B0E9423
:108C6A00845BE1E30E94685651F413E0EDB7FEB766
:108C7A00FA93EA931F930E94C13F1F91AF01C2CF9B
:108C8A00A5DDA4DD0F5F59CF8ADD0E945E5F6E9677
:108C9A0008950E94595FAC81BD81EC91E1702E2F3D
:108CAA000E948C5BE12F0E9411520E94FD510E948A
:108CBA00915BE4E0EA930E948538203019F4E7E0FA
:108CCA00F9E002C0ECE0F9E0FA93EA930E94243951
:108CDA000E94E45834970E9469580E94E9582FDE8E
:108CEA003E2F333409F431E20E9488383D3311F0C3
:108CFA00313209F402C0E1E02E273D3311F031325E
:108D0A0009F401C0CFCF3D3319F4AC81BD812C9356
:108D1A00E32F0E94605FDAC10E94595FAD81BE8174
:108D2A002C910E948C5BE12F0E9411520E94FD51EE
:108D3A000E94915BECE3EA930E94FA38EC81EA9391
:108D4A000E9485382A93ED81EA930E94F842EEE365
:108D5A00EA930E94FA380E94955B0E94E9580E94A1
:108D6A00985B333409F431E2313320F0EC81E05D71
:108D7A00E31708F407C0E32F0E94D65AE255FF4FC3
:108D8A00E4912E273D3311F0313209F401C0CBCFE3
:108D9A003D3319F4AD81BE812C93E32F0E94605FAD
:108DAA00279608950E94575F20E0AF81B8855C91AD
:108DBA000E948C5BE12F0E9411520E94FD510E9479
:108DCA00915BE2E0EA930E9485385A930E9433430A
:108DDA000E94955B0E94E9580E94985B303310F01C
:108DEA003A3308F00EC0203009F450E021E0A52FF4
:108DFA00EAE00E943B5DAAE0EA9FF001E30FE0533C
:108E0A005E2F3B3211F4533608F001C05F5F3D32EA
:108E1A0011F4513008F401C05150333429F4203090
:108E2A0009F431E250E020E03D3319F4EE81E51710
:108E3A0008F005C0AF81B8855C9130E020E03D3391
:108E4A0011F0313209F401C0B5CF3D3319F4AF81C5
:108E5A00B8855C93D0C00E94575F20E0AF81B88587
:108E6A004D915C910E948C5BE12F0E9411520E94ED
:108E7A00FD510E949D5BAE81A23031F4FA010E943D
:108E8A0051520E94144304C05A934A930E941B43AE
:108E9A000E94955B0E94E9580E94985B303310F05B
:108EAA003A3308F022C0203011F440E050E021E0CB
:108EBA004031E7E25E0734F0DA01E0E1F7E20E94CE
:108ECA003E5DAF01493BEBE05E0724F0DA010E9408
:108EDA00F258AF01DA01EAE0F0E00E94E15CDF015A
:108EEA00EE27A30FBE1FD097AD013B3221F44033CA
:108EFA00E5E75E070CF002C04F5F5F4F3D3221F499
:108F0A000024041605060CF002C0415050403334C8
:108F1A0031F4203009F431E240E050E020E03D3302
:108F2A0011F0313209F401C09FCF3D3321F4AF81F2
:108F3A00B8854D935C935FC00E94575F0E948C5B1B
:108F4A0020E050E04FEFE12F0E9411520E94FD51A4
:108F5A000E949D5BEF81F885FA93EA93E885EA938C
:108F6A000E944439E52FE10F0E9411520E94FD51DF
:108F7A000E94E9580E94985B303310F03A3308F0A7
:108F8A0022C03053431729F04F3F09F05F5F20E0BA
:108F9A0005C0A22FAF5FEA2FE3702E2FE52FAF8116
:108FAA00B8850E943F560F01E32FA8E8B6E0F0E02B
:108FBA000E94995CAE0FBF1FE22F0E943F56E491B8
:108FCA00D001EC93432F3B3219F4EE815E1708F07F
:108FDA0002C05F5F4FEF3D3211F4513008F402C016
:108FEA0051504FEFEE815E1720F4313211F03D33CC
:108FFA0009F401C0A8CFE32F0E945E5F2996089565
:10900A001A930A93A091120DECEDEA231E2F00E0A9
:10901A000C3040F40E9495543A96E491E11711F00D
:10902A000F5FF6CF0E9495540E946451E02FEAC365
:10903A00A2E1BDE0E8810E943556EC91E17019F495
:10904A00E1E1F9E002C0E5E1F9E0FA93EA930E946E
:10905A002439219608950E94575F0E948C5BE12F64
:10906A000E9411520E94FD510E949D5BC9DF5E2F32
:10907A000E94955B0E94E9580E94985B3D3211F06C
:10908A00363311F4503009F401C051503B3211F01B
:10909A00333311F45B3008F001C05F5FA091120D09
:1090AA00E1E0EA232E2FACE05A9FF001E450FC4F96
:1090BA003A96E491E20FE093120D3D3311F031320A
:1090CA0009F401C0CCCFE32F0E945E5F2696089573
:1090DA000E94595F0E948C5BE12F0E9411520E94EC
:1090EA00FD510E949D5BEC81EA93A2DF0E94955B91
:1090FA000E94E9580E94985B303310F03A3308F026
:10910A0010C0A2E1BDE0EC810E943F560F01A2E12E
:10911A00BDE0EC810E943556AC91E1E0EA27D0012E
:10912A00EC933D3311F0313209F401C0D5CFA0914F
:10913A00120DE2E0EA232E2FE091130DED7FE22BD0
:10914A00E093130DE091140DED7FE22BE093140DE3
:10915A00E32F0E94605F259608950E94CE510E94D7
:10916A009D060E94A15B0E94A0510E9489380E941C
:10917A00C052EAE0EA93E0DEE13209F46EC20E94EC
:10918A00A0510E94A0510E943952E9E1F9E00E94DF
:10919A006451EDE0FDE00E9488565DDEE13209F49B
:1091AA005CC20E94A0510E94A0510E943952EFE174
:1091BA00F9E00E946451EFE0FDE0FA93EA93EAE0F5
:1091CA000E94A55B09F449C20E94A0510E94A051C5
:1091DA000E943952E8E2F9E00E946451E4E2FDE0BB
:1091EA000E94AA5B09F439C20E94A0510E94A051B0
:1091FA000E943952EEE2F9E00E946451E6E2FDE093
:10920A000E94AA5B09F429C20E94A0510E94A0519F
:10921A000E943952E4E3F9E00E946451E1E1FDE081
:10922A00FA93EA93E3E60E94A55B09F416C20E9448
:10923A00A0510E94A0510E943952EDE3F9E00E9428
:10924A00645109DFE13209F408C210E0133010F06A
:10925A000C94B1490E94A0510E94A0510E94395217
:10926A00E12F0E94A058E3E4F9E00E9464510E94B1
:10927A00B25B0E948938A5E1BDE00E9456520E9465
:10928A00B65B09F4EAC1E9E0F0E00E94C3510E942A
:10929A008938A8E1BDE00E9456520E94B65B09F4E3
:1092AA00DCC10E94A0510E94A0510E943952E12FB4
:1092BA000E94A058EEE4F9E00E9464511A9308DF74
:1092CA00E13209F4CAC10E94B25B0E94BC5BE17040
:1092DA0049F40E94CA570E94CE540E94AA5B09F41C
:1092EA00BCC10AC00E94CA570E94CE540E94885626
:1092FA00B2DDE13209F4B1C10E94A0510E94A0512D
:10930A000E943952E12F0E94A058E0E5F9E00E943C
:10931A0064510E94B25B0E948938A1E2BDE0EE2747
:10932A00A10FBE1F2C913327EDB7FEB73197FA93E1
:10933A00EA933F932F93E0E0EA938DDD2F913F91DB
:10934A00E13209F48AC1A1E2BDE00E945652EA0F55
:10935A00FB1F20831F5F7ACF80C10E94595F10E0F4
:10936A001A930E941F590E94A15B0E94A0510E9459
:10937A00C15B0E94C0520E94B1520E9415550E94C0
:10938A00CA520E94A0510E9473510E941F550E9406
:10939A0051520E941443E7E0F0E00E94CC5BE09156
:1093AA00260DF091270D0E9451520E9414430E94EB
:1093BA00A0510E947951E7E5F9E00E946451E091D9
:1093CA000F0DEA930E943343E7E0F0E0FA93EA9341
:1093DA000E94795115DE0E94D05B00E00330D0F57F
:1093EA000E94A051E02FED5F0E9411520E9489381D
:1093FA000E94F257EA930E943343EBE2EA930E94F7
:10940A00FA380E94F957EA930E94D45B0E940058E6
:10941A0051F40E9408580E944A520E9451520E94D6
:10942A001443E3E707C00E9408580E944A520E9468
:10943A00CA52E9E4EA930E94FA380E94D05B0E9479
:10944A000B58EA930E943843E3E7EA930E94FA38FA
:10945A000F5FC4CF0E94A4443E2F3B3211F4103454
:10946A0008F001C01F5F3D3211F4113008F401C049
:10947A0011503D3439F41A930E9419186EDE1A936A
:10948A000E943918313209F06BCFE7C00E94595F48
:10949A0010E00E94D038012F0E94A0510E94A051D2
:1094AA000E948938EBE5F9E00E94645131E03630D8
:1094BA0020F5103800F50E94A0510E94E3510E9445
:1094CA00915B1A930E947218E12FEF5FEA930E9450
:1094DA00D45BA091A90DE1E00E94D75BA091AA0DEF
:1094EA00E7E00E94D75BE091E607EA93E8E0EA93B7
:1094FA000E94F84213953F5FDACF0E9447050E9407
:10950A00A4443E2F3D34D9F50E94CF58102F10386D
:10951A00B0F51A930E9472180E94A0510E94A0519D
:10952A000E943952EFE6F9E00E9464510E94DC5B26
:10953A000E94E55B0E948938E2E7F9E00E946451E3
:10954A00E9EAFDE0FA93EA93E1E00E94A55B09F4F7
:10955A0084C00E94E55B0E943952E8E7F9E00E9464
:10956A006451EAEAFDE0FA93EA93E7E00E94A55B18
:10957A0009F473C01A930E94A4181F5FC8CF31322E
:10958A0011F0103808F001C084CF67C00E94CE5194
:10959A000E94A15B0E94A0510E948938EEE7F9E07F
:1095AA000E94645110E01830E0F41A930E94B01837
:1095BA000E94A0510E943D520E94C15BE091A40DFD
:1095CA000E94E95BE091A70D0E94E95BE091A50D7D
:1095DA000E94E95BE091A60DEA930E9438431F5F5F
:1095EA00E2CF0E94A4440E2F0D34B9F50E94CF5841
:1095FA0010E0183090F51A930E94B0180E94A051FA
:10960A000E94A0510E943952E1E9F9E00E94645196
:10961A000E94DC5B30E03430D8F40E94E55B0E94A3
:10962A003952A6E13A9FF001E05DF94F0E94645178
:10963A00E8E0F0E00E94CC5B0E94CC38A6E13A9FB9
:10964A00F001E05DF94F0E94ED5B39F03F5FE3CF37
:10965A001A930E94C8181F5FCCCF0E94605F24969D
:10966A0008951A930A930E94D0380E949D0600E03A
:10967A00053210F00C94074C0E9444050E94A05138
:10968A000E94A0510E9489380E94F75B31960E947D
:10969A0064510E94D05BE8E0F0E00E94CC5B0E943B
:1096AA00F75B0E947E54A9F40E9419531E2FEDB74E
:1096BA00FEB7FA93EA931F93E0E1EA9373DB1F91F3
:1096CA00E13209F49FC0E12FA1E0B0E00E94B75D4A
:1096DA0095C0E238A0E0FA07A9F40E94DF541E2FD1
:1096EA00EDB7FEB7FA93EA931F93E0E1EA935ADBE8
:1096FA001F91E13209F486C0E12FA6E0B0E00E9492
:10970A00B75D7CC0E138A0E0FA07E1F40E94E454B6
:10971A001E2FEDB7FEB7FA93EA931F93E3E0EA939D
:10972A0041DB1F91E13209F46DC00E9444050E9499
:10973A00E454E11731F0E12FA0E0B0E00E94B75DF8
:10974A00FFCF5CC0309749F40E94F75B0E94FD5B33
:10975A00A0DAE13209F456C051C0E130A0E0FA07BC
:10976A0039F40E94F75B0E94ED5B09F44BC046C0D6
:10977A00E230A0E0FA0769F40E94F75BDF010E9479
:10978A00FD5BFD017296E491EA9365DBE132D1F16A
:10979A0035C0E330A0E0FA07D1F40E94F75B729675
:1097AA000E94905DABE0B0E0AE1BBF0BBA93AA93E8
:1097BA000E9473510E94F75BDF010E94FD5BFD016D
:1097CA007296E491EA93A8DAE132E1F017C0E43044
:1097DA00A0E0FA0799F40E94F75B3E960E94905D1A
:1097EA00E0937A10F0937B10FA93EA930E94F75B66
:1097FA007296E491EA93A0DBE13221F00E946517A8
:10980A000F5F36CF0991199108951A930E94D038A3
:10981A000E949D060E94470510E0133050F50E94F1
:10982A00A0510E94A0510E943952E12F0E94A058D3
:10983A00ECE1F9E00E9464511A93FADB0E94E55BBD
:10984A000E94BC5BE17049F40E94CA570E94CE5440
:10985A000E94AA5B09F4C2C20AC00E94CA570E94A7
:10986A00CE540E948856F7DAE13209F4B7C21F5F74
:10987A00D4CFB4C20E94595F10E01A930E941F59B4
:10988A000E94A15B0E94A0510E94C15B0E94C0522B
:10989A000E94B15200E0033060F5E4E0F0E0FA9390
:1098AA00EA93E02FEE5F0E9411520E948938E02F5E
:1098BA000E94A058EAE3EA930E94FA380E94D05B19
:1098CA000E94005851F40E9408580E944A520E946D
:1098DA0051520E941443E3E707C00E9408580E94AD
:1098EA004A520E94CA52E9E4EA930E94FA380F5F88
:1098FA00D2CF0E94A4443E2F3B3211F4103408F018
:10990A0001C01F5F3D3211F4113008F401C011503B
:10991A003D3439F41A930E94191877DF1A930E947A
:10992A003918313209F0A9CF0E94605F0C94255191
:10993A000E94CF580E94A0510E94A0510E948938CB
:10994A00E4E9F9E00E946451E1E0E0939B09EBE964
:10995A00F9E0FA93EA93E5E0EA9324DA0895229784
:10996A000E94575F0E94A4440E2FE0919309E030B1
:10997A0011F00C945D4E0132D1F4EAE0F5E0A091C9
:10998A00AF0DB091B00DEA17FB0761F4E7E0E09381
:10999A009009EAE2EA93EDE9F9E00E9488560E940A
:1099AA005C40D8C1E0E0E09394070E94035C0D3369
:1099BA0031F4E0919407F0E00E94005204910D34D2
:1099CA0041F4EAE2EA93E0EAF9E00E9488560E944A
:1099DA005C40063449F4E0ECF5E0E093AF0DF09317
:1099EA00B00DE0E0E0939407003311F00B3229F454
:1099FA00E0919407EF5FE09394070D3229F4E09128
:109A0A009407E150E0939407013329F491DFED3391
:109A1A0011F40E940A5C033321F48ADFED3309F45E
:109A2A0050D8063321F4E0E0E0939B094AD8043386
:109A3A0029F4E0E0E0939B090E940A5C093411F4DE
:109A4A000E944E05A0919D09A13010F40C94F24D8C
:109A5A00023311F56DDFED33F9F40E94175C0E2F16
:109A6A000D33D1F4E0919B09EA930E942D1A30E05C
:109A7A00303190F40E94E3510E945C5659F4E32F6E
:109A8A00E05DEA93E3EAF9E00E946156E0E3EA93D3
:109A9A000E947F403F5FECCF053341F5E0E0E09361
:109AAA009B090E94175C0E2F0D3301F511E0163049
:109ABA00E8F41A930E942D1A30E03031A8F40E947B
:109ACA00E3510E945C5671F4E32FE05DEA93E3EA06
:109ADA00F9E0FA93EA93E12FE05DEA93E0E3EA938F
:109AEA000E947F403F5FE9CF1F5FE1CF013451F40D
:109AFA00EAE2EA93E6EAF9E00E944359E1E0E093F8
:109B0A00900928C10A3409F4B5DE073311F00C9420
:109B1A00F24D0E94D038E0E0EA930E94DD05E1E0D0
:109B2A00E0939409E0E0F0E0E0938C09F0938D096A
:109B3A0030E0383030F40E94E3510E9434573F5FDE
:109B4A00F8CF0E94AC0CEE83FF830E941B5CEEE10F
:109B5A00F0E00E949858E03031F00E9496050E9489
:109B6A00AC0CEE83FF83E5E0F0E0FA93EA930E94FF
:109B7A00C04440E050E00E94C75894F0E09150077A
:109B8A00F0915107EF57F0403E2F313010F031314C
:109B9A0008F006C0E32F0E9402570E94905DAF01B1
:109BAA0040938C0950938D090091B007E0E0E0934F
:109BBA00B007013211F00B3209F401C0C6CF0B32E3
:109BCA0021F4E1E0EA930E94DD05013209F0B0CF09
:109BDA00E0E0E0939409E093B007A0919D09A230D8
:109BEA0011F00C94564E093309F43BDD053409F49F
:109BFA00CDDC033611F40E944305083309F4ADDBCA
:109C0A00023409F443DC0334A9F51091AE0D0E9425
:109C1A00D03800E0E091AD0DE11711F0063008F000
:109C2A001CC00E94A0510E94FD510E94915B1A9390
:109C3A000E949C1D1A930E94D45BE0919E0D0E9483
:109C4A00E95BE091A10D0E94E95B0E94DC560E944B
:109C5A00CA520E94CE560395DDCF0E9447050E9444
:109C6A00A4440E2F013221F0E091AD0DE11709F461
:109C7A0001C0CDCF0434A9F40E94175C0E2F0D3316
:109C8A0081F4A0914B0DA03021F4A091490DA03090
:109C9A0031F00E94B3530E94A0510E9423380E94BF
:109CAA00251CE0919309E03011F40E943C064DC056
:109CBA00E130B9F4A0919A09AB3010F4013209F4F9
:109CCA0005C00E941A090E9447050AC0E0E0E09315
:109CDA0097090E94205C0E94295CE2E0E0939309C4
:109CEA0034C0E23091F5013269F4E0E0E09393097F
:109CFA000E94D038EAE2EA93E0EAF9E00E94435986
:109D0A000E943C060B3281F4E0919709ED5FE093E3
:109D1A009709A0919709A03418F0EDE3E093970909
:109D2A000E94205C0E94295C0D3279F4A091970967
:109D3A00A63020F0E0919709E35001C0E0E0E093FB
:109D4A0097090E94205C0E94295CA0919009A33087
:109D5A0009F408CE0E945E5F289608951A93E3E0FC
:109D6A00E09391090E945A51ECEAF9E00E94645189
:109D7A000E94A0510E947351E2EDF7E00E948856BA
:109D8A00E0E1F0E00E948D5610E0E091410D1E17CF
:109D9A00E0F4E12FE05DEA93E4EBF9E0FA93EA9369
:109DAA00E0E3EA93E0E00E94685649F40E945652C2
:109DBA00EE52F84FA1E0A083E12FE05D01C0EEE290
:109DCA00EA930E94FA381F5FE0CF0E94035CE0E04A
:109DDA00E0939407E09393090E943C061991089531
:109DEA0099818881009641F0BD81AC81FB81EA812D
:109DFA0005900D920197E1F7FD81EC810C94535186
:109E0A00B981A881109631F0FC81EB816A81619356
:109E1A001197E9F7EB81FC8125960895E991F9916B
:109E2A00A991B9911D900590011421F40020D1F750
:109E3A00EE2708951018E1F3E1E008F4E2500895DE
:109E4A00E991F991A991B991CD0161916D93662337
:109E5A00E1F7FC010895E991F991A991B991CD0130
:109E6A0005900D920020E1F7FC010895A991B9919E
:109E7A00EE27FF276D91662311F03196FBCF0895E7
:109E8A00AA27BB27E991F9910590002011F01196B4
:109E9A00FBCFFD0108955D9BFECFE881ECB92196C9
:109EAA0008951A930A93AC81BD810E94815D30970F
:109EBA00C1F0AA81BB810E94815D8F01309749F070
:109ECA000230E0E01E0760F0F80131978F01ED9350
:109EDA00FC93AC81BD810E947F523197AE81A083F1
:109EEA0003C0EE81EA93D7DF198108812796089586
:109EFA0026970E94575F10E0EA89FB893196EA8B20
:109F0A00FB8B3197E4912E2FE03011F40C94A6507C
:109F1A00E12FE03039F4253211F411E002C00E9439
:109F2A00305C0EC1E130A9F4253219F40E94305C8C
:109F3A0006C112E040E000E02D3211F401E000C158
:109F4A002B3211F44BE2FCC0203211F440E2F8C08B
:109F5A0002C0E23039F450E013E0203311F4006813
:109F6A00EFC004C0E33011F00C94A550203310F078
:109F7A002A3308F009C0A52FEAE0EA9FF0015E2F14
:109F8A00E22FE0535E0FDCC0E22FE33649F40E9471
:109F9A003B5CE889F989A481AA930E94415CCFC0FD
:109FAA00E33741F40E943B5C0E944B5C0E943B4FAA
:109FBA001E2F0AC0E03761F40E943B5C0E944B5C92
:109FCA000E94454F1E2F086002600F7730E035C0AF
:109FDA00E43611F0E93611F4046002C0E53731F4D1
:109FEA00E0EBF6E0EE83FF8315E00DC0E83511F4EF
:109FFA00086004C0E83711F00C94A450EAEBF6E0CC
:10A00A00EE83FF8314E002FF14C00E943B5C0E94AF
:10A01A00535CAB85AA233AF4EA85FB850E94815CEE
:10A02A00EA87FB874DE2403011F01F5F01C00B7FCA
:10A03A0004C00E943B5C0E94535C00FD11C01517CE
:10A04A0078F407FF08C002FF04C00B7F242F1150C9
:10A05A0001C020E301C020E20E94305C5150EFCFE2
:10A06A00312F01FF17C03030A1F003FF05C00E9455
:10A07A0036533197E49105C0AE81BF81ED91AE832D
:10A08A00BF83EA930E94415C503009F0515031502D
:10A09A00EACF4BC020E3EE81FF810E94905DE88702
:10A0AA00F987EE81FF813296EE83FF83E885F98591
:10A0BA00AA85BB85AE17BF0750F02F5FA885B98563
:10A0CA00EA85FB85EA1BFB0BEA87FB87EFCF2A337E
:10A0DA0028F003FF02C0295F01C0295D04FD1AC0F0
:10A0EA00213320F4A885B985119709F409C05317BB
:10A0FA0010F000FF01C013C020E207FF0BC020E3ED
:10A10A00006102FF07C00B7F4A930E94415C5030F6
:10A11A0009F051500E94305C503009F051503150D2
:10A12A00A885B985129708F0B5CF00FF08C050304E
:10A13A0031F05150E0E2EA930E94415CF8CF10E01E
:10A14A00DBCE0E945E5F64960895FF92F82E2297F6
:10A15A001A930A93DE010E94785C8D01DE0116963D
:10A16A000E94785C0E94815DEA83FB83DE0114967B
:10A17A000E94785C0E94E9541A930A93FE0136966B
:10A18A000E94C351B5DEAA81BB81E0E0EC9319813C
:10A19A0008812496FF9008957B816A81F981E8817C
:10A1AA0077FB770F67FD7160972F9E5781F078F0E4
:10A1BA00983190F4AA27BB27882708948795B795E2
:10A1CA00A7959A95D1F7EA23FB23682305C0E8945B
:10A1DA007727EE27FF2766276F77769508F460685A
:10A1EA0077F9A991B99189919991EA17FB076807BB
:10A1FA00790797FB08950E94EC5A0E945B5C19F458
:10A20A000E94625C1DC0E6F7A881B9818A819B81A0
:10A21A00E0E0F0E060E87FE30E94555311C00E943D
:10A22A00EC5A0E945B5C19F40E94625C09C0E6F376
:10A23A000E94625CA0E0B0E080E89FE30E94685E52
:10A24A00249608950E94675C0E94495F39F4A881A8
:10A25A00B9810E944E560E948B5D20C0AA81BB81A3
:10A26A008C819D810E94515F34F40E94675C0E9438
:10A27A00945DC1DF05C00E94675C0E94945DCFDFD8
:10A28A00A881B9810E948B5DA881B9810E94855DF0
:10A29A00AA81BB818C819D810E945553269608957F
:10A2AA00EA93E0E0EA930C94A9380E94D038E0E0FF
:10A2BA00F0E0FA93EA93FA93EA930C948938FA93C2
:10A2CA00EA930C9424390E94AB5DEF5FEA930E94F3
:10A2DA003843E0E0F0E0FA93EA930895E1E0F0E031
:10A2EA00FA93EA930C948938E2E0F0E0FA93EA935D
:10A2FA000C948938E3E0F0E0FA93EA930C948938F5
:10A30A00EA930E943843E0E0F0E0FA93EA93089572
:10A31A00E4E0F0E0FA93EA930C9489380E94F0069C
:10A32A000C94A444EFEF0E94B75DE2E3F0E0FA93E5
:10A33A00EA930C946C5CE0E0F0E0FA93EA930895F7
:10A34A00A7E0B0E00E94AB5DF0E00895E081EA93F7
:10A35A000C943843FF27662777270E94945D84E090
:10A36A000E94AA5028960895EA93E2E0EA93EBE065
:10A37A00EA93E0E0EA93E1E0EA930895FA93EA9334
:10A38A00DACFEA93ECE0EA93E0E0EA93E1E0EA93D9
:10A39A0008950E94595F0C94D038EA93E4E080CF84
:10A3AA00E491EA93E1E0EA93EBE0EA93E0E0EA93EE
:10A3BA000895EA93E1E2EA93E1E0E3CFE32FF0E0E4
:10A3CA000895A091AF0DB091B00DBD01AEE0B0E01F
:10A3DA000E94B95CE60FF71F0E94905D30970895BE
:10A3EA00A0919407E3E0EA9FF001EF5F0E2F089532
:10A3FA00E02FF0E00895A091AF0DB091B00DBD012E
:10A40A00AEE0B0E00E94B95CE60FF71F0895E1E004
:10A41A00F0E0FA93EA930895F0E0FA93EA93089544
:10A42A00AEECB8E0E42FF0E00E94995C08950E9437
:10A43A001918E2E0FDE0FA93EA93EAE0EA930C9451
:10A44A004439E2E3F0E0FA93EA930E94C04473CFFE
:10A45A00E881F981FA93EA930895E0915007F0911F
:10A46A005107EF73F07008950E9489380C94CC3824
:10A47A00E12FEF5FD1CFE6E0F0E0FA93EA93F8CF6D
:10A48A00E02FAEE2B8E0F0E00895EE0FFF1FAE0F46
:10A49A00BF1F0E94815D08950E94A95C0E94945D7D
:10A4AA000895E12FF0E00895F0E0E0934E07F0936D
:10A4BA004F070895F0E0E0935007F093510708958D
:10A4CA00E0E0F0E0E0934E07F0934F07E093500787
:10A4DA00F093510708950A921A92FA926A937A931C
:10A4EA008A939A93AA93BA93EA93FA93EFB7EA9361
:10A4FA001A930895ED91FD913196FE93EE93089586
:10A50A00E4EFF1E0FA93EA930895ACE01A9FF001C0
:10A51A00E050FB4FE0810895E1E0EA930C94BF38E4
:10A52A00E2E0EA930C94BF38E1E0E093F305E093AC
:10A53A00F4050895E091A209F091A3096091A40994
:10A54A007091A5090E94945D08950E944A18EBE251
:10A55A00FDE0FA93EA930895EAE0EA930C94443909
:10A56A00AEE2B8E0F0E00E94995C0895AE0FBF1F1A
:10A57A000E94855D0895E2E0FDE0FA93EA9308956A
:10A58A00E091930DF091940D0895FA93EA930C9447
:10A59A001B43E091950DF091960D6091970D709186
:10A5AA00980D0895EF5F0E94B75DE150EAE0F0E090
:10A5BA00FA93EA930C946C5CE0918A09A9E0EA9F09
:10A5CA00F0010895A083E0918A09EA930E940F306E
:10A5DA00E0938A090895E5E0F0E0FA93EA930C948F
:10A5EA008938E1E0EA930E943C05E2E3F0E0FA935D
:10A5FA00EA930E946C5CE0E0EA930C943C05FA93BF
:10A60A00EA930C946C5CE1E0EA930E943C05E4E670
:10A61A00F0E0F5CFE0E0EA930E943C05E4E6F0E0E2
:10A62A00EECFE4E6F0E0EBCFA1E0B0E00E94AB5D54
:10A63A000895EA930E942A0BE0300895E091710090
:10A64A00E87F1E2F0895E0937300E4E8F2CFEA93BF
:10A65A000E94F70AE03008950A930E94030BE03043
:10A66A000895EE81FF813196EE83FF830895FF27D7
:10A67A00662777270E942E5E0895EE8DAE85BF85E8
:10A68A0088899989F4DF0E94B65EA9A1BAA18827B0
:10A69A0099270E949B5D0E949E5D0E94615E0895BB
:10A6AA000E949E5D0E94615E0895AE0FBF1FEC91ED
:10A6BA00EA930895F0E0EA17FB070895AC81BD819B
:10A6CA00EA0FFB1F08950E94C03EECE2EA930E9443
:10A6DA008E3EBECE0E94C03EEBE3EA930C948E3EC1
:10A6EA00A091D80CB091D90CAC910895A091D80C36
:10A6FA00B091D90CEC910895EA930E948E3EA8ED90
:10A70A00BCE0F8CEE091AC0DA091AB0DEA1708952C
:10A71A00FA93EA930C949F3EE0919C0DF0919D0D63
:10A72A00FA93EA930895A0919A0DB0919B0D08951A
:10A73A00F0E0A4E6B0E00E94E15C0895E0939A0D8F
:10A74A00F0939B0D0895EBE3EA930C948E3EA0914F
:10A75A00D60CB091D70CE0E0EC930895E0E0EA93D0
:10A76A00EACDEE81FF81E0939C0DF0939D0D10934D
:10A77A00990D0E94641BE1E3089541E050E00E94B4
:10A78A00DD3DE887F987EAE3EA930E946E3DE1300E
:10A79A000895FA93EA930C94C7171A93E985FA85F0
:10A7AA00FA93EA935A934A930895E0918809A9E0A3
:10A7BA00EA9FF0010895A885B985A083B183089519
:10A7CA00DF01EA85F0E0ED93FC930895E0918809B2
:10A7DA00EA930E940F30E093880908951A93E98555
:10A7EA00FA85FA93EA930895A091A10DB091A20D6A
:10A7FA000895E091A10DF091A20D0895E093A10DA5
:10A80A00F093A20D0895EA85F0E00895FA93EA9389
:10A81A000C942338E0918B09A9E0EA9FF00108958E
:10A82A00E05DEA930C948E3EE2E2EA930C946E3D6C
:10A83A00A8EDBCE05FCE0E94C03EEAE3EA930C9426
:10A84A008E3EFA93EA9346CFEAE3EA930E946E3D7C
:10A85A00E13008950E94DD3DE058FF4F0895EA93E4
:10A86A000E9419180E94501EE8310895EFEFE093F4
:10A87A00D00CE093D10C0895E0E0E093B70DE0939B
:10A88A00B80D08950E94DD3D3197E093B80CE09130
:10A89A00D10CA091B80CEA1708950E945710E091C4
:10A8AA00B80CEA930895E091B80CE093D10C08959E
:10A8BA00E091B80CF0E0E25DF74F0895ECE2EA931C
:10A8CA000E946E3DE0300895E454F34FA0E0A08367
:10A8DA000895EA930E946E3DE1300895A6E11A9F19
:10A8EA00F001E854FF4F0895ECEBFCE0FA93EA9389
:10A8FA00089570960E94905DE038A0E0FA070895E6
:10A90A003E960E94905DE093B50DF093B60D0895C2
:10A91A0072960E94905DA02FB0E0AE17BF0708950F
:10A92A00ACE00A9FF001E450FC4F0895A5E1BDE0B8
:10A93A00E091B90CF0E00895A8E1BDE0E091B90C0E
:10A94A00F0E00895E091B90CEF5FE093B90C089537
:10A95A00A1E2BDE0E091B90CF0E00895ABE1BDE001
:10A96A00E091B90CF0E0EE0FFF1FEA0FFB1F08950C
:10A97A00A2E1BDE0E091B90CF0E00895AE0FBF1F6F
:10A98A00EC91E160D001EC930895E091B90CF0E00C
:10A99A000895EE0FFF1FEA0FFB1F0895FA93EA933B
:10A9AA000C94D80CE091B80CA6E1EA9FF001E854A7
:10A9BA00FF4F0895A6E0B0E00E94AB5D0895A0E0C5
:10A9CA00B0E00E94AB5D08950E94815DFA93EA931C
:10A9DA000895A12FB0E00895EE27A10FBE1FEC91B4
:10A9EA00D001EC9308950E94C03EECE2EA930C94E5
:10A9FA008E3EECE2EA930C948E3EE091100DE295C5
:10AA0A00EF700ACD0E94CD0CE0E0E093B90C0895F6
:10AA1A00FA93EA930C94533FAE0FBF1FEC91FCCC10
:10AA2A00E0910D0DF0910E0D089584E00E94AA5058
:10AA3A0028960895E091240DF091250D0895A0918E
:10AA4A00A90DE1E0EA23E8CC1A93E8EBFBE0E093F6
:10AA5A00D60CF093D70C0895E8EBFAE0E093D80C03
:10AA6A00F093D90C0895E091D80CF091D90C08957F
:10AA7A00A6EDBCE03FCDA091D60CB091D70CEC93DB
:10AA8A00F7CFA091D80CB091D90C0895E093D80CC7
:10AA9A00F093D90C0895A091D60CB091D70C1397C6
:10AAAA000895E0E0EA930E942C0DE093AD09089521
:10AABA00E091B109EA930C941040EEE0EA930C9409
:10AACA008E3E1A93E0EAEA93EA81F0E0E054F14F0D
:10AADA00FA93EA930E94450B1E2F0895E0EAEA933F
:10AAEA00EA81F0E0E054F14FFA93EA931A930C9456
:10AAFA00740BE0EAEA93EBE5F0E0FA93EA93E0E01C
:10AB0A00FFE0FA93EA93E6E3FDE00895FA93EA9305
:10AB1A00E0E2EA930C94000CE0EAEA93E981FA8114
:10AB2A00E050FE4EFA93EA930895EA81F0E0A8E233
:10AB3A00B0E00E94E15C0895E0EAEA93E2E0F0E026
:10AB4A00FA93EA931A930A930895FA93EA930C9460
:10AB5A00950BE0EAEA93E8E2F0E0FA93EA931A93B3
:10AB6A000A9309CDEDE2EA93EAE0F0E0FA93EA9378
:10AB7A000E94054FE0E00895EA81F0E0ABE0B0E022
:10AB8A000E94E15CE050F24F8F01AA81AA30089539
:10AB9A00E0EAEA93EBE0F0E0FA93EA931A930A9375
:10ABAA00EAE2FDE00895EA81F0E0EE0FFF1FE050CF
:10ABBA00F04F8F01AA81A0380895E150F0E008957E
:10ABCA00EA81F0E00E94995CE058F14F8F01AA8176
:10ABDA00A8300895E0EAEA93E4E0F0E0FA93EA9311
:10ABEA001A930A93E4EAFDE00895E4EAFDE0FA9391
:10ABFA00EA93E0E0EA93E4E0F0E0FA93EA930C9453
:10AC0A00054FE1E9FDE0FA93EA93E0E0EA93E8E030
:10AC1A00F0E0FA93EA930C94054F0E94995C0E9423
:10AC2A00955CDF01F0CDAE0FBF1FE8E0F0E00E94B7
:10AC3A00E15CE050FA4E8F01E0EAEA93E8E0F0E0E6
:10AC4A00FA93EA931A930A93E1E9FDE07ECFE0933F
:10AC5A00950DF093960D6093970D7093980D089546
:10AC6A00F0E0AE0FBF1F0895EA93E8E0F0E0FA9330
:10AC7A00EA930895F0E0EA0FFB1F0895E091A00916
:10AC8A00F091A1090895E0939C0DF0939D0D0C9409
:10AC9A00641BE0E0F0E060E070E00895E093A20950
:10ACAA00F093A3096093A4097093A5090895EE523D
:10ACBA00F84FE081E1300895FA93EA93E0919B0915
:10ACCA00E05DEA930895EA930E947F40E130089597
:10ACDA000E94995CEA0FFB1F0895FA93EA93E8E051
:10ACEA00F0E0FA93EA930E94F54EA881AF5FEAE09A
:10ACFA000E94EB5CE05D0895A881AF5FEAE00E94E4
:10AD0A003B5DE05D0895FA93EA93E0E0EA930895E3
:10AD1A00FA93EA930C94054FEA930E94FA3810E0EA
:10AD2A0008957496E491D901EC930895E881F0E0CE
:10AD3A00A5E0B0E00E94E15C0895E0EAEA93E5E06C
:10AD4A00F0E0FA93EA930895EA930E94591BFA9362
:10AD5A00EA93E9E9FDE00895FA93EA93EFEFEA93BB
:10AD6A00E5E0F0E0D5CF0E94A45DEA1BFB0B089555
:10AD7A00A0919F0DB091A00D0895E0E0E093AD0D74
:10AD8A00E093AE0D0895E0E0E0939E0D1A930C94C3
:10AD9A00AA1D1A930E94EF1B1E2F0895E0939F0D80
:10ADAA00F093A00D08951A930E949C1D1DCDE09169
:10ADBA009F0DF091A00D0895EA930E949C1D0E9498
:10ADCA00401DE0300895E881EA930E94EF1BE88372
:10ADDA000895EB81EA930E94161CFA93EA93EEE92E
:10ADEA00FDE00895E0E0E093C00DE093BF0D089503
:10ADFA00EE0FFF1F0E94955C0895ACE8B0E0F0E00A
:10AE0A00C8CD0E94905DA0918E09B0918F09EA2B5E
:10AE1A00FB2BE0938E09F0938F090895A1ECBDE016
:10AE2A00F0E00895AEE1B8E0F0E00895EE0FFF1FFC
:10AE3A00AE0FBF1F0895EC93EC81E150ACE0EA9F9E
:10AE4A00F0010895E55FFA4FBF01E0810895E091AE
:10AE5A00F007B3CEE093F407F093F507F8CFE95182
:10AE6A00F84FA0E0A0830895A0914E07B0914F0734
:10AE7A000895A2E1BDE0E09192090895A5E1BDE03F
:10AE8A00E0919209F0E011CCE0919209F0E0089586
:10AE9A00AEE2B8E0F0E00895AEEAB8E0E52FF0E0FF
:10AEAA000895E951F84FE081E5CEE250F84FE0818C
:10AEBA00EA930C94911EED93FC93F3CA1396ED91C9
:10AECA00FD913197FE93EE9308950A930E94821E94
:10AEDA00E0300895A885B985EC91C6DFEBCB1396CF
:10AEEA00E0E0F0E0ED93FC930895BD01A9E0B0E045
:10AEFA000E94B95C0895E0E0F0E0ED93FC930895B8
:10AF0A00EE81FF81A181AA930895E12FA1EDBDE011
:10AF1A00F0E08CCFEE57F14EE491E0300895A88529
:10AF2A00B985EC91EA93E3E0EA930C949044A885FE
:10AF3A00B985E0E0EC93E2E0E093E3070895AE819F
:10AF4A00BF8117960E94815D30970895ED91FD911A
:10AF5A003197FE93EE930895E55AF64FEA87FB87F9
:10AF6A00AA85BB8511960895E0918A09EA930E9401
:10AF7A000F30E0938A090895F0E0ED93FC93089569
:10AF8A00E12FA6E0B8E0F0E00895ABE1BDE089CAA0
:10AF9A00A5E1BDE0EE27A10FBE1FEC910895EA934B
:10AFAA000E94C71EE0300895A8E1BDE0EE27A10F78
:10AFBA00BE1FEC910895E081EA930C94773AE8EB8E
:10AFCA00FBE0E093D60CF093D70C0895EA930E9425
:10AFDA008E3EE0E0EA930C948E3EA5E1BDE0EE27BA
:10AFEA00A00FBE1FEC910895A8E1BDE0EE27A00FC7
:10AFFA00BE1FEC910895A2E1BDE0EE27A00FBE1F8F
:10B00A00EC91E1700895ABE1BDE0F2C9A1E2BDE0C7
:10B01A00EE27A00FBE1FEC910895ACE0EA9FF00165
:10B02A00E75FFA4F0895ABE01A9FF001E954F84F31
:10B03A000895ABE01A9FF001EF54F84F0895AFEF6F
:10B04A00BFEFA083B1830895ABE00A9FF001EF54EC
:10B05A00F84F0895ABE00A9FF001E954F84F0895BC
:10B06A00FE013596FA93EA930895AFEFA083A6C935
:10B07A00E091FE0DF091FF0DFA93EA9308950E9474
:10B08A00AC0CE093FE0DF093FF0D0895FA93EA934A
:10B09A00E0E0F0E8FA93EA930C942D07FA93EA9326
:10B0AA00E091FA0D0895E55AF64FFA93EA930E9451
:10B0BA003A275ACFE0919A07EA930C944824EE89EA
:10B0CA00ABE0EA9FF0010895FA93EA9391C9E091FF
:10B0DA00FA0DEA930E94E9171E2F0895CFDDFA931D
:10B0EA00EA930895E093FA0DE0E0E093FB0DE1E3C3
:10B0FA00E093FC0D0E946D280C94FF230E94AC0C77
:10B10A00E093BB0DF093BC0D0895C0DCE3E0EA9335
:10B11A000C94083EE3E0EA930C94083EE093A009FD
:10B12A00F093A1090895FA93EA930C94B80CE1E01C
:10B13A00E093F40500C9EF5CEA930C94FA38E7E06F
:10B14A00E0939009EA930ACBEA930E94B5420E94DF
:10B15A00A4441E2F0895EAE2EA93E4E3F8E0D3CD8B
:10B16A000E947029E1E0EA930C944629E05DEA9393
:10B17A000C945C401F771A930E941918E091110DE4
:10B18A00E0300895A0915007B0915107A038E0E04F
:10B19A00BE0708950E94D0380C949A06E0E0F0E0C9
:10B1AA00E0939E09F0939F090895E091F805E55010
:10B1BA00F0E0E4C8E0919E09F0919F09E6C9E091A8
:10B1CA004207F09143070895FA93EA930C9487385B
:10B1DA00A0919E09B0919F090895E8EEF3E00E94BC
:10B1EA003E5D0895A0E024FCA1E0A0300895E0911E
:10B1FA00AB09F091AC09FA93EA9308950E94AC0C5A
:10B20A00E093AB09F093AC090895E0E0E093BF0D39
:10B21A000895DEDFEA17FB070895E0939009E0E05E
:10B22A00E093A90908950E945C400E94D92AE093FC
:10B23A009D0908950E9419180C94D038E09191093B
:10B24A00EA93E0E0EA930E94922A0E94ED260E9485
:10B25A00A144E03008950E94A4441E2F1A930E942C
:10B26A00092B103808951A93E0919A07EA930895E2
:10B27A00E091B409E053E0939B090895FA93EA93A5
:10B28A00E0E3EA930C945C40E0919109A091900963
:10B29A00EA170895E89423F8E0E0F0E03FDF0A9324
:10B2AA00E1E0EA930C94922AABE00A9FF001EE5493
:10B2BA00F84F0895A083ABE00A9FF0010895ABE030
:10B2CA000A9FF001EC54F84FA1E0A0830895FA9385
:10B2DA00EA93EAE7F8E0FA93EA93EA85ABE0EA9FB1
:10B2EA00F0010895AC81BD81EE27A00FBE1F08951D
:10B2FA00EE27A30FBE1FEC91D001EC930895AEEC9C
:10B30A00B8E00C94E351E32FA0919709EA0FEA936E
:10B31A0008951A930A93E091B80BE0300895E8541F
:10B32A00F44FE081E0300895E854F44F44CEE854F5
:10B33A00F44FE0810E0F1F5F0895E0918909A9E09B
:10B34A00EA9FF0010895E3E0F0E0FA93EA930E949D
:10B35A00EB3EF3CFE0E0EA930E948E3E0C94163364
:10B36A000E94815DF096EA930E941040E2E7EA9318
:10B37A000C948E3EE081EA930C948E3EEEE7F8E060
:10B38A00C7C95A934A930E94C7170E2F00340895CB
:10B39A00E2E5EA930C948E3E1A93E091B109E053E8
:10B3AA001E2FE5EBF9E072CBE0918A09A0918B0997
:10B3BA00EA170895E0918B09EA930E940F30E0930F
:10B3CA008B090895A091EC0CAF5FEAE00E943B5D07
:10B3DA00E093EC0CEAE2EA930E941040D9CFE091A4
:10B3EA00EC0CE05AEA930E948E3E67CBD901149680
:10B3FA00EC910C941152F901A281B381BA93AA93E8
:10B40A000895D9011196E0E0EC930E942C40D2CF26
:10B41A00E4E5EA930C948E3EEC91EA930C948E3E0A
:10B42A00EC91F0E00895EA930E941040B1CF0E9497
:10B43A002C400E94AC0CE093010EF093020EE2E065
:10B44A00E093AE09D9011196EC930E94605F0895CA
:10B45A00E881EA930C948E3EAF5FEAE00E943B5D7E
:10B46A000895E295EF70EA930E949D0C1E2F0895AD
:10B47A00EF70EA930E949D0C0E2F1A930E948E3E43
:10B48A000A930E948E3EE7E10895E0915707EA93F6
:10B49A000C944638E3E5EA930C948E3EA2E4B7E0B6
:10B4AA000C947F52A981BA81EE27A10FBE1F08957D
:10B4BA00F801AA81BB81EA0FFB1FE4910895D80124
:10B4CA00F0E0AE17BF070895FE013696FA93EA93A5
:10B4DA000895AA81BB81EC91E295E07FAE2FEC81C1
:10B4EA000895EA0FAA81BB81EC93A881B981EC91F6
:10B4FA00EF5F0895E091A20EA091A10EEA170895B8
:10B50A00E091B30AF0E0E854F54F08951083E09112
:10B51A00B30AEF5FE093B30AE12FA091B50A089549
:10B52A00E093B50AE091B40AE150E093B40AE0303E
:10B53A000895E854F54FA0E0A0830895E0916D0FB7
:10B54A00F0916E0F0895A0916B0FB0916C0FEA17EE
:10B55A00FB070895E12FA091720FEA0FE093720F93
:10B56A00E091740F0895F0E0E055F64F10830895C6
:10B57A00E0917910F0E0E858F04FE081E0939C0008
:10B58A00E0917910EF5FE093791008950E94595F76
:10B59A0000E010E00895D801EAE0F0E00E94E15CE2
:10B5AA000895E053F0E00895E12FA981BA8162CBB2
:10B5BA00E454F34FE081E03008952A97FE01FA93AC
:10B5CA00EA93089588E00E94AA502C960895E8818B
:10B5DA00F9816A817B810E94945D0895EA930E94B1
:10B5EA009D0CEA930C94773AEA930E946F41EAE53C
:10B5FA00E093B60A0895E6EDF4E0E0939507F09338
:10B60A0096070895E0939507F09396070895E4EC5A
:10B61A00F8E0FA93EA93AE85BF8588899989E4E6CA
:10B62A00F0E060E070E00E94365D0E94945DAA89B5
:10B63A00BB898C899D89E4E6F0E060E070E00E94B5
:10B64A004C5D0E94945DBECFFE01FA93EA930C947E
:10B65A000539EDECF8E0FA93EA93EE85FF850C9450
:10B66A005152EE27A10FBE1FEC910895EA930E9452
:10B67A00A0431F5F0895E0919807ABE9B7E0F0E0B7
:10B68A000895E0919707ABE9B7E0F0E082C9AC8191
:10B69A00BD81EE27A30FBE1FAC91A0300895ABE089
:10B6AA000A9FF001E750FA4FDF010895EA0FFB1FE6
:10B6BA000F01AC81BD811CCEA5E10A9FF001EB52BE
:10B6CA00F94FDF010895E0919507F09196070895E3
:10B6DA00A5E9B7E0ED91FD913296FE93EE930895B8
:10B6EA000E9412440C94EB430E94945D0E94084409
:10B6FA000C94EB430E941244E1E0F9E004CB40E0F1
:10B70A0050E0E02FE05DEA93E4E0F9E0D5CA109159
:10B71A004207009144070895FA93EA930C948938F2
:10B72A004EDD3197D1CC0E94A4443E2F0C94883828
:10B73A00FA93EA930C9439520E9447050C94A0514B
:10B74A00EA930E94D746E1320895FA93EA93E2E037
:10B75A00EA930E943047E1320895E6E0F0E00C9463
:10B76A00C351EA0FFB1FFA93EA93E0E1E9CF0E9483
:10B77A008938A2E1BDE075CF0E948938E12FEF5FD9
:10B78A00EA930E943343EAE3EA930C94FA38FA9371
:10B79A00EA930C947351E0E2EA930C94FA380E940B
:10B7AA003343F9CFEA23EA930E943843F4CFE12FD7
:10B7BA00EF5FEA930E943343EAE3EA930C94FA3880
:10B7CA00E8E0F0E00C94C351EA930E943843E3CFD7
:10B7DA00DF013E960E94905DFA93EA93FD0172960C
:10B7EA00E491AECFA6E10A9FF001E854FF4F089515
:10B7FA003E960E94905DFA93EA930895EAE0F5E096
:10B80A00E093AF0DF093B00D08950E949C19E0E00B
:10B81A00E0939A090E941A090E944705E1E0E09321
:10B82A00930908950E94D0380C949351EE81FF81B8
:10B83A00FA93EA930895EAE2EA93E9EAF9E0FA93D5
:10B84A00EA93E091970992CCE0919709EA930E94D2
:10B85A0064090C9447052A93EF85F889FA93EA93C9
:10B86A00FE013F96FA93EA930C94564FE889F989B8
:10B87A003497E88BF98B0895EF85F889FA93EA9360
:10B88A00FE013F96FA93EA930C94564FA889B98918
:10B89A0014960E94815DEE83FF83C8CFA889B98977
:10B8AA0014960E94815DEA87FB8708950E94D15011
:10B8BA00E883F9836A837B830895E881F9816A8141
:10B8CA007B810895EA81FB816C817D810895E991EC
:10B8DA00F991309639F080EA9FE00197F1F7A8953F
:10B8EA003197C9F708950024AF0DB01D0895EA0FE6
:10B8FA00FB1F681F791F0895F195E195F04008959F
:10B90A00F09560957095E195FF4F6F4F7F4F0895C1
:10B91A00EE230E2EEA2F19F0EE0F0A94E9F7089596
:10B92A00EE0FFF1FEE0FFF1FEE0FFF1FEE0FFF1FA1
:10B93A000895EF2FFF27E7FDFFEF0895FE2FFF0F72
:10B94A00FF0B6F2F7F2F08956F2F660F660B762FD1
:10B95A000895BA2FBB0FBB0B8B2F9B2F08958B2FEC
:10B96A00880F880B982F0895FA9FF02DEB9FF00D02
:10B97A00EA9FE02DF10D08957A9F702D6B9F700D4F
:10B98A00F89F700DE99F700D6A9F602D710DFB9FE6
:10B99A00600D711DE89F600D711D8827FA9FF02DBB
:10B9AA00610D781FEB9FF00D611D781FEA9FE02D56
:10B9BA00F10D681F781F08957ED0D6DF0EF49CDF44
:10B9CA00089587D0D9DF0EF49BDF0895002498E00C
:10B9DA00AA0F001C0E1A10F40E0E01C0A1609A954F
:10B9EA00B9F7EA2FA02D08950024112490E1AA0F97
:10B9FA00BB1F001C111C0E1A1F0A18F40E0E1F1E64
:10BA0A0001C0A1609A9599F7FD01D001089553D01C
:10BA1A00EBDF0EF471DF08953F934F935F93002499
:10BA2A0011244427552730E2AA0FBB1F881F991FEC
:10BA3A00001C111C441F551F0E1A1F0A460B570BD8
:10BA4A0028F40E0E1F1E461F571F01C0A1603A950B
:10BA5A0059F7FD01BC01D001CA015F914F913F9195
:10BA6A00089537D0D9DF0EF44BDF0895AFDFEA2F00
:10BA7A000895E894B7FF04C0A095B095119668940C
:10BA8A00F7FD3ADFB1DFFD010EF436DF0895E894E1
:10BA9A0097FF09C0A095B09580959095AF5FBF4F6D
:10BAAA008F4F9F4F689477FD2BDFB6DFFD01BC01F6
:10BABA000EF426DF0895E894F7FF02C01DDF6894AC
:10BACA00B7FF06C0A095B095119600F8039400FA46
:10BADA000895E89477FF02C013DF689497FF0BC0BC
:10BAEA000024A095B095809590951196801D901D83
:10BAFA0000F8039400FA0895ED91FC9111970895C6
:10BB0A00ED91FD916D917C9113970895ED93FD93BD
:10BB1A006D937C9308950590F491E02D08957A939E
:10BB2A006A93FA93EA930895689401C0E89401D05D
:10BB3A0091D0182E862F612D192E972F712D1B2E1D
:10BB4A00BF2FF12D1A2EAE2FE12D0895E199FECFC8
:10BB5A00FF93FFB7F894AEBBBFBBE09AEDB3FFBF4C
:10BB6A00FF910895E19B02C0A895FCCF9FB7F89476
:10BB7A00AEBBBFBBE09A8DB3E81719F0EDBBE29AF2
:10BB8A00E19A9FBF0895552342F4503811F4E0FF1B
:10BB9A0004C03196691F791F6BF050E8572711F4DA
:10BBAA005F93CDC05F3F31F0660F000C57956795E4
:10BBBA00752F08955F9300200AF0CDC0C6C050E8E3
:10BBCA00192E1522880F991F9527550F879550E82A
:10BBDA00072E0522660F771F7527550F679508955B
:10BBEA00689401C0E8945F93F2DF703818F07F3FE1
:10BBFA0008F4A5C056E1571BAAF4519558300EF423
:10BC0A00593030F0EFEFFFEF6FEF7FE777F91AC0A7
:10BC1A0077275523B9F0EE0FFF1F661F771F5A9536
:10BC2A00D1F710C07727583028F0EF2FF62F672F5B
:10BC3A005850F9CF552331F076956795F795E795E2
:10BC4A005A95D1F700200AF45BDE5F910895689453
:10BC5A0001C0E894309760407040B1F0002426F0AB
:10BC6A00772312F400944CDE172E7EE1112032F075
:10BC7A007A95EE0FFF1F661F111CF9CFEF2FF62FD3
:10BC8A00612D5F938ADF5F9108954F93AF01FD01A4
:10BC9A00DA01AB01BC01CA01402D012C142E4F91CF
:10BCAA000895EA0FFB1F681F0895E095F0956095C7
:10BCBA00EF5FFF4F6F4F08955F9381DF903871F107
:10BCCA0050E8152604C05F937ADF903839F170384E
:10BCDA0021F1572F591B13F112F4D7DFFACF58313C
:10BCEA0018F0AA27BB278827583028F0AB2FB82F7F
:10BCFA0088275850F9CF552329F08695B795A795E7
:10BD0A005A95D9F7502D512562F0CBDF38F4679553
:10BD1A00F795E795739513F41EC0B7DF3EDF5F9181
:10BD2A000895EA1BFB0B680B51F010F40094BDDF79
:10BD3A006623A2F3EE0FFF1F661F7A95CBF7EE2755
:10BD4A00FF27662777275F910895EFEFFFEF6FE7E9
:10BD5A007FEF5F910895EFEFFFEF6FE77FE75F9166
:10BD6A0008955F932CDF703851F3903841F3012422
:10BD7A000894791F23F41CF300203AF3ECCF0F92B6
:10BD8A001F932F933F934F93112722279927689F39
:10BD9A00A0018F9F302D410D591F6B9F300D411D02
:10BDAA00591F8E9F27D0BF9F25D06A9F23D0BE9F41
:10BDBA001DD0AF9F1BD0AE9F110D291F391F491FE0
:10BDCA00591FE32FF42F652F522F4F913F912F9137
:10BDDA001F910F9066232AF0550FEE1FFF1F661F53
:10BDEA0002C073954BF2CFDE5F910895100D211DAD
:10BDFA00391F02C0200D311D491F591F08955F9335
:10BE0A00DEDE703821F411200AF49FCFA4CF9038D7
:10BE1A0009F495CF01240894970B1BF4D4F300205E
:10BE2A00F3CF792F1F932F933F934F931124112709
:10BE3A00222733274427552790E2AE17BF078607E4
:10BE4A00410730F0AE1BBF0B860B410B089401C0B3
:10BE5A008894551F221F331F111CAA1FBB1F881F3E
:10BE6A00441F9A9551F7F901612D4F913F912F91F6
:10BE7A001F91662332F0550FEE1FFF1F661F7A953A
:10BE8A0043F281DE5F9108953097604070400895D3
:10BE9A0000240A160B06089500240A160B06080643
:10BEAA00090608955A934A933A932A931A930A933E
:10BEBA0008955D814C813B812A8119810881089509
:00000001FF
